:020000040800F2
:100000000050002059D9000805DA0008A9C30008EB
:1000100005DA000805DA000805DA0008000000002B
:1000200000000000000000000000000005DA0008E9
:1000300005DA00080000000005DA000899C300088E
:1000400005DA000805DA000805DA000805DA000814
:1000500005DA000805DA000805DA0008E1C2000840
:1000600005DA000805DA000805DA000805DA0008F4
:1000700005DA000805DA0008A5C2000805DA00085C
:10008000E5C2000805DA000805DA000805DA00080C
:1000900005DA000805DA000805DA0008DDC2000804
:1000A00005DA000805DA000805DA0008F1C10008E1
:1000B000E9C10008DDC10008D1C1000821C3000862
:1000C00019C300081DC3000815C3000805DA00089D
:1000D00005DA000869C20008FDC1000805DA000859
:1000E00025C3000805DA000805DA00080000000052
:1000F0000000000000000000000000000000000000
:0C01000000000000000000005FF808F1A3
:100110002DE9F04F674B684CA3B023600023636068
:1001200009F042F818B907F011FC05F07EF804F068
:10013000EBFD00230C93614D0D930E934FF4E013F0
:100140000F932B685E4943F480338A7B2B60AB6945
:100150008A4643F01003AB612B6803F400330D9320
:100160000C9B01330C930D9B1BB90C9BB3F5A06F3B
:10017000F2D12968514B11F4003101D0022315E06E
:10018000186840F0010018600C912B6803F002031E
:100190000D930C9B01330C930D9B1BB90C9BB3F57A
:1001A000A06FF2D12B68980738D501230E93454BE9
:1001B000454E196841F010011960196821F00301DA
:1001C0001960196841F0020119606B686B606B6817
:1001D0006B606B6843F480636B603C4B196821F083
:1001E000704119603A493160696821F47C11696095
:1001F000196841F000411960996821F40041996043
:100200005968090449BF334B4FF4E01333604FF48E
:1002100080130F930E9B012B01D117E0FEE7022BF9
:1002200018D16AB10F9BB3F5801F02D14FF4A01310
:1002300005E00F9BB3F5E01F02D14FF400130F93BD
:100240006A680F9B134343F4803302E06B6843F406
:1002500060136B602B6843F080732B602A68174B28
:100260009201FBD55A6822F003025A605A6842F0A4
:1002700002025A606A68114B02F00C02082A0792C7
:10028000F8D15A68DFF8548002F00C02042A03D037
:10029000082A05D00E4B00E03368C8F8003028E08B
:1002A0005A685968C2F38342CF0302F1020217D49D
:1002B000094B1BE05B2600081C07002000100240D1
:1002C000C01D002000200240140000200410014046
:1002D00000127A00001BB70000093D009C000020BE
:1002E0005B6813F4003F336818BF5B085A43C8F8D3
:1002F00000206B6822AFC3F3031333441A79D8F894
:100300000030DFF8F4B2D340AE4AC8F80030AE4B4C
:10031000AE48DA60AB69DFF8FC9243F00103AB61F1
:100320006B6A43F080736B62AB6943F01C03AB6193
:1003300000238DF85E304FF6FF7327F82C3D3946C9
:1003400002F094FE5846394602F090FEA048394625
:1003500002F08CFE9F4B5A6842F000725A6099E896
:100360000F0087E80F00AB69179843F00803AB61F3
:10037000AB6918A943F00803AB610823CBF8103030
:100380001023CBF81030039302F070FE19981AA9CD
:1003900002F06CFEAA6909F1100942F0040299E822
:1003A000030087E80300AA61D6F800908A4A039BFD
:1003B0009145934605D19DF86220142A08BF8DF817
:1003C000623018A9179802F051FED9450CBF834A34
:1003D000834A844B00201A6002F00CF9824B4FF0E4
:1003E000070993E80300AB6987E8030043F00803BB
:1003F000AB6118A9179802F039FE384605F0DCFF0A
:10040000179B7A4AF021B3FBF2F3D8F80020A360DF
:100410004FF47A73B2FBF3F2754B013A5A606A4AB1
:100420004FF0000882F823100120C3F80880C3F8B9
:10043000009005F0E9F8642006F037FCDAF808309F
:100440006C4F03F400604FF0100B069041465A4683
:1004500007F10C0003930FF054FC0422227384F87C
:100460000F90039B0221012218048DF84A108DF889
:100470004B80ADF848B0A27309D512233A747A7450
:10048000BA7487F81390ADF848300F4600E017466D
:100490003368514A93420ED1BDF84830012243F0EF
:1004A0002003ADF8483005232375A2757B1C072275
:1004B0006775E275DFB2454812A905F0C7FF069BD4
:1004C0007BB102234C4812A9ADF8483005F0BEFFBD
:1004D000092301222376A2767B1C07226776E27627
:1004E000DFB26B69454843F001036B61AB69DFF82C
:1004F0000C8143F40073AB6106F025F8404B0025F6
:100500001793404B012F18930CBF2B4680231C934D
:100510004FF480731D934FF480631E93202317A91B
:100520001F9340464FF400531A97209319951B953B
:10053000219505F0EAFFD8F80030012F43F00103C0
:10054000C8F80030304B98BF00215A6888BF01219D
:1005500022F4702222F4807242EA01225A609968E1
:100560002A4A013F0A4042F4602242F002029A60A5
:10057000DA6AFFB222F4700242EA0757DF622846C5
:100580000123234A11188D78002D00F08680825CAB
:100590005D1C092A91F803E0EDB21B493CD9A2F198
:1005A0000A0707EB47074FF0070C0CFA07FC0EFA97
:1005B00007FED1F80C8028EA0C0C4CEA0E07CF603D
:1005C00039E000BF0005FA0500ED00E00008014039
:1005D0000010014000000140001BB7004920000846
:1005E0005D200008982300202424010840420F00C9
:1005F00010E000E01C070020000C01400800024051
:100600004C2401403807002000240140FDF7F1FF91
:10061000280700200C24010802EB42074FF0070CCA
:100620000CFA07FC0EFA07FED1F8108028EA0C0C31
:100630004CEA0E070F61062B31490ED8013B03EB44
:1006400083034FF01F0E0EFA03FE9A404F6B27EA0A
:100650000E0747EA02034B6320E00C2B0ED8073B42
:1006600003EB83034FF01F0E0EFA03FE9A400F6B4D
:1006700027EA0E0747EA02030B630FE00D3B03EB8B
:1006800083034FF01F0E0EFA03FE9A40CF6A27EA4B
:100690000E0747EA0203CB6200E01D460430102833
:1006A00001D02B466DE7164B9A6842F480729A602F
:1006B0009A6842F001029A609A6842F008029A60D1
:1006C00099680F4A0907FBD4936843F004039360C9
:1006D0000B4A936813F00403FAD19168BAF8E60064
:1006E00041F4A0019160074A78B9B2F9E8305BB9EA
:1006F000B2F9EA30D3F1010338BF002305E000BFAF
:1007000000240140C01D0020034613F0010340F007
:100710008C80337500B20BF0AFFFADA3D3E900239B
:100720000CF010F80CF040FAAB4F0646B7F9E800B1
:100730000BF0A2FFA6A3D3E900230CF003F80CF002
:1007400033FA0546B7F9EA000BF096FFA0A3D3E908
:1007500000230BF0F7FF0CF027FA814630460FF02C
:10076000FFFC074630460FF06FFD804628460FF02D
:10077000F7FC064628460FF067FD054648460FF091
:10078000EFFC824648460FF05FFD394681465046F1
:100790000CF068FB3946069048460CF063FB514666
:1007A000089040460CF05EFB4946099040460CF02C
:1007B00059FB3146834650460CF054FB4946606273
:1007C00006F100400CF04EFB2946A062E562099854
:1007D0000CF048FB014608980CF03CFA29462063CF
:1007E00058460CF03FFB014606980CF031FA3146B2
:1007F000606308F100400CF035FB2946A0630698C1
:100800000CF030FB014658460CF022FA2946E06312
:1008100008980CF027FB014609980CF01BFA3946A2
:10082000206430460CF01EFB60646B4EB3689B0383
:1008300061D5142006F039FAAE2005F04AF8A4205C
:1008400005F047F8322006F030FA202005F041F894
:10085000022005F03EF8A12005F03BF8C82005F085
:1008600038F8A62005F035F8812005F032F8AF20E1
:1008700005F02FF8142006F018FAAF2005F029F83B
:10088000142006F012FAA62005F023F8AE2005F099
:1008900020F8202005F01DF8002005F01AF8B020FF
:1008A00005F017F8402005F014F8002005F011F8C5
:1008B000102005F00EF84FF48065013D0020ADB228
:1008C00004F0E0FF002DF8D1812005F002F8C820E7
:1008D00004F0FFFFAF2004F0FCFF404B29460C2240
:1008E0003F48A3640FF00DFA03F03EFF06F0D2F884
:1008F0003C4B034463653C4FDFF814A13B68002286
:1009000043F00E033B60394B8AF800201B68B6F8B1
:10091000EE50B3F85A3096F8ED800693059205F044
:1009200041FADFF8F0B08146059A28B3304B142D18
:10093000CBF800302F4BCBF804302F4BCBF80C30DA
:100940002E4B13D004D8052D14D00A2D10D00AE058
:10095000BC2D06D0B5F5807F06D0622D03D10222D2
:1009600002E0012200E003225A7588E00422FBE73E
:100970000522F9E70622F7E7192006F096F917ABEA
:1009800068200F21012205F0F1F89DF85C30D32B8F
:1009900042D11B4B4E2DCBF800301A4BCBF8043014
:1009A000194BCBF80C3009D05D2D184B0AD0362DE1
:1009B00002D083F8589062E0402204E0802384F85B
:1009C00058305CE0C02283F8582058E0AFF3008034
:1009D000399D52A246DF913FC01D0020CE1E00204F
:1009E00068070020404B4C002C020020DC03002054
:1009F00039590008675D000890C1793D1400002056
:100A0000B95A0008975E0008325C8F3D1C07002031
:100A1000F6030020E0030020192006F046F96820C4
:100A200015214A4604F0EEFE002801F0F082B74B93
:100A3000622DCBF80030B64BCBF80430B54BCBF879
:100A40000830B54BCBF80C30B44B0FD004D80A2D7E
:100A500013D0142D0FD00CE0BC2D05D0B5F5807F40
:100A600007D183F816900AE0012200E002229A756D
:100A700005E00322FBE70422F9E70522F7E701235B
:100A80008AF80030A64D00232B70A64CB8F1080F51
:100A900000F2BD80DFE808F00A0A2E7FA5BBBBBBD1
:100AA00005003B6823F002033B60B0E08DF85C304A
:100AB0009A4B4FF000091A689B4B9A4216D053206C
:100AC0004946012217AB05F051F878B19DF85C302A
:100AD000E52B0BD1954B964A83F85990954B1A60AC
:100AE000954A5A600123237004232B70B8F1010F3B
:100AF00000F08D8005F056F900284CD0062117AB88
:100B000068200A4605F032F89DF85F309DF861A034
:100B100003F001035B000AF0010A43EA8A0A9DF828
:100B20005D30DFF8089203F001035AEA030A08D0A7
:100B3000BAF1010F01D1002317E0BAF1020F0BD176
:100B400012E012AB68200C21012205F00FF89DF88D
:100B5000483013F00F0302D1052001F059BA042BDD
:100B600002D189F85AA002E0012389F85A30714B6A
:100B7000724A1A60724A5A6099F85A20002A14BFC1
:100B80006E226F221A7202232370B8F1020F4FF007
:100B900001032B703BD000238DF85C305F4B1A684B
:100BA000614B9A421DD01C200D21012217AB04F08D
:100BB000DDFFB0B19DF85C302A2B01D01A2B10D18B
:100BC0005C4A6049B8F1030F11605F495160574AB0
:100BD00082F85B304FF0030323704FF002032B7059
:100BE00015D0002122AB03F82C1D1820012204F09F
:100BF000BDFF60B19DF85C30FB2B08D14D4B534AD3
:100C00001A60534A5A600423237001232B702378FF
:100C100043B9B8F1000F01D0984633E73B6823F0A1
:100C200002033B603D4B1D683F4B9D4214D0494B36
:100C30004FF400549A6917A942F010029A610223F6
:100C40008DF85F3044481023ADF85C408DF85E307D
:100C500002F00CFA40494C610A2006F026F8772091
:100C6000A021012212AB04F081FFDFF8C080002830
:100C700000F097801E210122772004F0C3FD4FF47D
:100C80002F6006F007F80024A4F160014FF000097E
:100C9000C9B2022217AB77208DF85C908DF85D9079
:100CA00004F064FF9DF85D309DF85C2043EA022269
:100CB0001E4B03F15C0162520234102CE4D1B3F8F4
:100CC0006A404A4604F00F0004F47F44A3F86A40E7
:100CD000012331F802E00232BEF1000F18BF0023F9
:100CE000102AF6D1002B40F09F811A46511012F0C5
:100CF000010F08EB410104D091F85C104B40082132
:100D00002CE0B1F85C1083EA1123F8E7D959000808
:100D1000015E0008CF5D000890C1793D14000020FD
:100D20005E04002097230020001BB7001C07002052
:100D3000155B00084C040020195F0008D12500084D
:100D4000295D0008295A00083F5E0008F15A000892
:100D5000D55E0008001002400010014013F4004F5F
:100D600018BF83F4C05301394FEA4303F6D101326F
:100D7000102ABBD1C3F3033304439842A8F86A4056
:100D800040F05281AA4B42F210721A805A80A94A4E
:100D90005A60A94A9A60A94ADA60A94A1A61A94A1E
:100DA000EBE08246A84B9D4204D13B6823F004034C
:100DB0003B60E3E098F86C30A44C002B40F0DE8000
:100DC00003F1804303F504339A69DFF8B88242F0F7
:100DD00010029A6102234FF400598DF847304046C3
:100DE000102311A94FF480458DF84630ADF844909A
:100DF00002F03CF911A904234046ADF844508DF8A7
:100E0000463002F033F9924BC8F810905A6912A894
:100E100022F470625A615A6942F400725A610823DE
:100E2000129501258DF84D308DF84CA08DF84E505F
:100E300009F054F928238DF8403010A80F238DF8BD
:100E400041308DF842308DF8435005F0F3FB14200B
:100E500005F02BFF2A460DF12F037720D02104F057
:100E600085FE9DF82F300322552B84F88730A4F897
:100E7000902018BFC8F8149097D1D1212A460DF1BF
:100E80002F03772004F072FE9DF82F30772003F0B7
:100E90000F021B0984F8882084F88930162217ABCA
:100EA000AA2104F063FE9DF85C209DF85D3043EAC2
:100EB0000223A4F870309DF85E209DF85F3043EA6D
:100EC0000223A4F872309DF860209DF8613043EA57
:100ED0000223A4F874309DF862209DF8633043EA41
:100EE0000223A4F876309DF864209DF8653043EA2B
:100EF0000223A4F878309DF866209DF8673043EA15
:100F00000223A4F87A309DF868209DF8693043EAFE
:100F10000223A4F87C309DF86A209DF86B3043EAE8
:100F20000223A4F87E309DF86C209DF86D3043EAD2
:100F30000223A4F880309DF86E209DF86F3043EABC
:100F40000223A4F882309DF870209DF8713043EAA6
:100F50000223A4F88430364B41F2707284F86C504E
:100F60001A8046F678125A803A4A5A603A4A9A608B
:100F70003A4ADA603A4A1A613A4A5A6196F8E230D5
:100F80000BB1394A137096F8E3300BB1374A13703E
:100F900096F8E4300BB1364A13703B689A0702D5D5
:100FA000344B1B689847344C0DF1880823689847E8
:100FB000002308F82C3D1E200A210122434604F09C
:100FC000D5FD38B19DF85C30482B03D1284B032266
:100FD0001A7003E03B6823F008033B603B681B4C3E
:100FE00013F0080F1CD0069A4FF0640A0FFA82FB28
:100FF0009BFBFAF528460BF0E1FE81460AFB15B093
:1010000000B20BF0DBFE1D490BF02CFF01464846F9
:101010000BF020FE1A490BF025FFC4F8940033E0D2
:101020000023C4F894302FE04FF0000ABAE600BF66
:1010300090020020FB580008815C0008F35800086B
:10104000915C00089D230008001BB7001C070020CE
:101050000000014025590008F15C00080359000810
:10106000A15C0008F5240008F60300205E040020BF
:101070008F2300204C040020E00300208988883C56
:1010800000002041001001408D4B10225A610822BF
:101090001A614FF00A0A8A4D1920EB680AF1FF3AEB
:1010A00083F01003EB60EB6883F00803EB6005F05E
:1010B000FCFD012001F09EFA192005F0F6FD00204C
:1010C00001F098FA1AF0FF0AE5D108232B611023EA
:1010D0002B617C4B7C4D1B6893F90C000BF0CCFA18
:1010E00073A3D3E900230BF02DFB0BF05DFD0FF094
:1010F00037F8824628880BF061FE51460BF0B2FEAD
:101100000FF064F8714B188028880BF057FE0146E9
:101110006F480BF05BFF6F490BF058FF6E4B186088
:101120006E4BD8680BF0BAFA61A3D3E900230BF039
:1011300009FB61A3D3E900230BF004FB0BF034FDA2
:10114000674B71791860674B674A1970674B02EB00
:10115000C10191F82110C4F89830654B1960B1684D
:101160008B0602D56248012303603B681D0740F1EE
:1011700013815348102343615E4B5F4A1B689342BF
:1011800010D15E4B12A99A6942F008029A614FF49D
:101190008053ADF8483002238DF84B3004238DF88E
:1011A0004A300DE0564A93420CD1544B22A99A6919
:1011B000544842F010029A614FF4804321F8403DB8
:1011C00001F054FF322005F070FD002111221E2095
:1011D00004F018FB012160221E2004F013FB6420A0
:1011E00005F063FD404604F0FDFC00254FF00A0BBE
:1011F000A946AA46022101221E2004F003FB322048
:1012000005F053FD404604F0EDFCBDF95C10BDF95E
:101210005E00BDF960208A448842B8BF014615448B
:101220009142B8BF0A4612F5805F81440ADD244A24
:10123000BBF1010BD16881F01001D160DAD14FF020
:10124000010B01E04FF0000B1E200021122204F0E0
:10125000D9FA4FF00A0C022101221E20CDF810C04D
:1012600004F0D0FA322005F020FD404604F0BAFC2C
:10127000BDF95C10BDF95E00BDF96020C1EB0A0A42
:101280008842B8BF0146AD1A9142B8BF0A4612F56E
:10129000805FC0EB0909DDF810C035DD084ABCF1FC
:1012A000010CD16881F01001D160D4D12EE000BFD3
:1012B000399D52A246DF913F000000A0F7C6B03E24
:1012C000000C01409804002000000020BC04002015
:1012D0000AE81C4100401C46B0030020E003002047
:1012E00094040020880500200C240108D01D002053
:1012F000840500201400002000127A000010024033
:10130000001BB700001001404FF0000B50460BF0DF
:1013100055FD014695480BF059FEDFF86C8220F030
:101320000040C8F8180048460BF048FD01468F48B9
:101330000BF04CFE20F00040C8F81C0028460BF0D3
:101340003DFD01468A480BF041FE20F00040C8F800
:101350002000002170221E2004F054FA01212022D6
:101360001E2004F04FFA1E200221002204F04AFA47
:10137000642005F09AFCBBF1000F07D14FF07E53BB
:10138000C8F81830C8F81C30C8F82030794B102243
:101390001A61794B01221A70784D00214FF4A07226
:1013A00005F19C000EF0ADFC754BDFF8E081DA69C9
:1013B00042F00702DA619A6942F4006242F00C02DC
:1013C0009A61C4F8DC8106F07BFF152205F5F07008
:1013D000FF210EF096FC002384F8E0313B680122E7
:1013E000980784F8F52107D585F8E121032285F8CF
:1013F000F521022285F8E221590708D594F8F52154
:10140000511C84F8F5112244032182F8E01113F0F5
:101410000A0F14D094F8F5310421E21882F8E01193
:101420005A1CD2B22244052182F8E011DA1C0233A0
:10143000DBB284F8F5212344062283F8E021B36867
:101440009A0608D594F8F521511C84F8F511224428
:10145000072182F8E0111F060ED594F8F521092026
:10146000A11881F8E001911C0132D2B284F8F51183
:1014700022440A2182F8E0117279082A01D00E2A4A
:1014800008D194F8F521511C84F8F51122440B2160
:1014900082F8E01194F8F5210C27A518511CC9B267
:1014A00085F8E0715D07354884F8F51106D50232FC
:1014B00080F8F5210144102281F8E02194F8F5210B
:1014C0001227A51885F8E07196F84151511CC9B250
:1014D000002D0CBF002303F00103284884F8F51108
:1014E00033B102320144132380F8F52181F8E03151
:1014F00094F8F53123485A1C84F8F521234414222A
:1015000083F8E021002198220EF0FBFB0025D6F89D
:101510002C214FF0000900270097012039460323B2
:1015200009F082FF804638B9B9F1000F30D14FF48D
:1015300096424FF00109EEE7012DE8D84C2202FB5C
:1015400005F3DFF8409005F1010B09EB0305284690
:10155000394603930EF0D5FB039B5FFA8BFB49F8EA
:101560000380012385F84A305D46D0E700406F468E
:1015700001C05E46000C0140840200201C070020D0
:10158000001002401409002014000020E81E002072
:10159000022005F047FAD4F8DC510146C4F8900265
:1015A00040B9009103230220AA6809F03DFFBC4B1B
:1015B000C3F8900212A8002112220EF0A2FB737948
:1015C0000E2B01D0082B02D101238DF85130B54DDF
:1015D000AE6816F4005616D1B34A0023B05CD75C4F
:1015E000D118874203D01033602BF8D1002103F0CB
:1015F0003CFB83681B78012B03D01036602EEBD1A7
:1016000000238DF84B30A948AB680168C3F3400252
:1016100000318DF84C20C3F3801218BF01218DF8E2
:101620004D20C3F340328DF848208DF84F10C3F39E
:10163000C0329F498DF84A20C3F300428DF84E20F6
:10164000096803F001028DF8492091F82611B5F8D8
:10165000E000C1F380018DF85010B5F8DE10ADF850
:101660005400DF044FF47A70ADF85210ADF8560014
:1016700004D58C4BB3F8DA30ADF85630B1F5FA7FBB
:1016800084BF0023ADF85630B5F818318949ADF85C
:10169000583095F8203184F89432002384F895323C
:1016A0004B709DF85130002B14BF0223002302B170
:1016B000013381494FF0000801EB8303D3F838313F
:1016C000C3460693069A32F808704FF6FF729742A7
:1016D000FBB20CD194F8953284F89732774B93F89B
:1016E0000080B8F1160F40F05181002640E19DF8CE
:1016F0004B201AB19A1E012A40F225819DF84D20F7
:101700001AB11A1F032A40F21E81DFF8D0A19DF8FA
:101710004E204FEA03190AEB09062AB15AF80920AC
:1017200067498A4200F00F819DF84A2012B1012BCF
:1017300000F009813F0A022F05D19DF84820002AB8
:1017400008BF002703E0012F08BF9DF849709DF8EE
:101750004F203AB19DF8512022B9A3F10802012A85
:1017600098BF04279DF8502032B19DF851201AB936
:10177000043B032B40F2CF80012F3BD1484A00238A
:10178000FF2182F89832C2F89C32C2F8A032C2F827
:10179000A432C2F8D83282F8DC1282F8DD1282F864
:1017A000DE32F17B82F8DF3282F8E032C2F8EC629E
:1017B000B2687068ADF85C208DF85E10022217A93F
:1017C0008DF85F20039301F051FC039B5AF8090048
:1017D0001A46317B07F01FF830463A464FF6FF7144
:1017E00008F09AF9039B30461946364A364B08F002
:1017F00033FCA8E0022F38D15FFA8BF3DFF8E0E08A
:1018000018010EEB000100224FF0010C4B708A70A2
:101810008A720EF800C0CE60B16896F80FE070686A
:10182000ADF85C1017A98DF85EE00393CDF810C0F9
:1018300005928DF85F7001F019FC5AF80900317BB0
:10184000059A06F0E8FFDDF810C0304662464FF614
:10185000FF7108F061F9039B304619461B4A1C4B87
:1018600008F0FAFB0BF1010B6DE0032F51D1BDF82D
:1018700052300B4FB3F5FA7F97F8969232D9154A4A
:101880003046B2FBF3F20821BDF8563092B207F0B1
:1018900005F807EB8907C7F860030F4B31E000BF7D
:1018A0001C070020C01D0020E4240108840500203E
:1018B000DC030020B10900200C2401088805002069
:1018C00000040040512200085923000851880008F4
:1018D0002D23000800127A0079230008BC3C01087F
:1018E000FC090020904A3046B2FBF3F20121BDF81A
:1018F000563092B206F0D2FF07EB89078B4BC7F840
:10190000600383608A4B93F89622013283F8962213
:1019100019E0042F17D1BDF85430834A844F92FB4D
:10192000F3F23046BDF85830012192B297F8959203
:1019300006F0B4FF07EB8903C3F8900397F89532DC
:10194000013387F8953208F10208B8F11C0F7FF4D3
:10195000B9AEBFE6774F99E80F00374487E80F002C
:10196000754B10361A78C02E02F101021A7009D098
:10197000D4F898300021985903EB06090BF006FCC7
:101980000028E7D0AB68DE041ED418E06B486A4A32
:1019900000EBC80393F820E0D3F824C082F800E0FD
:1019A000BCF1000FEED000267645EBDA614F330133
:1019B0001F4463440FCB013687E80F00F4E7B8F10A
:1019C000080F5F4F26D128E05B4B93F80090B9F1E8
:1019D000010FF4D95B4E00274F4506F11006EEDAF1
:1019E00056F8100C4FF07C510BF03CFA4FF07C5144
:1019F00046F8100C56F8140C0BF034FA4FF07C51EA
:101A000046F8140C56F80C0C0BF02CFA013746F87B
:101A10000C0CE1E7B8F10E0F03D13B7843F0100353
:101A200002E03B7823F010033B7007F0C9FF464902
:101A3000464B4748474AC4F8743401600023B5F860
:101A40001801C4F87014A4F87A3484F87C34C4F80B
:101A50008024C4F88424404958520233242BFAD1FC
:101A60003E4B334C1A60AB6813F0080F00F0A480B3
:101A70003B4B002293F81631042B00F29780DFE8ED
:101A800003F003032A448100012B4FF0030208D125
:101A900084F88824072284F88A3484F889240C2363
:101AA00008E0022384F88834002384F88A3484F818
:101AB0008924072384F88B34002300930820012312
:101AC00028494FF4E13209F0AFFC274BC4F89004E9
:101AD000C4F8943466E001230093244905230820C8
:101AE000234A09F0A1FCB5F81811C4F89804A1F52F
:101AF0007771490000231F4A99500433302BFAD1E3
:101B00001D4BC4F894340C234AE0009201230820B2
:101B10001A494FF4E13209F087FC194BC4F89C04D0
:101B2000C4F8943410233BE040420F0069230008BE
:101B30001C070020CC0A0020642300200C2401088C
:101B400072020020D40A0020CE1E00205425010875
:101B50002C010020900B0020DE0600202002002037
:101B6000C01D0020296B000899600008356C000832
:101B7000A08601004C0100204D610008C16B0008E7
:101B80003D6100080092012308203B494FF4E132F7
:101B900009F04AFC394BC4F8A004C4F89434082373
:101BA00084F88B34003018BF012028B9082001F0D8
:101BB00089F80023C4F89434AB68580405D508228A
:101BC00084F88B242E4AC4F8942442F201021A406D
:101BD00003F0010103F400505AB12A4AC4F89424D6
:101BE00018B1294A082082F88B0411B10C2284F81C
:101BF0008B2494F88B241906A2F1040284F88C2417
:101C000058D5214B214AD5F83411C3F8A424002318
:101C10001F4A02EB0310D0F874011646884204D024
:101C20000133DBB2042BF3D9002384F8A934194B18
:101C30000020C4F8C43406F0DDFF174B94F8A92443
:101C40001B680021C4F8B03495F8263106EB021267
:101C50008B42C4F8AC144FF010000091D2F87421FC
:101C60000CBF0123032309F0DFFBC4F8C804A8B9A3
:101C7000802001F027F814E0756B00082961000846
:101C8000616100086D6100081C070020E81E00204B
:101C90000C240108E61E0020BC1D0020012006F0D7
:101CA000A9FF884B1868884B00F5947204301A60BD
:101CB00001F022F9AB689A050DD59E044CBF83480C
:101CC000834806F031FF834B1A6842F010021A6015
:101CD000814B00221A60AB68D80340F1C680DFF860
:101CE00030B2DFF8309240F22A3A5246584600218C
:101CF0000EF007F8D9F81830784843F00403C9F813
:101D000018304023ADF8403018238DF8433010A927
:101D100003238DF8423004F099FBD9F81C30704E43
:101D200043F00203C9F81C306E4B4FF000081A68EC
:101D30006D4BA9F69479B2FBF3F23388013A23F4A0
:101D40005C731B041B0C338092B21D23B385328558
:101D50000122B282338C23F001031B041B0C338459
:101D6000338CB088318B23F0020321F07301090416
:101D70001B04090C1B0C134341F0600180B2B080BE
:101D80003183A6F834803384338B23F008031B049B
:101D90001B0C43F008033383B6F844306FEA434327
:101DA0006FEA53439BB2A6F84430D9F8A83F1343D7
:101DB000C9F8A83F4846059204F0C5FB4B4BCDF847
:101DC00060B0179380231C934FF480734FF0100B77
:101DD0001D9348464FF4005317A92093CDF864B0E3
:101DE000CDF868A0CDF86C80CDF87880CDF87C80F7
:101DF000CDF8848004F089FBB389059A9BB243F443
:101E00000073B381D9F8003011A843F00203C9F878
:101E1000003002238DF844B08DF845208DF846300F
:101E20008DF8472004F006FC314B1A68314B48F816
:101E3000032008F10408B8F1800FF5D107F09AFFEC
:101E400007F098FF2C492D4BD4F880240B60803389
:101E5000C4F8F8372A4B1A6000F08AFF00F0C4FF7C
:101E600000F09EFF274B01221A70AB68590540F124
:101E70008780042007F0BCF90146042002F0F5FE3B
:101E800018B14368187A00F00100AB6884F8FC07C9
:101E900013F480690BD0042007F0AAF9014604204E
:101EA00002F0E3FE10F1000918BF4FF00109164BD4
:101EB00083F80090154B1E6833786BBBC4F800683C
:101EC00054E000BFDC03002078050020CC25010889
:101ED000D82501082C0200209800002000080140AD
:101EE000000400409C00002000366E0134040040D5
:101EF000D02301085C06002058060020041F0020A3
:101F000004070020480600209005002094050020CA
:101F1000E80B002000100240012B27D1DFF81C81C4
:101F2000002140462C22C4F804680DF0EAFE8E23FE
:101F300088F801304FF07C0BE0234FF07D0A88F8E1
:101F4000033088F800B088F82BA0DFF8F480002177
:101F500040462C220DF0D5FE8A2388F80130A023BC
:101F600088F800B088F8033088F82BA03378022B6B
:101F700008BFC4F80868B9F1000F01D009F0C0FA31
:101F800004F088FD254B18606B79052B03D1244B99
:101F90004FF4C8721A80234B4FF47A721A80224B86
:101FA000C8221A803B7843F008033B701F4B1A7815
:101FB00022F002021A70AB689A071ED51C4BC4F8B7
:101FC0000C3804F02BFC282004F06FFE079B013B2B
:101FD0000793F6D1174B95F8051118780A46012397
:101FE000904203D30133082B0A44F9D1124A1370EB
:101FF00095F806215343A4F81038AB689B0309D524
:1020000094F84F3043F0010384F84F3002E003208E
:1020100004F09AFE23B0BDE8F08F00BFF404002066
:10202000600400208C2300208423002096230020BD
:10203000C41E0020A405002092000020BC05002042
:10204000E9050020AFF30080034B4FF4805208B144
:102050001A6170475A61704700080140034B4FF402
:10206000805208B15A6170471A61704700080140F8
:10207000032810B50F4B0DD80F4A126894888C4274
:1020800008D2D2888A4205D9012202FA00F01A78D1
:10209000104318701B780F2B0BD1064B00221A70BF
:1020A000064B998808B2142802DD1439998010BDB6
:1020B0009A8010BD300F002070160020900B002079
:1020C000024B9A8801329A80704700BF900B002023
:1020D000074B1A68074B1178B3F9040053780B4487
:1020E00003EB83039842D4BF00200120704700BF58
:1020F00070160020900B0020064BB3F90400064B2D
:102100001B681B7803EB83039842D4BF0020012097
:10211000704700BF900B00207016002010B50446D9
:10212000FFF7EAFF002814BF2046002000F001005E
:1021300010BD024B01221A72704700BF900B0020A5
:10214000014B187A704700BF900B0020034BB3F986
:102150000400D0F1010038BF00207047900B002030
:10216000014B00229A807047900B002003685A1C94
:10217000026019707047016B0346C26810B5406970
:1021800041B1196C541A005D013918BF0A46C0B23A
:102190001A6410BD196A405C0131B1FBF2F402FB14
:1021A0001412C0B21A6210BD026B03691AB15168F1
:1021B000013B026C02E0C169026A013B881A1840C7
:1021C000C0B27047436B13B190F844007047826A05
:1021D000436AD31A58425841704743799B070AD53E
:1021E000436A8269D154426A03690132B2FBF3F156
:1021F00003FB112343627047437913F0010307D0B7
:102200000369C169026A013B881A1840C0B270476D
:1022100018467047437910B513F0010304460DD0FA
:10222000FFF7EAFF58B1226A6369985CE3680132FC
:10223000B2FBF3F103FB1123236210BD184610BD5E
:10224000426A806A131A5842584170474171704778
:10225000334A10B5136C90681944081A40F68C2361
:1022600098429160D060516013463CD9127893F93E
:1022700045108A420BD1111F082908D893F846103F
:10228000182901D8013103E083F8442002E000213D
:1022900083F8461093F944108A421CD1204991F8E2
:1022A0004710C1B1002191421E4806DA03EB8104B8
:1022B000246920F811400131F5E7511E00EB41017E
:1022C0001630814203D0002421F8024FF9E7164965
:1022D00008780130087083F84520002201211A7027
:1022E00083F8471010BD92F84710B9B1A0F2EF245F
:1022F00040F2DA518C4208D811780B2905D80B1D11
:102300000131117042F8230010BD002283F84720EC
:10231000991804320020302A0861F9D110BD00BF9D
:10232000B4090020FC170020C6180020084B03EB5E
:102330000010837A0133DBB20A2B837207D98378CA
:102340001BB94178034A22F8113000238372704789
:10235000FC090020FC170020024B1A6C1144196480
:10236000704700BFB4090020024B53F820301B68AF
:10237000198070477C0A0020074BA1F57A7153F849
:1023800020304FF47A701A689B884B4393FBF0F32C
:102390009BB21380704700BF7C0A00202DE9F04FEC
:1023A000504A514E1768738984463089A7EB03273A
:1023B00085B0039187FB0001B288CB111404C209D8
:1023C000F08842EA416287FB000114EB0208728840
:1023D0004FF000054FEAC2344FEA1022B08945EBB6
:1023E000030942EA01620B1287FB000114EB020AA7
:1023F0004FEAD05242EA41224FF0000545EB030B71
:1024000012F5FA604FEAE15343F10001CDE9000112
:10241000B0F5FA6F71F1000147DAA2FB024502FB49
:1024200003F1052605EB4105A4FB060106FB05119A
:102430004D104FEA3004B8EB040869EB0509840835
:102440002A4844EA81748D104FF0FF31BAEB040A38
:102450006BEB050BDDE9004584428D4125DA40F642
:10246000AC5012184FF0000143EB010302FB03F1E3
:10247000A2FB02236FF0060003EB4103544200FB72
:102480000344A2FB000118EB000821444FF00B04A9
:1024900049EB0109A2FB040104FB031149104FEAB7
:1024A0003000BAEB000A6BEB010B114B1A68A2FB70
:1024B0000A0102FB0B11420D42EAC1224B15B2EB9D
:1024C000080263EB0903D00B40EA4340BCF1000F64
:1024D00001D0CCF80000039808B10099016005B064
:1024E000BDE8F08FB41600207807002024FAFFFF23
:1024F000B8160020324B2DE9F0411C88314B0A26DA
:102500005A89B3F91250A41A1A89ED025443B3F947
:102510001420E413224495FBF2F22244DA6156437C
:10252000A2F57A6202FB02F4B3F90480B3F902C0A7
:10253000B3F90E7002FB0CFC02FB08F2B3F90C803D
:102540002413674304FB08F4241404EB62320232C0
:10255000DC88921002F50042B3F920506243B3F9CF
:1025600000304FEAEC2404EBE72404EB8304AC4096
:10257000154B02341B68D20BA3EBA4044CF250336E
:102580002B41634355BF5B00B3FBF2F3B3FBF2F3A4
:102590005B001A12524340F6DE3462430B4C08369D
:1025A0005C43241404EB224202F6CF62361103EBA3
:1025B000221300B1036001B10E60BDE8F08100BFDD
:1025C000C41600208C070020C016002043E3FFFF44
:1025D000064B1B7813B1012B03D070474FF40062F8
:1025E00001E04FF48052024B1A80704776070020BA
:1025F0000000002008B5024B1B68984708BD00BFCB
:102600009823002008B503685B69984708BD08B5A2
:1026100003681B69984708BD08B50368DB689847DD
:1026200008BD08B503689B68984708BD08B50368EE
:102630005B68984708BD10B5044C2068FFF7F6FFAB
:1026400018B12068FFF7EDFFF6E710BD2406002063
:1026500008B503681B68984708BD014B1868F7E781
:10266000F817002038B5054C05465E212068FFF7B5
:10267000EFFF20682946BDE83840E9E798050020CB
:10268000014B5E211868E3E79805002010B50A4C5D
:102690005E280146206805D15D21FFF7D9FF20683B
:1026A0003E2105E05D2903D1FFF7D2FF20683D21DF
:1026B000BDE81040CCE700BF9805002010B50446E7
:1026C000C0B2FFF7E3FFC4F30720BDE81040FFF7F7
:1026D000DDBF10B50024094BE0B21B7883420CD952
:1026E000074B33F81010074B53F820301BB10B2861
:1026F00001D89B6898470134EDE710BD64230020A2
:10270000662300207C0A0020054B1B6803EBC000F9
:1027100090F9063019420CBF01204FF0FF3070478E
:10272000741600200A4B1A6802EBC002D379FF2B03
:1027300007D008490978994203D9074A32F81300AB
:1027400004E00728D4BF908840F2DC5000B2704704
:1027500074160020A70B0020DE0600202DE9F04FA4
:102760000C68836889B0D0F800A0D0F804800646D1
:10277000204603938B460DF0F3FC074620460DF0F0
:1027800063FDDBF80440814620460DF0E9FC054678
:1027900020460DF059FDDBF8082004461046019252
:1027A0000DF0DEFC019A834610460DF04DFD3946D2
:1027B000029058460AF056FB3946049002980AF0F7
:1027C00051FB5946059048460AF04CFB0299069089
:1027D00048460AF047FB2946079058460AF042FB54
:1027E000014650460AF03EFB2146834606980AF011
:1027F00039FB014605980AF02DFA014640460AF0D9
:1028000031FB014658460AF025FA214683460498D2
:102810000AF028FB014607980AF01AFA01460398C5
:102820000AF020FB014658460AF014FA306002997B
:1028300005F100400AF016FB014650460AF012FB73
:102840002146834607980AF00DFB014604980AF0DA
:10285000FFF9014640460AF005FB014658460AF0DA
:10286000F9F92146834605980AF0FCFA01460698D4
:102870000AF0F0F9014603980AF0F4FA01465846C6
:102880000AF0E8F92146706050460AF0EBFA294652
:10289000044609F100400AF0E5FA014640460AF014
:1028A000E1FA014620460AF0D5F9394604462846A1
:1028B0000AF0D8FA014603980AF0D4FA01462046F5
:1028C0000AF0C8F9B06009B0BDE8F08F2DE9F84F03
:1028D000374E0446376838460DF042FC0546384608
:1028E0000DF0B2FC7668804630460DF039FC834628
:1028F00030460DF0A9FCD4F8049006462946484617
:102900000AF0B0FAA7688246414638460AF0AAFAA9
:10291000014650460AF09CF92168824658460AF062
:10292000A1FA4146044648460AF09CFA31460AF0AC
:1029300099FA014620460AF08DF931460446384698
:102940000AF090FA29460AF08DFA014620460AF06C
:1029500081F9014650460DF005FD16490AF082FA4C
:1029600009F09CFE10A3D3E900230AF015F8124BDE
:10297000044618680D4609F091FE02460B462046B3
:10298000294609F02DFD00220C4B0AF005F80AF04B
:102990000BF90DF01BFC83B21A0444BF00F5B473AD
:1029A0009BB218B2BDE8F88F182D4454FB210940A2
:1029B000C00400200000E144B007002000002440D3
:1029C00080EAE073A3EBE0738B4206DB002801DDB5
:1029D000401A704702D00844704700207047074BE8
:1029E0001B7803F0040303F0FF001BB1044B1888AD
:1029F000C0F3C01000F00100704700BF9623002014
:102A000046020020034B1A78510744BF22F004020B
:102A10001A7070479623002070B5FFF76DFB38B32E
:102A2000144C237A0BB9A38070BD134D2E78C6F3D6
:102A30008000FFF773FB90B1104B46F002061A6856
:102A40000F4B51892E7019805189598052899A8073
:102A50000C4A12685288DA80E3880133E380FFF77A
:102A600037FB10B92B785B0702D4BDE87040C9E78B
:102A700070BD00BF900B0020962300208C0B00201F
:102A8000DE060020701600202DE9F0410278034692
:102A9000202A00F10100F9D0092AF7D02D2A02D10D
:102AA0000346414D04E02B2A08BF03464FF07E55F4
:102AB0001E460024334616F8012BA2F13007F9B266
:102AC00009290DD8394920460AF0CCF90446384680
:102AD0000AF074F9014620460AF0BCF80446E9E71A
:102AE0002E2A17D1314F334616F8010B3038C2B2B7
:102AF000092A0FD80AF062F939460AF067FA014646
:102B000020460AF0A7F82949044638460AF0AAF9EF
:102B10000746E8E71A7802F0DF02452A38D15A78EA
:102B20002D2A02D10233012604E02B2A14BF0133DF
:102B300002330026013B002713F8012F303AD1B2AF
:102B4000092903D80A2101FB0727F5E7B7F59A7F82
:102B500028BF4FF49A77B8464FF07E51B8F1070F6F
:102B600007D9084612490AF07DF9A8F1080801467C
:102B7000F4E707F0070737B108460C490AF072F985
:102B8000013F0146F7E72EB120460AF01FFA04E0A4
:102B90004FF07E5120460AF065F9014628460AF0BA
:102BA00061F9BDE8F08100BF000080BF0000204156
:102BB00020BCBE4CF0B50124B0FBF4F58D4201D32E
:102BC0004C43F9E70026DCB1B0FBF4F504FB15003B
:102BD000B4FBF1F41EB9002D01DC002CF3D1092D5A
:102BE00003F101075FFA85FC04DD002A0CBF5725BD
:102BF000372500E0302565441D7001363B46E2E78D
:102C00001C70F0BDF0B50124B0FBF4F58D4201D38A
:102C10004C43F9E70026DCB1B0FBF4F504FB1500EA
:102C2000B4FBF1F41EB9002D01DC002CF3D1092D09
:102C300003F101075FFA85FC04DD002A0CBF57256C
:102C4000372500E0302565441D7001363B46E2E73C
:102C50001C70F0BD70B50646B6FBF2F4084615468A
:102C600014B12046FFF7F6FF05FB1464024B1B5D11
:102C700000F8013B70BD00BF763E01082DE9F04130
:102C8000069C002B06460F460CBF4FF020084FF065
:102C90003008234613F8011B09B9154603E0002A42
:102CA000FBDD013AF6E7002D04DD30464146B8472A
:102CB000013DF8E714F8011B11B13046B847F9E7B8
:102CC000BDE8F081024B9A6822EA000098607047E4
:102CD000C01D002030B50E4D0028B8BF40420D4C3D
:102CE00090FBF5F304FB03003C22424392FBF5F01A
:102CF00003EB830304FB002203EB830300EB83035A
:102D00000B804FF47A7392FBF3F24A8030BD00BF20
:102D100080969800806967FF094B1B7873B1094B57
:102D20001B685B782BB1084BD87C003018BF0120A2
:102D30007047064B1878C0F3800070470120704739
:102D4000180F002094050020300200209623002058
:102D500008B506480DF016F8C0B2132805D8034A86
:102D6000431C20211154D8B2F7E708BDB51100204B
:102D7000094A0A48002310B5116803701A46CC1896
:102D800064880CB9CC5C24B104330132802BD2B2FC
:102D9000F5D1027010BD00BF58060020DC060020EF
:102DA00010B50B4B0B4819780B4B5A784B085C1E2F
:102DB000047001F0010109480B44037008495308ED
:102DC000581E087002F00102064913440B7010BD32
:102DD0001507002010070020300F002012070020E8
:102DE0001307002011070020F0B50F4A0F4816788E
:102DF0000F4A0023176843701A4619460546D0B299
:102E0000B0420CD217F82200013204099C4200F0B3
:102E10000F00A8BF631C8842A8BF411CEFE76B707E
:102E2000044B1970F0BD00BFDC060020300F0020FD
:102E30005806002015070020F8B5101A0C461F464A
:102E400009F0BCFF0546381B09F0B8FF174B079E79
:102E500019680AF007F82946044628460AF002F8DD
:102E600021460746204609F0FDFF0146384609F095
:102E7000F1FE0DF001FC0E4909F0F4FF0AF0DEF955
:102E8000069B2146186005F100400DF06BFA0949D8
:102E900009F0E8FF084909F0DDFE0AF0A9F9002869
:102EA000BCBF00F50C40A0303060F8BD68000020C9
:102EB0002C7D8E3FA00CB34500A00C4610B509F048
:102EC0007DFF002104460AF089F908B1204601E09F
:102ED00004F1004005490AF079F8054909F0C2FFFC
:102EE0000DF03EF9034B186010BD00BF8096184BE3
:102EF00035FA8E3C6800002070B50446007909F070
:102F000059FF1E490AF062F81D4D1E4E2860A07B35
:102F100009F050FF19490AF059F8EE6068606079CD
:102F200009F048FF18490AF051F8184D2860E07B75
:102F300009F040FF11490AF049F86860607E09F025
:102F400039FF13490AF042F8EE60A860A07909F051
:102F500031FF0D490AF03AF80E4D2860207C09F047
:102F600029FF06490AF032F86860A07E09F022FFC6
:102F700007490AF02BF8EE60A86070BD0000C84257
:102F8000B81000200000FA4400002041C8100020C2
:102F900000007A44EC10002044F25063984203DDB4
:102FA000A0F50C40A0387047034B9842BCBF00F519
:102FB0000C40A030704700BFB0B9FFFF10B5002330
:102FC000094CDAB254F8224001338442F8D100238C
:102FD000064CD8B234F8104001338C42F8D102EBE1
:102FE0008000C0B210BD00BFC02A0108AC2F01088C
:102FF00090F83B3210B57BB990F83A3290F839220C
:10300000934209D201219940B0F840420133214353
:10301000A0F84012DBB2F3E710BD8379012B03D196
:10302000D1F1010138BF0021D0F834315A689B68D2
:1030300009B11361704753617047044B53F8203056
:103040001BB107289CBF1B6819807047AC0A002081
:1030500010B5054C00202188FFF7EFFF61880120A3
:10306000BDE81040E9E700BF820000202DE9F041F3
:103070000F88002347FA03F2D2072BD58A7803F092
:10308000070512F0100F18BF91F803C002F00F06E9
:1030900018BF46EA0C06AD004FF00F0C0CFA05FC09
:1030A00006FA05F5DC0850F82480282A28EA0C0CDA
:1030B00045EA0C0540F8245005D101229A40C46825
:1030C00024EA020205E0482A04D101229A40C46899
:1030D0002243C2600133102BCCD1BDE8F08100BF88
:1030E0002DE9F04F974B91B01B68BBB9964C2378F4
:1030F000013B042B00F2F886DFE813F015061506F5
:103100001506E606CC062068FFF78BFA8F4B0446BF
:103110001B681B784BB1012B00F0ED80894C2068B7
:10312000FFF784FA0028EED1E0E72428884D0CD080
:1031300006D80A2800F08E800D2800F08B80C6E0AB
:103140002A2806D02C2804D0C1E02B706B70AB70FD
:10315000CEE06A782E782A4400217D4BD170EEB9FA
:10316000DA789E74472A19D11A79502A16D15A79D9
:10317000472A07D19A79472A04D1DA79412A01D11D
:1031800001229A746A79724B522A07D19A794D2A90
:1031900004D1DA79432A04BF02229A74AB7C6C4FC3
:1031A000012B02D0022B36D049E0B31E072B46D8A4
:1031B000DFE803F0040810141C27452C07F00CF876
:1031C00068613CE0EA78624B532A38D15A6952422E
:1031D0005A6134E007F000F8A86130E0EA785C4B0F
:1031E000572A2CD19A6952429A6128E0EB78302B09
:1031F000584B1A788CBF42F0020222F002021A7079
:103200001DE0002007F042F8287718E0002007F0C2
:103210003DF8E88313E0072E06D0082E0FD10120D9
:1032200007F034F878840AE0012007F02FF841F223
:10323000184358434FF47A72B0FBF2F33B840136E3
:1032400000232A2C424A2E706B704CD1012182F847
:1032500024104DE095F82430002B34D03C4BDB7823
:10326000402B04D9A3F137021201D2B202E01B01B4
:1032700003F0F0022B79A978402B8CBF373B303B11
:10328000DBB21344DBB29942314A1BD1937C012B50
:1032900008D0022B16D1118C2F4B528C19802F4B3A
:1032A0001A800FE02B4909788E070CD52C495069FC
:1032B000086090694860107F2A490870D18B2A4ABB
:1032C000118000E00023002285F8242010E06B78B4
:1032D0001F4A0E2B03D8591C13445170DC7095F80B
:1032E00024301B4A1BB991784C40947000E00023B5
:1032F00003F001035BE1164B002193F82520082A17
:1033000000F25481DFE802F00B0514324353718D53
:103310009A00622801D1022207E083F82510B52C1B
:1033200040F0448193F82520013283F825203DE1C7
:10333000032283F8252083F8260083F8270083F8EA
:10334000280033E1E40B0020C40B0020E00B002038
:10335000380F00207202002016060020C41C002036
:10336000B0050020E80500201A060020042283F89A
:10337000252093F8272093F828100244D2B283F82E
:1033800027200A4483F8282083F829000EE105222B
:1033900083F8252093F8272093F828100244D2B20E
:1033A00083F827200A4483F828205885FEE0062168
:1033B00083F8251093F8271093F828002144C9B208
:1033C00083F82710014483F82810598D6A4A01EBCD
:1033D0000424A4B2B4F5007F89BF0021548551852F
:1033E00082F8251000229A85E0E093F8272093F8D0
:1033F00028100244D2B283F827200A4483F82820F8
:103400009A8DC72A03D85C49114481F830000132F3
:1034100092B29A855B8D934240F0C8800722564B4A
:1034200083E7082283F8252093F82730834200F0B1
:10343000BD80514A002382F82530B8E083F825107A
:1034400093F828104C4A814240F0B08092F829103D
:10345000062946D004D8022912D003292CD0A5E091
:10346000122957D0302940F0A18092F83410434AF5
:10347000102988BF1021117010784149002257E0AF
:103480004049506B4860906B0860116C4FF47A7043
:1034900091FBF0F13C48018092F8F8103B4A19B1D9
:1034A000117841F0020102E0117821F0020111705F
:1034B000012283F8F92050E092F8351011F0010153
:1034C00005D092F83420D41E6242624100E00A46E0
:1034D00083F8F820002A40D12C4A117821F002010B
:1034E00016E092F83B1011F0010105D092F83A2055
:1034F000D01E4242424100E00A4683F8F82022B939
:10350000224A117821F00201117093F85F10204ACD
:10351000117022E0516C1F480180916C42F21070D2
:1035200091FBF0F11C480180012182F8FA1014E0AF
:10353000824201F10C0110DA11F8045C174C1555A8
:1035400011F8035C164C155511F8015C154C155516
:103550000D78154C15550132EAE793F8F930064A13
:1035600023B392F8FA300BB3002382F8F93082F8D3
:10357000FA3001231BE000BF380F0020C61C0020DA
:10358000680F0020B00500201A06002072020020FB
:10359000E805002016060020C41C0020C71C0020DF
:1035A000D71C0020E71C0020F71C00200023002B64
:1035B0003FF4B4ADA54BA64E9A68DA6032689A60C3
:1035C000A44B1A6842F020021A60A34B1A78012A11
:1035D0000CBF002201221A70A04B1A7891077FF5C8
:1035E0009DAD9F49097804297FF698AD9D490978DA
:1035F00001F0040101F0FF0011B922F001021A707C
:103600001B78964F13F0010F974C984D11D180B154
:103610009B070ED5964B28686A6818605A60FFF7BA
:103620004DFC944B1B88A4F8FC303B7843F001031D
:103630003B7094F8FE304FF00509013393FBF9F924
:1036400009EB8909C9EB03098B4B8C481B7884F87B
:10365000FE900593831D03EB890907900023DFF893
:103660000CE2874A53F80E00864F985090FBF7FC07
:1036700002F1080743F807C0834F03EB0E0107FB75
:103680000C0742F2107097FBF0F00691079980B298
:1036900021F8020F02F1100A03EB830B049007914B
:1036A00053F80A0059F80B1049F80B70C1EB0008E9
:1036B00008EB0700734F4FF0050843F80A0090FB32
:1036C000F8F007FB0C00059918320129985077464D
:1036D00008D1DDF810E0AEF10202B2F5797F9CBFAF
:1036E000069908600433082BB9D1DFF87C81306873
:1036F000D8F84C31C01A09F05DFB644909F066FC4A
:1037000033684FF07E51C8F84C31814609F048FDCE
:1037100010B94FF07E5000E048460CAAC4F85001A2
:10372000534B00920DAA019297E803000CCBFFF7D0
:1037300083FB0C9B56496422B3FBF2F30D980B807C
:10374000544B90FBF2F21A80444A474E127812F022
:10375000010208BF1A8098F8543108BF0A80002B74
:103760003AD0D6F850114FF07E5009F02FFCD6F821
:10377000583181462868C01A09F020FB494609F0F3
:1037800071FB09F035FDD6F85C211FFA80FA6868F4
:103790000FFA8AFA801A09F011FB3F4B196809F0F9
:1037A00061FB494609F05EFB09F022FDB6F9623182
:1037B00000B2C218B6F960310221534492FBF1F213
:1037C00093FBF1F392B29BB2A6F86621A6F864319E
:1037D000A6F86221A6F86031012388F854312F4BF6
:1037E00079681B88386803F030031F4D1F4EC8F8F6
:1037F0005C11C8F85801002B3FF490AC05F5B87384
:10380000009305F5BA730193D5F86821D5F86C31AA
:10381000FFF712FB7368D5F86C01C01A09F0CEFAF5
:103820001D4B196809F01EFB09F0E2FCD5F8683160
:103830003268C5F87C019B1AC5F878310E4B1B78AD
:10384000012B2DD0022B00F0F98067E4C40B00207F
:10385000BC1D00202C0200209D23002072020020AD
:10386000E805002096230020380F0020B005002036
:10387000C0190020D4040020D019002036100020E8
:103880006410002080969800806967FF00007A44E9
:10389000180600201C0600206800002046020020B8
:1038A000D5F88071D5F89C410497D5F8907104F152
:1038B00000400597D5F89471D5F85061079709F045
:1038C00097FC8046204609F093FC8F4BD5F8985121
:1038D0001B688E4C0695089009930025DFF84CA2D2
:1038E0005AF81570AAF11403384635F8039009F018
:1038F00065FA049909F0B6FA09F07AFCC9EB000000
:1039000080B20AF1280A25F80A000FFA80FA504618
:1039100009F054FA059909F0A5FA09F069FC1FFAB3
:1039200080FB0AEB070009F049FA079909F09AFAB7
:10393000314609F097FA216809F08CF909F058FC32
:10394000404505DBDDF820E07045A8BF704600E08B
:10395000404609F033FA206009F04AFC58441FFA47
:1039600080FB606809F13109381A09F027FA3146FD
:1039700009F02CFB0999206184468878D4F808A0C6
:10398000CDF80CC009F016FA08F088FE5CA3D3E964
:10399000002308F0D7FE02460B4600205C4908F0E1
:1039A000FBFF09F001F9314609F054F901463046B0
:1039B00009F00CFBDDF80CC003465146604603934A
:1039C00009F046F9039B0146184609F04BFA0146F7
:1039D000504609F03FF91FFA89F9B9F1620F014623
:1039E00020616760A0600ED9069809F03BFA09F0E3
:1039F000FFFB484BB0F5FA6FA8BF4FF4FA6098424E
:103A0000B8BF184600E00020834440F6B8330FFAF0
:103A10008BFB9B45A8BF9B463F4B0A229B45B8BFEB
:103A20009B466A433D4B54F8141B25F803B03C4BAE
:103A30000235042DD1503FF471AB4FE7324BD5F82E
:103A400070B11F68B5F8A461B7F808904FEA5B033E
:103A5000994528BF994633B2994502DC1FFA89F986
:103A60000BE03049D5F8500109F0FCF909F0C0FB32
:103A700030441FFA80F9A5F8A491D8F87451D8F809
:103A8000A861AE1B3046FFF787FA0028D8BF404236
:103A900041F293139842CCBF00200120002847D068
:103AA000304609F08BF9204909F0DCF90CF0CCFB29
:103AB0000646584609F07EF90146304609F0D2F92B
:103AC00009F096FB80B240F6B83203B29342A8BF29
:103AD0001346114AA8F8AC019342ACBFEB18AB18DF
:103AE00048F6A042934203DDA3F50C43A03B04E05B
:103AF000002BBCBF03F50C43A033C8F8B03119E06C
:103B0000182D4454FB21194078050020481100204D
:103B10000000F03F30F8FFFF48F4FFFF8005002071
:103B2000701100200000C842D3023739B0100020C5
:103B3000C8F8B051D4F8B021C2F50C502830049226
:103B400009F03CF9AE4909F08DF905460CF008FB87
:103B50000F9028460CF078FBD4F8C051D4F8B4315B
:103B6000D4F8B8E10E9005F100400793CDF828E0B5
:103B700009F03EFB0590284609F03AFBD4F8508145
:103B8000D4F8BC410B9009949E4C0025484609F09E
:103B900015F90EAB53F8151009F064F9DFF8A0A27F
:103BA00006463AF9050009F009F90146304609F0E0
:103BB0004FF809F01DFB944B06B2B6F57A7FA8BF0B
:103BC0004FF47A769E42B8BF1E46B0B20AF13C0A64
:103BD00025F80A0000B209F0F1F80799824609F0C9
:103BE00041F909F005FB80B208900A99504609F0A6
:103BF00039F9414609F036F9216809F02BF809F046
:103C0000F7FA0599884204DB0B9A9042A8BF104648
:103C100000E0059809F0D2F882462060606814340C
:103C2000301A09F0CBF8414609F0D0F954F80C3CB1
:103C300044F8040C8446B8780693CDF80CC009F01B
:103C4000B9F808F02BFD6CA3D3E9002308F07AFD46
:103C500002460B4600206D4908F09EFE08F0A4FFC6
:103C6000414608F0F7FF0146404609F0AFF9DDF89C
:103C70000CC0034606996046039308F0E9FF039BD6
:103C80000146184609F0EEF80146069808F0E2FFF2
:103C900044F8106C014644F8040C44F80C0C0998E4
:103CA00009F0E0F809F0A4FA089E0644504609F02D
:103CB0009FFA304440F6B83300B29842A8BF184685
:103CC000534B0A229842B8BF18466A43514BE852F8
:103CD000514B0235042D42F803A07FF457AF3B79D6
:103CE0002BB1049864224D4B90FBF2F21A803B8872
:103CF0004B4C9B450ED9D4F8A831D4F87401C01AA6
:103D0000FFF74AF942F210730028B8BF40429842C8
:103D10007FF704AA434B01221A70B4F8FC203F4BF2
:103D20001A80FFF7FBB9404A116890460F7817B127
:103D3000012F0DD0ABE0012B00F2A98062783B4B44
:103D400003EB02133A4A59681068FEF765FC9BE0E2
:103D5000374E3068FEF75BFCB146002800F09780D4
:103D60002378344D022B29D0032B31D0012B40F086
:103D70008E80314B1F686B69FB1A632B40F2878082
:103D80002B69042B18D8DFF8A480306808EB0313E4
:103D90005968FEF741FC6B78366808EB03139D68A1
:103DA00015F8011B19B13046FEF752FCF8E72369FC
:103DB0006761013323616AE0022066E06A781B4B89
:103DC000306803EB02135968FEF726FC03205CE021
:103DD0002B7E03B92F76237E164D012B36D12B690E
:103DE0007B2B2FD8154AD9F80000D15CFEF730FCA8
:103DF0002B6901332B6129E0182D4454FB21194014
:103E0000D30237397011002018FCFFFF0000F03F8B
:103E100048F4FFFF80050020481100206E050020B7
:103E2000380F0020D0190020E00B00207C2501086D
:103E3000E40B0020C40B0020BC1D0020D02A010888
:103E40009C10002000232B6102232B76237E284D1B
:103E5000022B16D12B690F2B11D8D8F80020254939
:103E60005278D9F8000002EB02120A44134493F886
:103E70007D10FEF7EDFB2B6901332B6101E003237D
:103E80002B76237E022B02D9042004F0B3FE0023FC
:103E9000636029E063680522013363606378012071
:103EA0000133DBB2B3FBF2F202EB82029B1A6370C6
:103EB000114B00221B68A360104B1A70104B1A782C
:103EC00022F002021A700DE00B4B1A68A368D21A96
:103ED00040F6C4139A4207D90A4B05201A6822F00B
:103EE00020021A6004F086FE11B0BDE8F08F00BF1A
:103EF000C40B0020D02A0108BC1D0020E8050020CA
:103F0000720200202C020020642928BF6421F8B529
:103F100001FB00F7642497FBF4F40546E4B20026A5
:103F2000F3B2A34204D29F2001F0B0FC0136F7E7C0
:103F3000AC420BD2142097FBF0F0C4EB841366382C
:103F4000C4EB83031844C0B201F0A0FC0134E4B216
:103F5000AC4238BF9A20F7D3F8BD0F4B10B50446DA
:103F6000185C01F093FC0D4B33F91430B3F57A7FF4
:103F700005DBB3F5FA6FA8BF4FF4FA6301E04FF425
:103F80007A73A3F57A730A2293FBF2F10920C9B27E
:103F9000BDE81040FFF7B8BF9B3E0108DE060020D9
:103FA0002DE9F74F9E4A9F4913689F4D03F59C43A7
:103FB00020330B60AB68174613F4807F04D09B4B13
:103FC0001B681B681B699847AB6842F201041C40E0
:103FD0005CB9974E337873B1944B1B681B681B68B0
:103FE000984705F009FD347005E0924B1A780132CC
:103FF0001A7005F001FDAB68D80404D58E4B1B7810
:104000000BB9FEF7FFFC8D4B3C681B681E7CCEB1E4
:104010008B4A013E32F91600A0F57A70B0F57A7F2E
:10402000A8BF4FF47A7020EAE07008F0C7FE854917
:1040300008F0CCFF844908F015FF09F0FFF87D4B2C
:1040400058803EE0AB6819043BD57A4A5368E31ABE
:10405000002B36DB04F59C43203353607B4B5979AE
:104060007B4B33F81100137A80B2013303F00F0356
:104070001372D71808F0A2FE764908F0A7FF09F0DE
:10408000DDF83346787230466A4E06F109029A5CD2
:1040900001331044102B80B2F6D100B290FBF3F044
:1040A00000B26428A8BF642020EAE07008F086FE11
:1040B000694908F08BFF644908F0D4FE09F0BEF8A6
:1040C0007080AB68DA0510D5644B9C42644C08D90B
:1040D00023681B681B6A984718B923681B685B6ACA
:1040E000984723681B685B699847AA68544E12F486
:1040F000805F4D4BB5F8DC10B6F9062007D0B3F859
:104100001831581A824207DD19448A4202E0B3F896
:104110001A319A42C0F2ED820122524F0021D7F8A3
:10412000009095F8218195F822C1B5F81A41B5F8AB
:104130001CA10B46705E9B08A042C4BF63F07F03C6
:10414000DBB202315045B8BF43F040030829F1D13A
:10415000384C617E994204D1A17EF92903D80131FE
:1041600000E00021A1766376D9F88030B3B1324BFC
:104170001B783BB192B93C4B1B78DB070ED502F0A4
:10418000C5FD0BE0384B1B78580707D5BCF1000F75
:1041900002D0FEF737FC01E0002AFAD0A37E254AC0
:1041A000142B40F09380304B18F100081B7818BF97
:1041B0004FF0010803F0040303F0FF00A3B1D9F8A6
:1041C000803023B9537E5F2B01D1FEF71BFCB8F181
:1041D000000F7BD0D9F88030002B77D1637E7D2B08
:1041E00074D1FEF70FFC71E0537E572B0BD11F4BA0
:1041F0004FF47A721A801E4B1B6813F0080365D1C6
:104200001C4A138062E0A968490743D55A2B41D163
:10421000194B1978A1B318700122184B4AE000BF5E
:104220008023002024020020C01D00202002002046
:1042300028010020FC100020300200202C0100206A
:10424000DE06002000007A4400C07F4428070020DA
:1042500038070020CDCC23420000C842404B4C0020
:104260009C0B0020DC030020962300208C230020E0
:104270002C020020D40400208D0400208F04002094
:10428000D17E894B81F00101D17609B1022211E082
:1042900003220FE05D2B00F0FC815B2B00F0FB8123
:1042A0005E2B09D1F9E1A72B40F0DA817F4B1A7818
:1042B00042F004021A7009E0D9F88020002A40F088
:1042C000C7816F2B40F0BE8102F020FDD5F808C0F9
:1042D0001CF0040F2FD0E27E754B8AB1754A12781C
:1042E00052070DD5744AB6F90610B2F81A21914258
:1042F00006DD1A7822B97149322008807049CA76E1
:104300001B7C53B16F4B1A782AB96F4A127812B9D5
:104310006A4A3221118001220CE06B4B1A7852B1AB
:10432000644A127802F0040202F0FF011AB919700F
:10433000664B01221A70664B3F68002293F8018099
:104340008037104611461346434501DB00233BE00E
:10435000082BFBD02BB19C0703D1043A1030D2B20A
:10436000C0B25C4C40F2A46904EB4304268954B209
:104370001C44A6F2155A04EB440436B2BAF5C77FC2
:10438000E4B204F1010B8CBF4FF0000A4FF0010AB8
:104390004E450AFA0BFAD4BF4FF000094FF001095D
:1043A00004F1020B09FA0BF94AEA090940F2135A1F
:1043B0005645CCBF0026012606FA04F449EA040457
:1043C000844001332143BFE757F82320384E114280
:1043D0000CBF002201229A550133152BF4D17378BA
:1043E0003D4F3E4C1BB13B689B070BD416E01CF4C1
:1043F000807F13D03A4B1B681B689B689847002846
:10440000F1D10BE0228812F001030DD12C4942F0CA
:104410000102CB610B6231490A8006E0238823F058
:1044200001032380012300E00023B2788AB183B125
:10443000238823F0010203F0020392B29BB2228090
:104440005BB91F4942F00202CB610B62234B1A8019
:1044500003E0238823F0020323802388214A13F0FA
:10446000030F4FF0100114BF516111613A6812F04F
:104470000A0F47D0317949B15F070AD443F00403EA
:104480002380194B1988194B198002E023F004038B
:104490002380737963B3238858062DD40F4943F0E2
:1044A00040030B8028E000BF8E0400207202002031
:1044B0003002002096230020C01D0020740400203C
:1044C000FC1000208C0400208D0400208F040020AC
:1044D000A70B0020DE0600202C0200204602002050
:1044E0009C0B0020000C0140D40400206E0500202D
:1044F000238823F040032380B3791BB1874B1988AD
:10450000874B1980910640F1898086490B789A077C
:104510007DD5854A1278042A79D9727A9AB103F046
:10452000100303F0FF02002B78D123887F4823F08B
:10453000200343F0100323807D4B011D1A7003F00C
:10454000B9FB022268E023F010030B70794B9B7AD1
:10455000002B2ED0784B1B685989784BB3F900009B
:104560000028B8BF4042884209DAB3F90230002B74
:10457000B8BF5B428B42ACBF0023012300E013466F
:10458000DB0716D5228802F020039BB2002B45D111
:104590006B4942F020020A80654A6A4813706A4BF0
:1045A000011D1A685B680260436003F083FB01220F
:1045B00032E023885E4A23F02003238013786BBB0C
:1045C000012111701A466149002050526049614F23
:1045D0005052614907EB030C50520021D95102326D
:1045E000CCF80400CCF8081007F1280C503743F839
:1045F0000C10D9519C441F44042ACCF80400CCF878
:1046000008107860B96003F11403DCD106E0238858
:10461000002223F030032380504B1A70F37A1BB131
:10462000238843F4807302E0238823F4807323807B
:104630006B79082B01D00E2B6DD1238823F040031A
:10464000238068E0B8F1000F02D07E2B3FF43CAE2F
:10465000972B7FF428AE424B4FF4C8721A8035E690
:104660000022BB2B019201D1022303E0B72B04D11E
:104670004FF6FE73ADF8063020E0BE2B01D10223C9
:1046800004E0BD2B7FF422AE4FF6FE73ADF804308C
:1046900014E0012202E0022200E003225FFA82F825
:1046A00008F1FF3385F8A03500F0BFFD00F02CFBCA
:1046B00002202821424602F002FB07E63B68BDF8D3
:1046C0000410B3F85C200A44A3F85C20BDF806107F
:1046D000B3F85E200A44A3F85E2000F0A6FD00F0C7
:1046E00013FB0F201421012202F0E9FA0023A37624
:1046F000ECE51C4B00220021DA611A62C3F89C2011
:10470000C3F8A020C3F8A420C3F8A810C3F8AC10C5
:10471000C3F8B01001E503B0BDE8F08FD404002069
:104720008819002072020020E8050020C01900202E
:104730006C0000203002002078050020520200208A
:1047400046020020C8190020B00500209223002056
:104750007C0500202011002080050020D0190020B9
:1047600060040020FC1000202DE9F34102F092F9D2
:104770009B4DD5F8B430C31A002BC0F22E8100F542
:10478000C333A033C5F8B430964B95F8B8201E78E3
:10479000C6F38006B21A18BF012285F8B8604EB180
:1047A000002A00F01A81904B5A789A7001225A70B0
:1047B0001A7027E08C4B2AB1DA7842F00202DA70E4
:1047C0009A785A70D9788F0705D4874A9468041B61
:1047D000E443E40F00E00124834A1C7094B1CC0749
:1047E00010D51179814B01310344C9B29360032381
:1047F000B1FBF3F303EB4303CB1A7D49DBB2137137
:10480000CB5C5370784C23780BB3B02001F061F887
:10481000402001F05EF8002001F05BF8102001F06C
:1048200058F84FF48067013F0020BFB201F02AF82A
:10483000002FF8D1384601F050F86E4B627853F8EB
:10484000220001F03DF8E37823F00203E37063787F
:10485000042B00F2AD80DFE803F003AB16439800B1
:104860006549664A664805F031FD012001F035F8DA
:10487000634801F025F8634B614863491A6805F005
:1048800025FD02207BE0614C0A232178604FB1FBBB
:10489000F3F203FB12133978DBB2009158485D49FB
:1048A00005F014FD012001F018F8554801F008F852
:1048B000FEF74EFA584B247818683B7882786421CA
:1048C00003FB12444C43417802208A1A5343B4FB41
:1048D000F3F401F002F81520E1B2FFF715FB67E0F1
:1048E00001204E4F00F0F9FF4D4800F0E9FF3B6812
:1048F000990715D54B494248B1F90020B1F902306A
:10490000B1F9041003240091474905F0DFFCFEF7DC
:104910001FFA022000F0E1FF394800F0D1FF00E06B
:1049200002243B68DA0718D540493548B1F9002020
:10493000B1F90230B1F9041004F1010800913C49C9
:1049400005F0C4FCFEF704FA204600F0C6FF2C4830
:1049500000F0B6FF5FFA88F844463B681B0727D58E
:1049600034492748B1F90020B1F90230B1F90410F7
:104970000091314905F0AAFCFEF7EAF9204600F063
:10498000ACFF1F4800F09CFF12E0002460080130DB
:1049900000F0A3FF2046FFF7E0FA202000F076FFAA
:1049A000601C0234C0B2E4B2FFF7D7FA082CEDD194
:1049B0009EB9B02000F08DFF082000F08AFF17207C
:1049C00000F087FF95F8CE401C4B185D013404F0D1
:1049D000030400F05BFF85F8CE4002B0BDE8F08133
:1049E000FC1000209623002068070020404B4C005C
:1049F000A42B0108A0000020A43E0108AC3E010841
:104A0000B5110020B4000020B43E0108A405002028
:104A100092000020BF3E0108280F00202C02002039
:104A2000D73E0108A8040020ED3E0108F003002055
:104A3000FD3E01086C0200200D3F01081D3F0108EA
:104A40001FB50123ADF80830ADF80410002301A90B
:104A5000ADF80A30ADF80C30ADF8062001F099FB46
:104A600005B05DF804FB464B10B54FF4127404FB1F
:104A7000003494F83C22C2B9A36A616A994229D0F1
:104A8000591CA069A162C05C2369C0B299424FEA77
:104A9000400343F40073A4F83E324FF00A0384F855
:104AA0003D3228BFA262012312E094F93D327BB16E
:104AB000B4F83E1220464B08A4F83E3201F0010142
:104AC000FEF7ABFA94F83D32013B84F83D3201E049
:104AD00084F83C3294F83832002B4FD194F83932B4
:104AE0000133DBB2092B84F8393204D12046BDE80A
:104AF0001040FEF77DBA0A2B40D194F83B322BB917
:104B0000B4F8403243F00103A4F840326379D90786
:104B10001CD5B4F84002820501D4C30705D4B4F80B
:104B200044320133A4F8443210E0E36AC0F3470092
:104B30000BB198470AE0E3696269D054E269E3681F
:104B40000132B2FBF3F103FB1123E361012284F88C
:104B5000382294F83B220023012A84F839320DD1FF
:104B6000A27984F83B32236B012A1868197B14BFA1
:104B700002220022BDE81040FFF762BF10BD00BF57
:104B8000CC1100202A4B10B54FF4127404FB0034F2
:104B90006379DB074AD594F8383203B3236B0022DC
:104BA0001868828494F83C2222B1B4F8422201327F
:104BB000A4F84222A279197B012A0CBF022200220A
:104BC000FFF73EFF012384F83B32002384F839329B
:104BD00084F83A3284F83832A4F8403210BD94F8A0
:104BE0003B322046012B04BF94F8393284F83A3224
:104BF000FEF7FEF994F83B12236BA27949B9012123
:104C000084F83B128A421868197B0CBF02220022EA
:104C100008E0002184F83B12012A1868197B14BFB0
:104C200002220022BDE81040FFF70ABF10BD00BFFE
:104C3000CC110020426A10B58469A154416A02690E
:104C40000131B1FBF2F402FB14124262426B32B149
:104C50001368DB0708D4BDE8104005F061B9036DA7
:104C6000DA6842F08002DA6010BD2DE9F0431422C8
:104C700085B081468846214800210BF042F8042483
:104C8000013C32D01E4A0C2303FB142300277AB2C6
:104C9000A242F5DA0C214A4355181A490A44127AFD
:104CA0000D440021CEB2013112B1501E0240F9E78D
:104CB000297AD0B2013211B1481E0140F9E7321A07
:104CC000002A10DD1868596801AE324603C29868A0
:104CD00010602A4603CA596018601068986096E808
:104CE000070085E807000137D1E7044A48464146F6
:104CF00005B0BDE8F04304F009BE00BF5C1600201B
:104D00005C000020380000202DE9F74F04F04CFA39
:104D100010B90A2002F018F8924C40F2A452204632
:104D200091490AF0E5FF94F8A0354FF49A72022BEE
:104D300084BF002384F8A03594F8A0358B4F02FB84
:104D4000034303F501733B60A36842F201021A407A
:104D50003AB944F208021A401AB9824A43F400539D
:104D60009360A368DA0703D54FF40050FDF7AAFF5C
:104D7000A3685B0409D50820FDF7A4FF4FF4005099
:104D8000FDF7A0FF0120FDF79DFFA3681E0706D5D4
:104D90004FF40050FDF796FF0120FDF793FFA36845
:104DA0009D040ED54FF40040FDF78CFF4FF40060DA
:104DB000FDF788FF4FF48030FDF784FF4020FDF7BA
:104DC00081FFA368580603D54FF48030FDF77AFFC2
:104DD000A368990408D503F42063B3F5206F03D1C9
:104DE0004FF40060FDF76EFF614B624D1D6003F0F4
:104DF00067FA614B05F11A0201201A6004F0F8F914
:104E000001460120FFF731FF002840D0022004F0C6
:104E1000EFF901460220FFF728FF002837D01020C5
:104E200004F0E6F901461020FFF71FFFA3681A06F9
:104E300000D560B3082004F0DBF901460820FFF735
:104E400014FFA3681B0700D508B3042004F0D0F9B1
:104E500001460420FFF709FFA3685E0503D4002381
:104E60001A46194609E00028F9D110E079B9012164
:104E7000C00708D40C33302B0BD040481844007ABC
:104E80008507F5D5F2E70132D2B2022AF2D903F052
:104E900089F93868002390F8516090F8505003FB6E
:104EA00003F11939714301F6C4115943694340F6BE
:104EB000C41291FBF2F1324A22F813100133072B8E
:104EC000EDD190F85230B4F8D0E0B4F8D22090F898
:104ED00053C0CEEB0202C3F1640B03EB83085D42C7
:104EE00001925FFA8BFB4FEA4808CCF16409ADB23E
:104EF0000022AEB231B2002904DC002E14BF1E46DF
:104F0000012600E05E4601FB01FA76430AFB0CFA3B
:104F10009AFBF6F64E4471434FF00A0A91FBFAF100
:104F200008EB0106019936B24E434FF47A7196FBB5
:104F3000F1F614497644565202325544182AADB25D
:104F4000D7D1114B114A1360114A4C3313600278C8
:104F5000104B012A03D0022A22D00F4A21E00F4A27
:104F60001FE000BFC01D002000F80108DC03002086
:104F70002C010020CE1E0020F80800203800002060
:104F80005819002070190020B41E0020F8030020DA
:104F9000940500209400002081720008ED70000844
:104FA000414A1A60414B00F5947204301A60FDF7D3
:104FB000A3FF3E683E4D06F58E73C5F8A4343D4B05
:104FC00000229A803C4B3D4A06F59271136006F12F
:104FD000DC02C5F8A824A3F12202C5F8AC24A3F191
:104FE00028022C33C5F8B024C5F8B434344A163B33
:104FF000C5F8B83406F59373C5F8BC341160B4F83D
:10500000F00007F0D7FEC5F8C404B4F8F20007F0CA
:10501000D1FE96F86030C5F8C80485F8C03496F81B
:105020007C3005F598656B7094F82331321D2B7335
:10503000244BB6F8D8001D60234B1A60234B06F1B1
:105040006C021A60224B06F168021A6007F0B6FE85
:105050000146204807F0BAFF07F020FB0EA3D3E972
:10506000002307F06FFB07F09FFD1B4B1860706E6D
:1050700007F014FB0AA3D3E9002307F063FB024601
:105080000B460020154907F087FC07F08DFD144BF7
:10509000186003B0BDE8F08F3B597E90A9E78140CE
:1050A000182D4454FB21094009750008780500209B
:1050B000CC110020900B0020B81E002064040020BA
:1050C0008C05002098040020C4030020B8020020B2
:1050D000E404002000006144740500200000E03F6B
:1050E000E00400202DE9F7431F464FF412734343B9
:1050F0009146424A0646D41808B9414802E00128C0
:1051000004D1404820631030C4F834013E480025E3
:10511000D050032363714FF480734FF00108E360B4
:105120002361D4F8343184F83C5284F8388284F80E
:10513000395284F84662586804F134029B6862610F
:1051400004F59C72A261E1622562E561A562656277
:10515000A4F84252A4F84452ADF8043002251023BA
:1051600001A9C4F80890A7718DF806308DF8075092
:10517000FDF77CFF236B01A958689B688DF80750E9
:10518000ADF8043048238DF80630FDF76FFF414637
:105190002046FDF742FF322001F087FD1B4BD4F87B
:1051A00034811B681D46B5FBF9F1B1F5803F03D38F
:1051B000012DF8D96D08F6E7154A4046B3FBF2F227
:1051C00089B2D2B204F0A8FC404631460023114A0D
:1051D00004F042FF256B012F14BF02220022286831
:1051E000297BFFF72DFC284631460B4A002304F0AB
:1051F00033FF204603B0BDE8F08300BFCC11002090
:10520000FC3C01081C3D0108AC2B01089C0000205F
:1052100040420F00674A0008854B000803460A46D3
:1052200090F84602D96A9B795CE74B4B4F222DE9F7
:10523000F3411A7040F2A4525A80BE221A71EF2232
:1052400083F8A125002283F8A22511461E46B35CEF
:105250000132594040F2A4539A42F8D13E4B3F4AA2
:1052600083F8A2153E4B04275A6002F188325A6037
:105270000020013F17F0FF075DD0394B3422394C35
:10528000DA60C4F309037BB1331903F17843A3F562
:10529000FC33D3F800804FF400500023019301F059
:1052A00023F90428E5D11BE04FF4302001F01CF96C
:1052B0000428DED12A4D4FF430202B6943F002033D
:1052C0002B616C612B6943F040032B6101F00CF9F9
:1052D0002A6941F6FD73134004282B61D4D0C8E736
:1052E0001F4D4FF400502B6943F001032B611FFA4F
:1052F00088F3238001F0F8F8042812D1A31C01934D
:10530000019B4FEA1848A3F800804FF4005001F0C9
:10531000EBF82B6941F6FE721A4004282A6106D088
:10532000A7E72B6941F6FE721A402A61A1E70E4BEE
:1053300004349C42A5D10A4B04281A6942F0800229
:105340001A6102D103F030FF10B90A2001F0FCFC11
:1053500002B0BDE8F08100BFC01D002023016745F9
:105360000020024000F80108A4FD010810B5044621
:1053700020460AF007FD10F0FF0F07D10B4B0C4839
:1053800093F8A015BDE8104002F0ACBD20460AF02D
:105390004EFD022808D8054B064C83F8A005FFF700
:1053A00044FFFFF7B1FCE3E710BD00BFC01D0020C4
:1053B0004C3F0108804101082DE9F04F754985B047
:1053C00004460AF0A7FC7449002820460CBF0126B9
:1053D00003260AF09FFC002808BF0226F20740F1CE
:1053E000BE806E4802F07EFD002004F0AFFB6C4FE3
:1053F0006C4802F077FD6C4802F074FD7A796B4BD3
:105400006B4803EB8203596902F06CFD3869002197
:1054100007F0BCFE00285CD13C460546D4F810805D
:105420000021404607F0B2FE00284ED10135614808
:105430002946D4F814B0D4F818A0D4F81C9002F07F
:1054400051FD4046002107F0ABFE10B15A4802F072
:1054500049FD6946404602F05DFF0146574802F0AB
:1054600041FD5846002107F09BFE10B1524802F062
:1054700039FD6946584602F04DFF01464F4802F09B
:1054800031FD5046002107F08BFE10B14A4802F072
:1054900029FD6946504602F03DFF0146474802F0AB
:1054A00021FD4846002107F07BFE10B1424802F082
:1054B00019FD6946484602F02DFF0146404802F0BA
:1054C00011FD0C2D04F11004A8D13E48691C02F016
:1054D00009FD3D4802F006FD3C4CD7F8088054F821
:1054E000041F19B13A4802F0FDFCF8E70C46394BAD
:1054F00053F8245055B10123A34013EA080F03D0F9
:105500003548294602F0EEFC0134F0E7334802F05A
:10551000E9FC29467B1893F80E3104AA1344304A5B
:105520008A5C0131082903F8102CF3D10023694665
:105530002C488DF8083002F0D5FC2B4802F0D2FC44
:105540002A4804F0D9FE2A4802F0CCFC274802F091
:10555000B7FD284802F0C6FC402004F0E9FFB3077D
:1055600014D5254802F0BEFC244802F0BBFC1F48BD
:10557000FFF7FCFE224802F0B5FC1C4802F06EFD6D
:105580001C4802F0AFFC802004F0D2FF05B0BDE85B
:10559000F08F00BF593F0108603F0108683F0108D4
:1055A000C01D0020763F0108883F0108AC2B010890
:1055B000943F01089F3F01084F41010890440108B2
:1055C00068450108A73F0108B93F0108CC30010830
:1055D000C93F0108D0300108D73F0108E43F010866
:1055E0009B3E0108F03F0108F93F01088041010896
:1055F00005400108974501081340010826400108AD
:1056000034400108AFF300802DE9F04F1421012848
:1056100034BF0746012701FB07F3DFF8C4B189B0A7
:105620000BEB03025BF80340684B10691C601F71B1
:10563000674B1689DD69B2F80A902843556849EA34
:105640000608D8610222C5F8108028468DF80E1091
:1056500003A90193ADF80C808DF80F20FDF706FD2E
:10566000019B4FF0080A9B46AA68164203D10A2004
:1056700001F010FBF8E70A206E6101F00BFB2E61D0
:105680000A2001F007FBBAF1010AEDD10A20C5F8A2
:10569000149001F0FFFA0A206E6101F0FBFA0A2073
:1056A0002E6101F0F7FA0222C5F8109028468DF815
:1056B0000F2003A91C228DF80E20ADF80C80FDF7F9
:1056C000D5FC444A9442DBF8102008D142F4001281
:1056D000CBF81020DBF8102022F4001207E042F48F
:1056E0008002CBF81020DBF8102022F48002CBF8E7
:1056F0001020A38803A823F440731B041B0CA38071
:1057000023889BB243F001032380A58800F054FE58
:1057100025F03F050599304A2D04B1FBF2F22D0C1E
:105720001543ADB2A5802388012523F001031B0496
:105730001B0C2380294B03A8B1FBF3F34FF49671A4
:105740004A439BB24FF47A71002B92FBF1F208BFEF
:105750000123013243F4004392B22284A3832388BD
:105760001F4A9BB243F001032380238823F4816303
:1057700023F002031B041B0C23804FF4804323817E
:10578000142303FB07277B7B00248DF80C308DF856
:105790000D408DF80E408DF80F5000F04BFF3B7B15
:1057A0009DF80F208DF80C308DF80D401AB103A82C
:1057B00000F040FF07E0590903F01F039D40094A2C
:1057C000203142F8215009B0BDE8F08F9C1600202E
:1057D000001002400054004040420F00804F120071
:1057E000202C010800E100E008B5054BDA881879A3
:1057F000013292B2DA80FFF707FF002008BD00BF38
:105800009C16002013B51E4B400002ACC0B21872AB
:1058100004F8012D5972012200219A72D9721A7569
:105820005A751A6899759188DC6089051C6115D4D0
:105830001188CC050DD447F230511088800502D56F
:105840000139FAD112E089B1118889B241F480712D
:105850001180918889B241F44071918047F23052B1
:10586000597D11B1013AFBD100E012B9FFF7BCFF3D
:1058700003E0034B987D80F0010002B010BD00BF33
:105880009C160020024640213C20BBE770B50A4E22
:1058900000EB800006440024331913F8A00C074BDA
:1058A00001341D786840FFF7EDFF052CF4D1284640
:1058B000BDE87040E6E700BF482C01089C230020AB
:1058C00010B5441E14F8010F10B1FFF7DFFFF9E720
:1058D00010BD024680213C2094E708B55038C0B284
:1058E000FFF7F7FF0020FFF7F4FFBDE808401020A6
:1058F000EFE777204821012284E777205821012211
:1059000080E7064B002193F82020054B92013432AA
:1059100019707720F42102F0FC0273E78C07002055
:10592000B81D0020034B00221A707720F4212E228C
:1059300068E700BFB81D002007B54FF40053ADF86D
:10594000043002238DF8073004238DF806301C4BF9
:105950001C4A1B68934201D11B4803E01B4A934237
:1059600003D11B4801A9FDF781FB6B218022682030
:10597000FFF748FF052001F098F91921002268205F
:10598000FFF740FF6B2103226820FFF73BFF372121
:1059900002226820FFF736FF0E4B1A211A78682082
:1059A000FFF730FF1B2118226820FFF72BFF1C2177
:1059B00010226820FFF726FF03B05DF804FB00BF4C
:1059C0001400002000127A00000C0140001BB700F8
:1059D000001001402900002008B5192001F065F9E8
:1059E000682015210022FFF70DFF10B9032001F0F8
:1059F000ABF90C4B16211A78682042F01802FFF719
:105A000001FF172100226820FFF7FCFE3D21012243
:105A10006820FFF7F7FEBDE8084068203E2101221C
:105A2000F0E600BF2A00002013B500222A211C2026
:105A3000FFF7E8FE0E2102221C20FFF7E3FE0F21F4
:105A400003221C20FFF7DEFE2B2112221C20FFF771
:105A5000D9FE164B02249A69154842F004029A6155
:105A60002023ADF8043004230DEB03018DF806303C
:105A70008DF80740FDF7FAFA22462C211C20FFF78B
:105A8000C1FE2D2101221C20FFF7BCFE2E21002289
:105A90001C20FFF7B7FE2A2105221C20FFF7B2FECB
:105AA000044B4FF480721A8002B010BD0010024007
:105AB000000801400000002008B5642001F0F5F85E
:105AC00068202321F022FFF79DFE10B9032001F08A
:105AD0003BF9052001F0E9F8044B68201A782021F1
:105AE00042F00F02BDE808408CE600BF74070020BA
:105AF00008B50F2108221820FFF784FE0E22182077
:105B00001021FFF77FFE024B4FF480521A8008BD30
:105B10000000002008B5134B53201B782D210822CC
:105B20007BB1FFF76FFE31210A225320FFF76AFE97
:105B30002C210C225320FFF765FE532038219022A0
:105B400009E0FFF75FFE31210A225320FFF75AFEDA
:105B500053202C210A22FFF755FE034B40F2091275
:105B60001A8008BD750700200000002010B5400015
:105B70001B4CC0B220722361617201200021E360DE
:105B80002368A172E07222756075A1759A889205EA
:105B900015D41A88D0050DD447F2305219888905DA
:105BA00002D5013AFAD112E08AB11A8892B242F4CF
:105BB00080721A809A8892B242F440729A8047F2B8
:105BC0003053627D12B1013BFBD100E01BB9BDE84F
:105BD0001040FFF709BE024B987D80F0010010BD18
:105BE0009C16002037B50622044603216B461E2072
:105BF000FFF7BCFF9DF801309DF80000154D43EA0A
:105C0000002000B207F0DAF8296807F02BF907F056
:105C1000EFFA9DF8033020809DF8020043EA00204F
:105C200000B207F0CBF8A96807F01CF907F0E0FA1A
:105C30009DF80530A0809DF8040043EA002000B2E2
:105C400007F0BCF8696807F00DF907F0D1FA608039
:105C500003B030BD2C00002007B5002101AB0322AA
:105C60007720FFF783FF9DF805009DF804300002C0
:105C700040EA03409DF80630184303B05DF804FB8A
:105C800008B5FFF7E9FF014B986108BD9C1600209D
:105C900008B5FFF7E1FF014BD86108BD9C16002055
:105CA000104B13B51B78104C13B9238C013323848C
:105CB00001ABF62103227720FFF758FF9DF805304E
:105CC0009DF804201B0243EA02439DF8062013437B
:105CD000064AB2F92020C2F10802D340636202B042
:105CE00010BD00BFB81D00209C1600208C070020AE
:105CF0000B4B13B51B780B4C13B9238C0133238446
:105D000001ABF62102227720FFF730FF9DF8042037
:105D10009DF8053043EA0223238502B010BD00BF81
:105D2000B81D00209C16002013B5062204466B46C1
:105D30003B216820FFF71AFF9DF800209DF80130F5
:105D400043EA022323809DF802209DF8033043EAB2
:105D5000022363809DF804209DF8053043EA022366
:105D6000A38002B010BD13B5062204466B46432142
:105D70006820FFF7FBFE9DF800209DF8013043EA04
:105D8000022323809DF802209DF8033043EA02237A
:105D900063809DF804209DF8053043EA0223A38028
:105DA00002B010BD07B5232000F07FFF68207521E9
:105DB00001220DF10703FFF7D9FE28B19DF8070076
:105DC000B0F168035842584103B05DF804FB13B5C5
:105DD0000222044601AB1B216820FFF7C7FE9DF895
:105DE00004209DF8053043EA022303F54E534FF497
:105DF0008C72103393FBF2F32333238002B010BD77
:105E000013B5062204466B461D216820FFF7AEFE3F
:105E10009DF800209DF8013043EA022323809DF87D
:105E200002209DF8033043EA022363809DF804209A
:105E30009DF8053043EA0223A38002B010BD13B5DC
:105E4000062204466B4601211C20FFF78FFE9DF8B9
:105E500001309DF800209DF8021043EA022242F32F
:105E60008D02042392FBF3F222809DF8032042EA84
:105E7000012242F38D0292FBF3F262809DF804103E
:105E80009DF8052042EA012242F38D0292FBF3F3D2
:105E9000A38002B010BD13B5062204466B46A821AC
:105EA0006820FFF763FE9DF800209DF8013043EA6B
:105EB000022323809DF802209DF8033043EA022349
:105EC00063809DF804209DF8053043EA0223A380F7
:105ED00002B010BD13B5062204466B4602211820FD
:105EE000FFF744FE9DF800309DF801209B0803EB6E
:105EF000022323809DF802309DF803209B0803EBCA
:105F0000022363809DF804309DF805209B0803EB75
:105F10000223A38002B010BD2F4B2DE9F3411B7863
:105F20000546002B39D0002426462746A0460822E5
:105F30006B4653203221FFF719FE9DF801209DF892
:105F40000030013403EB02231BB29DF80320984478
:105F50009DF80230E4B203EB02231BB21F449DF80C
:105F600005209DF80430202C03EB02231BB21E44B5
:105F70009DF8073003F07F0301D0002BD7D1174BDA
:105F800098FBF4F897FBF4F796FBF4F6A5F800807D
:105F90006F80AE8083F82A401AE006226B465320B9
:105FA0003221FFF7E3FD9DF801209DF8003003EB5F
:105FB00002232B809DF803209DF8023003EB02237F
:105FC0006B809DF805209DF8043003EB0223AB8025
:105FD00002B0BDE8F08100BF750700209C160020CC
:105FE00013B5224C23689A8A92B20192019A12F454
:105FF000706F1CBF0122A275019A12F4E06F29D0C4
:106000001A8B9A8822F480621204120C9A80019AE8
:1060100091051FD41A8892051CD41A88D0050ED574
:106020001A88D105FCD41A8892B242F400721A8000
:106030001A889205FCD42079FFF7E6FA0AE01A885C
:1060400092B242F400721A809A8822F440721204CA
:10605000120C9A802268938A23F470631B041B0C31
:1060600093820023637502B010BD00BF9C16002010
:10607000084BDA68D10709D4DA68520708D4DB681C
:1060800013F0100F0CBF042003207047012070474D
:1060900002207047002002401E4B2DE9F0431A7881
:1060A0001D460AB31C4B07781E781C4B93F800C0A2
:1060B00002231B4A03F10108D45C344104F00F04AD
:1060C000BC420CD20B2C0AD812F8039012F80880AC
:1060D00002EB840209EA0C0408EB04241461023385
:1060E000102BE6D100232B7003788B420FD90C4B79
:1060F00093F8400060B10B4A890012780B4418698C
:1061000002B1400800F5777080B2BDE8F08300204E
:10611000BDE8F08330010020A40B0020A50B002077
:10612000C8160020A60B002007299ABF024B33F89F
:1061300021000020704700BFFC010020024B53F8F3
:106140002100C0F3CF007047A4010020034B53F897
:106150002100400800F5777080B270474C010020A4
:10616000014B33F811007047DE060020014B33F875
:1061700011007047FC17002038B50C680546204612
:1061800009F000FE214602462868BDE8384009F0C3
:1061900001BE0A88F0B54B888F880E89CD88002A09
:1061A0003AD1048C834A24F001042404240C04848E
:1061B000018B048C89B221F0F30141EA0616B6B2D4
:1061C0009042A4B246EA070743F0010315D002F556
:1061D0000062904211D0B0F1804F0ED0A2F59832FB
:1061E00090420AD002F58062904206D002F58062A9
:1061F000904218BF24F00A0401D124F00204234382
:1062000007830384038B23F00C031B041B0C038301
:10621000038B9BB21D4344E0042A44D1048C654A9D
:1062200024F010042404240C0484018B048C21F435
:1062300040710905090D41EA063189B241EA072793
:106240009042A4B2BFB212D002F5006290420ED0CA
:10625000B0F1804F0BD0A2F59832904207D002F5F2
:106260008062904203D002F58062904207D124F010
:10627000200444EA03139BB243F0100304E024F02B
:10628000A00443F01003234307830384038B23F408
:1062900040631B041B0C0383038B9BB243EA05255D
:1062A000ADB20583F0BD082A018C3ED121F4807186
:1062B0000904090C0184818B3E4A89B221F0F30163
:1062C000048C41EA0616B6B29042A4B246EA070729
:1062D00012D002F5006290420ED0B0F1804F0BD088
:1062E000A2F59832904207D002F58062904203D026
:1062F00002F58062904207D124F4007444EA03233B
:106300009BB243F4807304E024F4206443F480736C
:10631000234387830384838B23F00C031B041B0C10
:106320008383838B9BB21D4341E021F48051090498
:10633000090C0184828B048C22F440721205120D28
:1063400042EA072242EA06361A4AA4B29042B6B29C
:1063500012D002F5006290420ED0B0F1804F0BD007
:10636000A2F59832904207D002F58062904203D0A5
:1063700002F58062904207D124F4005242EA0332CF
:1063800092B242F4805205E047F6FF52224043F4B5
:1063900080531A4386830284838B23F440631B0457
:1063A0001B0C8383838B9BB243EA0525ADB28583A7
:1063B000F0BD00BF002C01401F4B10B55A6802F021
:1063C0000C02042A03D0082A04D01C4A14E01C4AF8
:1063D000126811E05A685968C2F38342C90302F196
:1063E000020201D4174906E0596811F4003F14492C
:1063F000096818BF49084A4302605968124AC1F344
:106400000311545C0168E14041605C68C4F30224FC
:10641000145D21FA04F484605C68C4F3C224145D42
:10642000E140C1605B68C3F381331A44137CB1FB64
:10643000F3F1016110BD00BF0010024000127A00AC
:106440001400002000093D006D000020CB78F0B55D
:10645000DA0648BF8A78098803F00F0548BF15435C
:1064600011F0FF0F1DD0046800220127974007EAB2
:106470000106BE4211D197004FF00F0C0CFA07FC39
:1064800005FA07F724EA0C04282B44EA070401D193
:10649000466102E0482B08BF06610132082AE4D1B8
:1064A0000460FF291FD94468002202F10806012771
:1064B000B74007EA0106BE4211D197004FF00F0C1A
:1064C0000CFA07FC05FA07F724EA0C04282B44EA27
:1064D000070401D1466102E0482B08BF0661013282
:1064E000082AE2D14460F0BD10B50446FFF7C0FDB4
:1064F000012806D11CB1FFF7BBFD013CF8E70520E0
:1065000010BD002C08BF052010BD8A6810B50C6AAC
:10651000036814430A6923F4FF4314434A6923F0D0
:10652000700314438A691443CA6914434A6A1443C2
:106530008A6A224313430360CB6843600B6883601D
:106540004B68C36010BD02684FF6FE7313400360D2
:106550000023036043608360C3602A4B984222D0CB
:10656000294B984229D0294B984230D0284B984249
:1065700037D0284B98423ED0274B984206D153F84B
:10658000682C42F4700243F8682C7047234B984201
:1065900006D153F87C2C42F0706243F87C2C704793
:1065A0001F4B984206D153F8042C42F00F0243F8D7
:1065B000042C70471B4B984206D153F8182C42F01C
:1065C000F00243F8182C7047174B984206D153F845
:1065D0002C2C42F4706243F82C2C7047134B9842D9
:1065E00006D153F8402C42F4704243F8402C7047D7
:1065F0000F4B984205D153F8542C42F4702243F8C3
:10660000542C7047080002401C0002403000024039
:1066100044000240580002406C00024080000240EA
:10662000080402401C0402403004024044040240BA
:106630005804024010B5104B4178DB688478DB4386
:10664000C3F30223C3F1040201FA02F20F21D9407D
:1066500021401143094B02780901C9B21A4482F85A
:10666000001302780120510902F01F0200FA02F221
:1066700043F8212010BD00BF00ED00E000E100E084
:106680002DE9F843574B0C460168013AC3F8421014
:106690008188A3F84610072A42D8DFE802F0040AEE
:1066A000101822292F35B3F842202280B3F8442055
:1066B00013E0B3F844202280B3F8422005E0B3F899
:1066C000422052422280B3F84420524205E0B3F8FF
:1066D000442052422280B3F842206280B3F8463010
:1066E0001DE0B3F8422052422280B3F8442012E069
:1066F000B3F844202280B3F842200CE0B3F84220E3
:106700002280B3F8442005E0B3F8442052422280AE
:10671000B3F8422052426280B3F846305B42A38015
:10672000314B1B78002B5AD1B4F9000006F046FB20
:106730008046B4F9020006F041FB0746B4F90400B4
:1067400006F03CFB294D06462968404606F08AFBC8
:10675000E9688146384606F085FB0146484606F062
:1067600079FAA9698146304606F07CFB0146484625
:1067700006F070FA09F02AFD69682080404606F0AC
:1067800071FB29698146384606F06CFB0146484694
:1067900006F060FAE9698146304606F063FB01467F
:1067A000484606F057FA09F011FDA9686080404696
:1067B00006F058FB69698046384606F053FB0146EF
:1067C000404606F047FA296A0746304606F04AFB7B
:1067D0000146384606F03EFA09F0F8FCA080BDE814
:1067E000F88300BFC81600202800002040070020C2
:1067F000074B084A1B7812889A4207D3064A126848
:10680000907898428CBF002001207047002070478C
:10681000A40500202C0F0020280F002010B5194BD4
:1068200093F84820511C83F84810174902F00702DA
:106830004878164903EB420331F81010A3F84A10C8
:1068400000231846124A9A5A02331044102B80B281
:10685000F8D1C00806F0B2FA0E4906F003FB0E4963
:1068600006F0B4FB0D4B04461B68187806F0A6FA38
:106870000146204606F0F6FA06F0E0FC084B1870D8
:1068800010BD00BFC81600202807002038070020D0
:10689000121700203333534000F07F45280F0020AB
:1068A000A4050020034B1B68DA79511CD9711344ED
:1068B000187A70473C06002010B5FFF7F3FF044636
:1068C000FFF7F0FF04EB002080B210BD10B5FFF71A
:1068D000F3FF0446FFF7F0FF04EB004010BD064B4A
:1068E00010B5044621461868FBF7B2FE034B1B683F
:1068F0009A7954409C7110BD400600203C0600204F
:1069000038B5044624200D46FFF7E9FF4D20FFF778
:10691000E6FF002C084C0CBF3E202120FFF7DFFFD4
:106920002368002228469A71FFF7D9FF236893F85D
:106930004900BDE83840D2E73C060020014600206F
:10694000DEE7F8B50E4E0F4C0F4DC1B2074630686A
:1069500084F85A10FBF77CFE2B6894F85A109A7949
:1069600030684A409A71C7F3072184F85A10FBF740
:106970006FFE2B6894F85A109A794A409A71F8BDC4
:1069800040060020C81600203C060020F8B51B4D2C
:106990001B4C1C4F0646C1B2286884F85B10FBF7FD
:1069A00057FE3B6894F85B109A7928684A409A71C0
:1069B000C6F3072184F85B10FBF74AFE3B6894F8A6
:1069C0005B109A7928684A409A71C6F3074184F8A7
:1069D0005B10FBF73DFE3B6894F85B109A792868E2
:1069E0004A409A71310E84F85B10FBF731FE3B6828
:1069F00094F85B109A794A409A71F8BD40060020DD
:106A0000C81600203C06002010B5441E14F8011FD3
:106A100021B1034B1868FBF71BFEF7E710BD00BF61
:106A2000AC0900200B4AA2F13003197A81420BD045
:106A30000C339342F9D1084B197A014004D10C333D
:106A40009342F9D1084603E018460BB158687047E5
:106A5000704700BF6800002038000020002305496F
:106A6000DAB2595C814203D00133092BF7D11A46BF
:106A700010467047A041010801460023044818440D
:106A800042688A4203D00C33302BF7D10020704784
:106A90003800002010B5094A094913688C6812684B
:106AA0009342F8D1074A106811684FF47A72504344
:106AB000001BB0FBF1F002FB030010BDBC1D002069
:106AC00010E000E02407002038B5124B124C996802
:106AD000124B1A681D4652880A4203D0FFF7DAFFAC
:106AE000E06511E0FFF7D6FFE36D98420CD9C01ABC
:106AF0000B4B3B22B0FBF2F01B68B0F5967FC8BF92
:106B00004FF0FF3003B118602B685A68054B5A618B
:106B100038BD00BF000C0140C8160020D40300207F
:106B2000D00300200004014038B5104C0123054675
:106B300084F84030FFF7AEFF236E41F28832C31A6B
:106B40009342636684BF002384F8683094F8683009
:106B5000EDB20F2B2066E55403D1054B01221A70CC
:106B600038BD024A013382F8683038BDC8160020AB
:106B70003001002010B50446FFF78CFF0D4B41F2A9
:106B80008831DA6ED866821A8A421A6784BF002278
:106B900083F8742093F87430074A142BD45403D12B
:106BA000064B01221A7010BD024A013382F874307C
:106BB00010BD00BFC8160020E5010020E401002040
:106BC00010B50446FFF766FF164A936F9067C31A25
:106BD000B3F57A6F84BF002382F87C3092F87C3062
:106BE00023B9A82C1CD110490B7006E0022B02D14E
:106BF0000E490C7001E0242B01D80D49CC5401330F
:106C0000DBB282F87C30094A127852000532934296
:106C100006D1044B002283F87C20034B01221A701A
:106C200010BD00BFC81600207C010020A20100207A
:106C30007D01002038B50446FFF72CFF124B40F6CB
:106C4000C411D3F88020C3F88000821A8A4284BF1E
:106C5000002283F8842093F884200AB90F2C11D1E4
:106C60000A480021017052B1094D182A154405F84F
:106C7000014C04D1012283F88410027038BD013226
:106C800083F8842038BD00BFC816002031010020E1
:106C90003201002038B50446FFF7FCFE0546FFF739
:106CA000F9FE401BA042FAD338BD10B504462CB102
:106CB0004FF47A70FFF7EEFF013CF8E710BD2DE9C5
:106CC000F04106460F4690460025EBB2434518D2E8
:106CD0000024E3B2B3420FD20B4B0120DA68013437
:106CE00082F00802DA60FBF785FC3846FFF7DDFF2B
:106CF0000020FBF77FFCECE73C20FFF7D6FF0135D7
:106D0000E3E7BDE8F08100BF000C01400B490B78C0
:106D100013F0010F03F004020AD072B9980707D4E8
:106D200043F004030B70064B1A88064B1A80704719
:106D30001AB90220FF210122C1E7704796230020E3
:106D4000D40400208819002040F2DB14604308B509
:106D50000D4B10225A6108221A61841E0A4B2046EC
:106D6000DA6882F01002DA60DA6882F00802DA602B
:106D7000FFF79BFF0120FBF73DFC1920FFF795FF74
:106D80000020FBF737FCE9E7000C0140A14B2DE99F
:106D9000F04F1B7885B0013B012B00F237819E4BF1
:106DA0001D78854240F032819C4B1B78022B00F00D
:106DB0002D819B4E002333809A4B13F805B09A4BDC
:106DC00083F800B0994B1A7803921AB1984B33F9B3
:106DD000150008E0974B1A6802F100421A60944AC5
:106DE00032F91500404205F0E9FF934906F0EEF84C
:106DF0009149044606F036F806F0FAF98D4F8E49AF
:106E0000D7F800A01FFA80F85046A6F8028006F0D6
:106E100029F806F0EDF9DFF84092B080D9F80020AB
:106E200000211046029206F0B1F90027834B029A26
:106E3000002857D01A68204611460292019306F0A6
:106E4000CDF9029A019B38B11C607D4BC3F800A0BC
:106E5000734BA3F80680BFE01046394606F0BEF932
:106E6000002800F0B980774B1A789846002A31D173
:106E70002046514605F0ECFE4FF07E5106F090F9A9
:106E8000714C28B16068714905F0ECFF60600FE05B
:106E90006F49606805F0E6FFDFF8D0918246494609
:106EA00006F07EF910B9C4F804A001E0C4F804901B
:106EB000012388F80030674B00221B685B449A72FC
:106EC000039A82F00103594A1370634B1F605B4BB6
:106ED0001F6081E0614BC9F800401A68584BFA32D4
:106EE0005A6079E020461146019306F059F9019B5A
:106EF00020B1594A14604A4AA2F80680D3F80080AB
:106F0000554B4046D3F80090494605F0A1FE534B3F
:106F1000824619684A4B5A688A1A002A0BDA4FF0DF
:106F20007E5106F05BF9002856D02046494606F00F
:106F300055F9002850D0424A4046116806F04EF9F3
:106F4000414C48B1012320684149338005F08AFF54
:106F50003E492060A06809E0022350464FF080417E
:106F6000338006F03BF928B1A068394905F07AFF73
:106F7000A06004E02068354905F074FF2060354BBF
:106F80002D492068D3F8008005F06CFF06F056F913
:106F900008F80B00A06806F051F9039AD84482F073
:106FA0000103224A88F8140013702B4B1F60234BF7
:106FB0001F60244B1A780132D2B2032A01D01A7012
:106FC0000AE000221A70204B2549586805F04AFF54
:106FD00006F034F988F80A0015B933886433338031
:106FE000124A13780BB11F4B00E01F4B114A13607C
:106FF0000F4B33F9150005F0E1FE0F4905F0E6FFF0
:107000000C4A0146106805F023FE00E0084605B072
:10701000BDE8F08FF80400204C0500205C0500203E
:10702000081D0020702301085D0500204D0500208B
:1070300098030020FC04002000002041540500209B
:10704000501700204E050020600500200AD7833F1E
:10705000EC51783F5805002050050020BC1D002051
:1070600000007A440000A0410000A0C16F12833AE2
:1070700010B50848FFF7C8FC074B1C682046FBF713
:10708000C6FA18B90A20FFF710FEF7E7034A044BC7
:10709000DA6010BDEC400108AC0900200400FA05DC
:1070A00000ED00E008B50448FFF7AEFCFEF7BDF8C0
:1070B000BDE80840FFF7DCBFF840010810B5044602
:1070C0000748FFF7A1FC074A002313729363064A9F
:1070D000137002F075FC2046BDE81040E2E700BFE7
:1070E000FF40010850170020902300202DE9F04FA9
:1070F000002487B0074603919146049382462546B3
:10710000022DDFF878814FEA450607D103984379CD
:10711000B8F904001B3343435B1148E04D4B38F989
:10712000151033F9153003EB4101C9F10003994201
:1071300003DB4945B4BF0B464B464749049A31F936
:1071400006B0915FCBEB030303EB010BFBF747FCAE
:1071500098B1424B58465B5D029305F02FFE4049C3
:1071600005F034FF029B01461846FFF70FFE3C492D
:1071700005F078FE06F03CF883463A4B1988C807BC
:1071800011D403988A07037938F9060003F11B0329
:1071900000FB03F34FEA231309D57A7C02FB0BFBB8
:1071A00003EB2B2303E0FB7903FB0BF31B112E4AAC
:1071B0002E49905F042290FBF2F0181A7B5D9AF83A
:1071C0000AC0434305932A4B6258B3F800B0013517
:1071D0000BFB00F3DB120CFB0323264AB3F5001F65
:1071E000A8BF4FF400139342B8BF1346635022491F
:1071F0004FEA1B1B62584FF6FF7C821ABCFBFBFC5C
:107200000CFB02FC605001F1180B01F10C0054F86A
:10721000008054F80B204FEAAC1C44F800C04244F4
:107220009AF814006244019242430598121202EB4C
:10723000E012243102EB6333032D44F80B808B53AF
:107240000AF1010A04F104047FF45AAF07B0BDE863
:10725000F08F00BF9223002098030020C82E010861
:107260000000204146020020E80400209811002080
:10727000F00400200000E0FF8C17002052020020E4
:107280002DE9F04F89B00793914B0692B3F9022094
:10729000B3F90030002AB8BF5242002BB8BF5B429E
:1072A00000249A42B8BF1A46039005922646A1468A
:1072B00027460494A0462546DFF844A2BAF80030D9
:1072C00099075AD0022D58D0814BDDF818B0F25EE4
:1072D000804BF35E03EB4202CBF100039A4203DBE7
:1072E0005B469A42B8BF13467B4ADDF81CC036F9AC
:1072F00002B03CF90620CBEB030303EB020BFBF7D8
:107300006EFB90B1754B584615F8038005F056FD9D
:10731000734905F05BFE01464046FFF737FD7049B3
:1073200005F0A0FD05F064FF834603996423CA7944
:1073300002FB0BF292FBF3F2CB7E6FF0040101FB38
:1073400003F8424505DB03EB83039A42B4BF904642
:107350009846644A42F21071A3585B448B42A8BF1E
:107360000B4661498B42B8BF0B46A350039A92F873
:1073700011B00BFB03F31B130493BAF8003003F0B6
:107380000302012A01D1022D3ED15849504A895F9A
:10739000B75EDDF80CB0564A81EAE170A0EBE1700F
:1073A000B0F5206F1BF805C054F802901DDC022DCB
:1073B00015D05020784390FBFCFC042091FBF0F1A9
:1073C000C1EB0C0CE1444B48B9F57A5FA8BF4FF410
:1073D0007A598145ACBF42F80490105107E087EA22
:1073E000E770A0EBE7706428E3DD00211151404A0B
:1073F000A1587D2291FBF2F9039A2A44927A02FB6A
:1074000009F9402299FBF2F99A0716D5022D14D0FA
:10741000DDF814C0DDF810B00CFB07F30CFB09F02D
:10742000CCF5FA7101FB083301FB0B014FF4FA7242
:1074300093FBF2F391FBF2F108E0DB0701D5022D9B
:1074400002D149463B4601E004994346274ADFF80A
:10745000B4B0B25A04200FFA82FC15F80BB09CFBB2
:10746000F0FA0BFB0AFB6FF04F0A9BFBFAFA9A4407
:10747000214BCDF804A036F903A0F252CAEB0C0C54
:107480009CFBF0FC03F1120A981D225854F80AB034
:1074900044F800C019489344285CCDF808B0E34490
:1074A00044F80A2000FB0BF2202092FBF0F2DDF8FA
:1074B00004C08A1A0135063B6244032DF25204F1DE
:1074C000040406F102067FF4F7AE09B0BDE8F08FC0
:1074D000520200209223002098030020C82E0108A9
:1074E0000000204118110020F0D8FFFFE804002020
:1074F0009811002080C1FFFFB61700206C190020F2
:1075000046020020661900202DE9F04F89B007934C
:107510007A4B814618880491059205F04BFC784916
:1075200005F0A0FC002403904F4625462646022E77
:10753000DFF80CA20BD10499BAF904004B790A3395
:10754000584305F03BFC6F4905F040FD44E06E4BAD
:107550003AF90520EB5E05991A444B429A4203DB47
:107560000B469A42B8BF1346684AAA5E9B1A079A0E
:10757000505F184405F022FC654905F027FD804660
:10758000FBF72DFA28B1634B4146985DFFF7FEFBF0
:107590008046614B1A88D10705D54046D9F844107A
:1075A00005F060FC18E004993AF905000B790192A6
:1075B0001433584305F002FC524905F007FD019AC7
:1075C0008346930709D5D9F84810404605F04AFC90
:1075D0000146584605F03EFB8346504A505F05F091
:1075E000EDFB4F4AD16805F03DFC824651465846B6
:1075F00005F02EFB396A804605F034FCDFF844B113
:1076000006900399404605F02DFCF96A05F02AFC26
:1076100054F80B1005F01EFB4249804605F0C0FDF2
:1076200038B94046404905F0D9FD20B1DFF8F8806F
:1076300001E0DFF8F0804BF80480DFF80CB1504631
:1076400054F80B1005F004FB44F80BA00346039913
:107650004FF07E50029305F0B9FC029B014618469C
:1076600005F000FC0BF10C03E2580BF1180B54F879
:107670000B10824610460192029305F0EBFA514638
:1076800005F0E8FA019A029B44F80B2044F803A0A5
:10769000264905F09BFCB96B05F0E4FB24498246C2
:1076A00005F07EFD38B95046224905F097FD20B11E
:1076B000DFF880A001E0DFF878A00698414605F0E9
:1076C000C9FA514605F0C4FA08F080FD1A4BB0F52E
:1076D0007A7FA8BF4FF47A709842B8BF1846013637
:1076E000164B032EE85204F1040405F1020507F1DC
:1076F00004077FF41CAF09B0BDE8F08FF004002050
:10770000BD378635000048429223002098030020B0
:1077100000002041C82E010846020020E804002095
:10772000E003002000007AC300007A4300004040DC
:10773000000096C30000964318FCFFFFB01700201E
:1077400052020020A4110020D41700202DE9F04798
:10775000704B86B01A789946DFF8C88192B9D8F88C
:1077600000400123204689F80030FFF785F9022305
:107770004372694B6948C3F8A840FFF745F9684868
:10778000FFF742F9D8F80000FAF750FF002800F0A0
:10779000BE80644B604C1868FAF743FF0928014625
:1077A00001D03F284FD14FF0000AA56B5E4F5646DF
:1077B0002DB15E4839682A4608F0ECFA10B9BA468D
:1077C00006B93E465A4B0C379F42F1D3CEB13768CB
:1077D000DAF800E02B46F85C1EF80310814201D075
:1077E000A3630EE05A1C41B92D2B06D8A263234493
:1077F000202022441872117203E04C495854134659
:10780000E9E7A36B0BB1564512D04A48FFF7FCF8E5
:10781000564509D856F80C0BFFF7F6F8D8F80000D3
:107820000921FAF715FFF3E73D48FFF7EDF80025CA
:10783000A36B9D42A6D23D4BD8F80000595DFAF7E4
:1078400007FF0135F4E7A36B33B904283BD104F1FA
:107850000800FFF733FC5AE00C2801D136488CE7CA
:107860000A2901D00D2949D13448FFF7CDF8A36B7F
:10787000E21800231372227A232A17D00493304B84
:107880002A4E009303A8284913220C23039608F0DC
:10789000D2FA054638B1006808F074FA0130AB68D6
:1078A0003044984702E02748FFF7AEF81F48002110
:1078B000302208F026FA0023A36399F80030002B49
:1078C0007FF45DAF23E00C28C8D07F2903D159E7AE
:1078D0002F2B3FF657AFA1F12002D2B25E2A3FF61E
:1078E00051AF13B920293FF44DAF5A1CA263D8F809
:1078F00000001C442172FAF7ABFE43E77F29E7D171
:10790000013BA363002223441A720F4838E706B0F4
:10791000BDE8F08790230020501700201441010893
:107920004C410108AC090020EC2F01085817002039
:10793000D03001085141010856410108974501081E
:1079400079610008614101087D4101082DE9F74F87
:10795000BF4AC04C106851686B4603C3DFF82C83E4
:10796000002140F2A452204608F0CBF904F501733F
:10797000C8F800304F2323700323637140F24C4258
:107980000223A360A4F81A214FF4167340F26C721C
:10799000A4F8F030A4F81C21FA231922A4F8F2303C
:1079A00084F823212A2340F27E42A4F8EE30A4F882
:1079B000D0204FF4FA7340F23A72A4F8F630A4F8EB
:1079C000D22020234FF47A7284F8F430A4F8D42023
:1079D0006E2340F27E5284F80431A4F8D6202B2383
:1079E00040F2EA524FF0320984F80531A4F8D82069
:1079F000212340F2B452012684F8063140F2DC5BC8
:107A00004FF4C873A4F8DA20A4F8DC9084F8EC6092
:107A1000A4F8083184F8226184F82561A4F8DE30E6
:107A2000A4F818B1A4F8E09000F0BCFB40F6AC5309
:107A3000A381D8F8003000251E21A573D97399734E
:107A40000B211972142117225972197550211A76B7
:107A50005A769977552264219A71D9772D22082078
:107A600078211A74D8745A775973DA75DFF820E2DE
:107A7000794A7A490E20282798724FF00A0A5A202C
:107A8000D87283F82160C3F824E01D701F715F7104
:107A90009D7683F807905D74DD769D741D7783F87D
:107AA00015A01F731A63D96319644FF08241D9621C
:107AB0004FF07C5199636A495A631A67694A59645D
:107AC0006949C3F828E083F85000DFF8C8E1412095
:107AD0005A67664A996483F8510059660420152153
:107AE00083F860009A6783F87C60C3F84CE083F801
:107AF000545083F8555083F85650A3F858B083F883
:107B0000529083F85350A3F85C50A3F85E50A3F84A
:107B10005A5083F8687083F8697083F86C10544881
:107B200000F064FBD8F800304FF44872A3F8D82076
:107B3000C82283F81D214FF49662A3F81E2140F25B
:107B4000D932A3F8202140F6430283F8D760A3F886
:107B5000222183F8D45083F8D55083F8D67083F867
:107B6000DA5083F81CA11A4646464FF47F71A2F8FA
:107B7000DC104FF4FA61A2F8DE1040F2DC51A2F8FA
:107B8000E0101DF80510013582F8E210082D4FF0C5
:107B9000FF0182F8E31002F10802E6D1012283F826
:107BA000242183F8252183F82621C82183F82C215C
:107BB0006422A3F82811A3F82E2114214FF4967201
:107BC00083F82A11A3F830211E21282283F82B11D3
:107BD000A3F832210023E21810330021C02B1161D9
:107BE000F9D124480021402208F08BF800232249D3
:107BF000E218595804330868382BC2F8C401F6D18A
:107C00001E480021802208F07CF81D4B1B4C03F11C
:107C1000300518685968224603C20833AB4214463F
:107C2000F7D1FBF7A5F8FBF7DFF8FBF7B9F83468F5
:107C30004FF49A722146134808F05AF81248214628
:107C40004FF49A7203B0BDE8F04F08F051B800BF8E
:107C5000CA2E0108C01D00209A99193F8FC2753D98
:107C6000CDCC4C3DF6287C3F0000A0403D0A773F3C
:107C700081410108841F0020D4230108041F002033
:107C8000D22E0108F82000202C220020DC03002046
:107C9000000020400000404008B50548FEF7B4FE53
:107CA000FFF754FEFDF7C1FABDE80840FFF7E0B961
:107CB0008A410108F7B50368174C184D23600B681B
:107CC000174E63600068FBF7F9F895E80300154B61
:107CD0000196009394E80C00FBF7AEF83668124B5F
:107CE00060681E606B68114FC01A05F067F8104B92
:107CF000196805F0B7F805F07BFA22682B68786000
:107D0000D31A3B600B4B1E600B4B1B68DA880B4B86
:107D10001A8003B0F0BD00BFA0100020B005002005
:107D2000AC100020A8100020E8100020B0100020A7
:107D300068000020E010002078050020DC10002002
:107D400008B5FDF772FAFCF7DFFFBDE808400F2029
:107D500014210122FEF7B3BF2DE9F04F064689B08A
:107D60000F4615469B462978002900F0B880252942
:107D700002D001353046B0E06C78302C03D00235AB
:107D80004FF0000903E0AC784FF001090335A4F18E
:107D90003003092B4FF000081AD8A4F13003DAB2EF
:107DA000092A07D80A2B13DC0A2202FB083815F827
:107DB000014BF2E7A4F16103052B02D8A4F15703AC
:107DC000F0E7A4F14103052B02D8A4F13703E9E75A
:107DD0006C2C03BF2C78012201350022632C66D065
:107DE00006D8252C77D0582C3FD0002C77D0BAE776
:107DF000732C63D002D8642C11D0B4E7752C02D058
:107E0000782C32D0AFE70BF1040A05ACDBF80000A8
:107E10000A2112B10022234613E0234620E00BF191
:107E2000040A05ACDBF8000072B1002806DA2D2345
:107E30008DF8143040420DF1150300E023460A216D
:107E40000022FAF7DFFE0DE0002806DA2D238DF878
:107E5000143040420DF1150300E023460A210022B0
:107E6000FAF7A8FED34600941AE00BF1040303933B
:107E70000DF1140ADBF80000102132B1583C6242C7
:107E800062415346FAF7BEFE06E0B4F158035A4287
:107E90005A415346FAF78EFEDDF80CB0CDF800A03B
:107EA0003046394642464B46FAF7E8FE5BE7304635
:107EB0009BF800100BF10404B8470AE0DBF800302F
:107EC000304600933946424600230BF10404FAF78A
:107ED000D5FEA34647E730462146B84743E709B0F9
:107EE000BDE8F08F0FB407B50A4904AB08680A492A
:107EF00053F8042B09680193FFF72EFF074B18680E
:107F0000FAF785FB0028F9D003B05DF804EB04B064
:107F1000704700BF200700201C070020F817002032
:107F2000F8B5074607F02EFF044638B9194B1A4832
:107F30005A791A4B013A53F8221028E0384618496A
:107F4000224607F027FF60B91648FEF75DFD164C84
:107F500054F8041F19B11548FFF7C4FFF8E7144897
:107F600005E000250D4B53F8256026B91148BDE802
:107F7000F840FEF749BD38463146224607F00AFF71
:107F800001350028EED1034B0B485D713146BDE849
:107F9000F840A7E7C01D0020A9410108C42B010833
:107FA00082470108BD410108C02B0108D0410108EA
:107FB00097450108D4410108E941010870B504461C
:107FC00007F0E0FE08B91E482EE020461D4907F0E4
:107FD00053FF00242646254678B12CB1012C06D14A
:107FE00007F025FF064602E007F021FF0546154988
:107FF0000020013407F040FFEEE70B2D04D9BDE867
:10800000704011480C216DE7012C07DC0F4B29460D
:1080100033F915200E48BDE8704063E7A6F57A7382
:10802000B3F57A7F03D90B48BDE870405AE70A4898
:1080300029463246FFF756FF044B23F8156070BD02
:10804000FB4101084F41010835420108A8190020F1
:108050005B420108734201089542010838B50546A4
:1080600007F090FEC0B270B90446124B04F1200232
:108070001B682146104853F822200134FFF732FFD5
:10808000152CF2D138BD284607F0D1FE142804463D
:108090000BDC2021284607F068FE07F0C8FE054BE0
:1080A00020341B6843F8240038BD04481521BDE87E
:1080B000384017E7DC030020AE420108BA4201084D
:1080C0002DE9F743044607F05DFEC0B290B9304C8D
:1080D000054694F8C711B4F8C42194F8C6312D4868
:1080E000009129460135FFF7FDFE102D04F104042F
:1080F000EFD14AE0204607F09AFE0F28054636DC0D
:108100002046202107F031FE234FEDB2D7F8009032
:10811000441CAD000026204607F089FE5FFA86F871
:10812000B8F1010F83B208D0B8F1020F0BD0B3F54C
:10813000B47F1ED23A6853530AE0FF2B19D83B682C
:108140002B44987004E0FF2B13D83B682B44D87065
:1081500020462C2107F009FE044608B1441C02E029
:10816000B8F1020F05D10136032ED4D10DE00B4832
:1081700006E009EB05000021042207F0C2FD0848D3
:10818000102103B0BDE8F043ACE603B0BDE8F083D6
:10819000C01D0020E0420108140F0020F442010835
:1081A0001843010810B52720FEF758FC0E4C84F840
:1081B00028011020FEF752FC84F829010020FEF768
:1081C0004DFC4FF4E133C4F82C31C4F83031C4F81D
:1081D0003431C4F83831522384F82A0184F82B0151
:1081E00084F83C3110BD00BFC01D002070B50546AD
:1081F000441E14F8011F61B1064E304607F0B5FD6C
:108200000028F6D0861B0448631B304480F80E31EA
:10821000EFE770BD9B3E0108C01D00207FB50446FE
:1082200007F0B0FD082824D100231F49E25C09684B
:108230001144497801F00301022908BF203AE254B1
:108240000133082BF1D10025665D1848314607F04F
:108250008CFD28B101356019314607F086FD18B153
:108260001348FEF7D1FB1CE0082DEDD12046FFF7A7
:10827000BDFF1048FEF7C8FB00230F4A04A91A44AB
:1082800092F80E210A440949595C0133082B02F87F
:108290000C1CF2D10023094801A98DF80C30FFF71E
:1082A00021FE04B070BD00BFB80000209B3E010855
:1082B0002643010846430108C01D00206845010807
:1082C000F0B500231946CEB200220C2505FB02F7BB
:1082D0000D48D4B23F5CB74203D00132042AF4D136
:1082E0000BE0FF2C09D0094A05FB04001A4492F860
:1082F0002821074C0133A25C02720131052901D00B
:10830000032BE0D9F0BD00BF38000020C01D0020C5
:10831000A041010830B587B005460C4603A80021EE
:108320000C2207F0EEFC2846002104F057FF20B194
:1083300028462A4904F08EFC03E02846274904F029
:1083400087FC274904F08EFD04F052FF054685EABC
:10835000E570A0EBE57069460A22FAF77BFC002382
:108360009D420370ACBF20232D2368468DF80C304E
:1083700007F008FD012807D130238DF80D308DF866
:108380000E308DF80F300CE0022805D130238DF827
:108390000D308DF80E3004E0032804BF30238DF833
:1083A0000D30694603A807F0D3FC03A807F0EAFCE8
:1083B0000338C5B22A4603A9204607F00DFD002365
:1083C00063552046074907F0C3FC03A9204629440A
:1083D00007F0BEFC204607B030BD00BF6F12033A65
:1083E00000007A445B43010837B502790D46110657
:1083F0000446836806D526494FF49A7091F8A01573
:1084000000FB013302F03F02042A12D006D8012AF1
:108410000DD0022A2FD193F900102DE0102A0AD096
:10842000202A0AD0082A26D1B3F9001024E01978AE
:1084300022E0198820E019681EE069461868FFF7F5
:1084400069FF01461348FFF74DFDF5B1E06804F000
:10845000B5FC6946FFF75EFF01460F48FFF742FD96
:10846000206904F0ABFC6946FFF754FF01460A4857
:10847000FFF738FD09E000210848FFF733FD25B17B
:108480000748E1682269FFF72DFD03B030BD00BF4A
:10849000C01D0020904401088F440108D43E01080B
:1084A0005D4301082DE9F04389B0044607F06AFCFA
:1084B000C6B2002E6CD18B48FEF7A6FA8A4C206912
:1084C000002104F063FE40BB013688483146FFF7C7
:1084D00009FD206904A9FFF71DFF01468448FFF745
:1084E00001FD606904A9FFF715FF01468048FFF709
:1084F000F9FCA06904A9FFF70DFF01467C48FFF7CE
:10850000F1FCE06904A9FFF705FF01467948FFF790
:10851000E9FC0C2E04F11004D1D10025764C2F4635
:108520002B464FF00008B04504F1100415DA184648
:1085300054F8101C04F08EFB54F80C1C814628469D
:1085400004F088FB54F8081C0546384604F082FB0A
:1085500008F101084B460746E5E768480193029594
:108560000397FEF751FA002401ABE058644920F06C
:10857000004004F033FE634B634A0434002814BF08
:1085800010461846FEF740FA0C2CEDD15F4891E0FA
:1085900020465F49052207F0FDFB38B9524B002207
:1085A00003441030C0281A61F8D197E02046594999
:1085B000042207F0EFFB06462046002E40D1202182
:1085C00007F0D3FB002800F08980451C284607F0FF
:1085D000D9FB34468046504B53F824600EB94F48BF
:1085E00068E0284631465FFA88F207F0D3FB671C43
:1085F00020BB3D4B0021C2181030C02811619C46A1
:10860000F7D1474B002403EBC702D2F804E09846A9
:10861000BEF1000F04D143483146FFF763FC55E03B
:1086200018F837309C42F6DA23010CEB03051035BD
:1086300073440FCB013485E80F00F1E73C46CAE7ED
:1086400007F0F5FB461E0B2E074643DC2046202193
:1086500007F08BFB054640B1451C2846FAF714FA93
:10866000214B3F01D851012400E004462846202137
:1086700007F07BFB054640B1451C2846FAF704FA93
:10868000194B013403EB061358612846202107F0EB
:108690006CFB054640B1451C2846FAF7F5F9124B2C
:1086A000013403EB061398612846202107F05DFB97
:1086B00018B91D48FEF7A8F910E00130FAF7E4F9FF
:1086C000094B032C03EB0616F061F2D11748FFF7B4
:1086D000E9FE03E016480C21FFF704FC09B0BDE8F1
:1086E000F08300BF6C430108C01D002097430108C0
:1086F0009D43010868450108D41D0020A1430108DD
:108700000AD7233C684301086443010897450108E0
:10871000B0430108B6430108C42B0108D441010845
:108720002C240108BB430108CB4301088041010808
:108730000544010870B5447986B004F004038668E6
:1087400003F0FF0523B14FF480654FF4005300E0C0
:108750002B4614F0010F14BF04220022A107046D60
:1087600048BF42F00802218A48BF92B289B221F480
:1087700040510B432382A38901A89BB223F4B05339
:1087800023F00C031D432A43A281A38A23F44073E0
:108790001B041B0CA382FDF70FFE1649049A039BD2
:1087A0008C4208BF1346A2891921594312B2002AEC
:1087B000B4BF7600B600B1FBF6F16423B1FBF3F26F
:1087C0001201100903FB1011A08900B2002806DA7B
:1087D000C9003231B1FBF3F303F0070305E00901EF
:1087E0003231B1FBF3F303F00F031A4392B222814B
:1087F00006B070BD0038014041719BE7816099E788
:10880000038A828911EA030092B203D011420CBF9D
:108810000020012070471FB50123ADF80830002368
:10882000ADF80C30ADF80A30084BADF804101B78E9
:1088300001A9012B08BF0323ADF8062008BFADF83E
:108840000C30FDF7A6FC05B05DF804FBB009002074
:1088500038B5104C04EB0014A278E36842B9012249
:10886000A270A1801868197B0222BDE83840D2E7C7
:10887000A288E1806078891A074A89B2002522F827
:108880001010A57021811868197B2A46FFF7C3FFD5
:10889000A57238BDFC090020FC1700202DE9F74F18
:1088A0009F4E9B4633780C4691465A1C054606F867
:1088B000042B0068224649460C275F4301F038FC30
:1088C000AB686868ADF8043018238DF8063001A94C
:1088D00002238DF80730FAF7C9FB2B7B06EB070A5A
:1088E0002C680C2B00F2F280DFE813F00D00F00092
:1088F000F000F0004D00F000F000F0008200F00009
:10890000F000F000B600238C864823F001031B041E
:108910001B0C2384218CA288238B844223F07303B5
:108920004FEA03434FEA134389B292B243F0700314
:1089300014D000F50060844210D000F540608442FD
:108940000CD000F58060844208D000F5806084423D
:1089500004D021F0020141F0030107E021F00E01F3
:1089600022F4407241F0030142F48072A28023831A
:10897000A4F834B02184238B23F008031B041B0CC0
:1089800043F0080332E0238C664823F010031B04F5
:108990001B0C2384218CA288238B844223F4E6437E
:1089A0004FEA03434FEA134389B292B243F4E043E0
:1089B00008D000F50060844204D021F0200141F08D
:1089C000300107E021F0E00122F4406241F0300183
:1089D00042F48062A2802383A4F838B02184238BE0
:1089E00023F400631B041B0C43F4006323836DE03A
:1089F000238C4C4823F480731B041B0C2384218C90
:108A0000A288A38B844223F073034FEA03434FEA07
:108A1000134389B292B243F0700308D000F50060AE
:108A2000844204D021F4007141F4407107E021F444
:108A3000606122F4405241F4407142F48052A280BD
:108A4000A383A4F83CB02184A38B23F008031B0468
:108A50001B0C43F0080338E0B4F820C0314A2CF472
:108A6000805C4FEA0C4C4FEA1C4CA4F820C0B4F8D0
:108A700020C0A388B4F81C802CF4005C28F4E648DD
:108A80004FEA08484FEA0C4C4FEA18484FEA1C4C92
:108A900094429BB248F4E0484CF4405C03D002F5A9
:108AA0000062944203D123F4804343F48043A380C3
:108AB000A4F81C80A4F840B0A4F820C0A38B23F431
:108AC00000631B041B0C43F40063A383AB7B43B123
:108AD000B4F844306FEA43436FEA53439BB2A4F8BF
:108AE000443023889BB243F0010323802B7B0C2B63
:108AF00010D8DFE803F0070F0F0F090F0F0F0B0F50
:108B00000F0F0D00343404E0383402E03C3400E050
:108B10004034F4515046AAF8049003B0BDE8F08FF9
:108B200014180020002C01407FB52B4B2B4C9A6968
:108B3000206042F001029A61294D03881026ADF8A9
:108B400004302846022301A98DF807308DF806600D
:108B5000FAF78CFA236828465B88ADF804300423C2
:108B60000DEB03018DF80630FAF780FA22680F202A
:108B7000137A03F003018900884003F0FC0303F13A
:108B8000804303F580339D6825EA0000012505FA3E
:108B900001F198609868014399605368114A02A8EE
:108BA0005361029300238DF80C308DF80E508DF830
:108BB0000D6001F093FA23680B4A5B7A59B203F017
:108BC0001F039D404909094B42F821501A68084B80
:108BD0003C3A1A6004B070BD00100240D40300207B
:108BE000000C01400004014000E100E0BC1D002039
:108BF000CC0300200449054B0968002218701A6153
:108C000059611A76704700BFBC1D0020C40B0020BC
:108C100038B5144B144D1A78144C2968A2B1D4F805
:108C20009420024491421BD300201870F9F7E2FC13
:108C30002B68C4F894300E4B1A780AB1013A1A70B6
:108C4000012384F8983038BDD4F89420C83291427A
:108C500006D301201870F9F7CDFC2B68C4F89430C6
:108C600038BD00BFA3190020BC1D0020141800202F
:108C70008E04002037B5254D8DF8073095F89930D2
:108C80008DF8062002AA8DF804008DF805101A440C
:108C900012F8042C443AD2B20F2A30D81C49022BC5
:108CA00031F8124003D814B12046FFF7B1FF95F810
:108CB0009930164A022B0BD9164B1968D2F894300A
:108CC000091B8B4204D2002382F89930124A137098
:108CD00095F89830012B00D0B4B995F89930022B53
:108CE00003D80A4A013382F899300C4B002085F8EA
:108CF0009800187003B0BDE83040F9F77BBC022B38
:108D00004FF0C804D0D9D2E703B030BD141800200A
:108D1000022F0108BC1D00208E040020A319002092
:108D2000F0B5934C934A23689D8AADB2E9B211F035
:108D3000010F36D0198821F400610904090C19804B
:108D4000198889B241F480611980002182F89A1053
:108D5000894908788949B8B192F89B0018B98848C0
:108D60000078FF2810D1012082F89B008548007808
:108D7000022804D1188880B240F400601880097875
:108D800041F00101198216E1097801F0FE01198212
:108D90007B4B1B78FF2B00F00E81FF2382F89A306B
:108DA00009E18F0740D5BFF35F8F76490878C0B2DD
:108DB000012816D1704D2D789DB192F89B5085B148
:108DC000198821F480610904090C1980BFF35F8FB1
:108DD000198B198882F89C0089B241F400711980BE
:108DE0001DE0188BBFF35F8F087802280CD1624812
:108DF000007848B192F89B0030B1198821F4806165
:108E00000904090C1980D0E00978032907D15A49CF
:108E1000097821B192F89B10002940F0C68099880A
:108E200089B241F48061C5E04E0764D5012182F822
:108E30009C105149097800293ED092F89B100029D6
:108E40003AD0504992F89A0009784F4D0229198872
:108E50001FD921F480610904090C19801F8A2E682A
:108E6000C1B2FFB240B23754188880B240F40070EB
:108E700018808B1C82F89A30236828681D8A01317B
:108E800049B2EDB24554998889B241F48061998024
:108E90002CE089B241F4007119801E8A2D68C1B29C
:108EA000F6B240B22E541B8A481C40B2DBB20331EA
:108EB0002B5482F89A1019E092F89B1011B933499B
:108EC000097851B1198889B241F40071198092F87A
:108ED0009A30013382F89A3008E0198889B241F457
:108EE00080711980234B012183F89B1021680B8826
:108EF000D805FCD45FE001F0400101F0FF062148F5
:108F000009B32149B3F810C00F6892F89A105FFABC
:108F10008CFCCDB26E1C49B2F6B207F801C082F8E3
:108F20009A60077876B2F11C8F4205D1998821F4B6
:108F300080610904090C99800378B3423BD1023562
:108F400082F89A5037E0290635D592F89A104DB23A
:108F50006F1C1FD00E4E01313668C9B2755D82F8A4
:108F60009A10EDB21D82007849B2884223D11CE0EC
:108F70009C16002014180020A7160020A41600201C
:108F8000A5160020B0160020AC160020A616002062
:108F9000A8160020144982F89A600978C9B219828B
:108FA0001249097809B9017829B9998821F48061B1
:108FB0000904090C99800E4B92F99A1018780D4B00
:108FC000421C91420FD1002283F89B2093F89C30E1
:108FD00033B12268938823F440731B041B0C9380E5
:108FE000054B00221A70F0BDA5160020A716002020
:108FF000B016002014180020B11600204B8810B5C0
:10900000DC0607D52C4B14791B6853F824402B4BF6
:1090100043F820404B889B0607D5274B54791B68A3
:1090200053F82440254B43F820404B881C070DD5AE
:10903000234B0C781B78B3EB141F07DB1E4BD47843
:109040001B6853F824401D4B43F820404B889B0776
:109050000DD51C4B0C781B78B3EB141F07DC164B9B
:1090600054781B6853F82440144B43F820404B8835
:10907000DC070ED5144B0C781B7804F00F049C42CF
:1090800007DC0D4B14781B6853F824400B4B43F856
:1090900020404B885B070ED50C4B09781B7801F0FC
:1090A0000F01994207DB044B92781B6853F822208A
:1090B000024B43F8202010BD140F00205C06002056
:1090C00013070020110700201007002012070020BE
:1090D000234B70B519684FF47A73B1FBF3F1214B50
:1090E00021481A78214B224D1B78FEF7FBFE214BBD
:1090F00021481968214B2E68B1FBF3F1FEF7F2FE0F
:1091000000241F4BE2B253F8221049B1012303FAA5
:1091100002F2324202D01B48FEF7E4FE0134F0E7CF
:109120002A6892070DD5184A1848127803EB820373
:10913000196AFEF7D7FE164B197A11B11548FEF7DA
:10914000D1FE1548FDF760FCBDE87040134B144894
:109150001A88144B92B2198840F2A453FEF7C2BE8B
:10916000BC1D0020A40500202D4401089200002011
:109170002C0200209C0000206B44010840420F009C
:10918000242F0108D04101089723002089440108B9
:109190004C0400209344010897450108A2160020C2
:1091A00097440108F00400200F4B1A784F2A17D17A
:1091B000598840F2A452914212D11A79BE2A0FD195
:1091C00093F8A1250020EF2A0CD113F8012B504071
:1091D000064A9342F9D1D0F1010038BF0020704710
:1091E00000207047704700BF00F80108A4FD010887
:1091F00030B5002205462E4910014318415CA942B2
:1092000004D00132062AF6D1002030BD294C042DAD
:109210000FCB84E80F00234618D007D8012D0CD0BF
:10922000022D43D1244B1B689B680DE0102D37D0D5
:10923000202D06D0082D39D11CE01F4B1B685B6820
:1092400031E01D4B1B681B6963602CE01B4A1268F0
:1092500012783AB1012A08D0022A0CBF4FF4964284
:10926000002204E04FF4165201E04FF496425A6097
:109270009A601BE0124A1268127A042A16D8DFE8B4
:1092800002F00808030808000E4A6260A260032288
:1092900004E04FF4E1326260A26001225A7305E0FB
:1092A000054B1B68DB68A360204630BD014830BD1C
:1092B000E4240108B4180020F808002094050020D8
:1092C0002C010020A08601002DE9F04FAE4E85B0A4
:1092D0003778032F14D9AD4BAD48B3F90410B0F96A
:1092E00004200029B8BF49426FF063035B1A9A4219
:1092F00004DB01F164039342A8BF134683801FE09F
:10930000012F1DD8A34BA44C1B78013B142B00F25A
:10931000E181DFE813F09100DF01DF0168009F00C9
:10932000DF01DF012F01DF01DF01DF01DF01DF01ED
:10933000BD00DF01DF01DF01DF01DF01A101B801B5
:10934000924B9649B3F806A0914B0968B3F8028096
:10935000B3F80090B3F904B0914C02910025BD42DE
:1093600004F11004CED20FFA8AF003F027FD54F86E
:10937000101C03F077FD03460FFA88F0019303F009
:109380001DFD54F8081C03F06DFD019B01461846B5
:1093900003F060FC03460FFA89F0019303F00EFD21
:1093A00054F80C1C03F05EFD019B0146184603F0C7
:1093B00051FC029A034692F90000019340420BFBD4
:1093C00000F003F0FBFC54F8041C03F04BFD019B80
:1093D0000146184603F03EFC03F00AFF714B23F8E8
:1093E00015000135BBE702210420F9F78DF9684D1E
:1093F0000121AF8878431FFA80F80420F9F784F937
:109400006D8800FB05801FFA80F80420F9F78AF9BF
:109410004044208102210520F9F776F978430121A3
:1094200087B20520F9F770F900FB057087B20520B7
:10943000F9F778F938440BE005200121F9F764F9D0
:10944000534B9D88684385B20520F9F76BF9284492
:1094500060813FE1544B00201D68F9F763F9DFF8A4
:10946000648195F90630B8F902203227534393FB03
:10947000F7F3184420800120F9F754F995F90E30DC
:10948000B8F90020534393FBF7F73844608021E19B
:10949000464B1B7813F0040F454B02D11B689B8889
:1094A0000BE01968394A0B88B2F9062049889A42BC
:1094B00003DB9142B4BF0B461346E381E289394B8B
:1094C000394F1A803B4B1B681D7845B30220F9F7D2
:1094D00029F93A68B2F91030518A984203DB0BB28D
:1094E0009842B8BF0346344909684889C3EB000E67
:1094F000324B0FFA8EFE198A0FFA81FCF44501DA1D
:109500000D4401E001DD4D1B1D8292F91620B3F9D7
:1095100010305343642293FBF2F31844A080284B8D
:109520001B88D9050CD5194B1A88D7F80090E28012
:1095300022819A88184F62815B880325A38101E00C
:10954000134BF1E709EBC50393F90630B7F9068031
:10955000284608FB03F8642398FBF3F8A7F8068075
:10956000F9F7E0F801354044072DF88007F10207CC
:10957000E8D1AFE00D4B1B7813F0040F0C4B23D157
:109580001B689B882CE000BF64230020520200204F
:10959000B017002088050020820000208C050020E4
:1095A000CC0A002066230020741600209623002099
:1095B0007C1600208016002084160020B41800209D
:1095C00046020020980300201968AD4A0B88B2F9C2
:1095D000062049889A4203DB9142B4BF0B461346EA
:1095E000E381E289A74BA84D1A80A84B03201B8872
:1095F0000121DA0503D5F9F787F8A14F02E0F9F761
:1096000083F8A34FB7F80280022100FB08F01FFA8D
:1096100080F90320F9F778F83F88012100FB0790D3
:10962000E8800420F9F770F800FB08F002211FFA27
:1096300080F80420F9F768F800FB078028810320F0
:10964000F9F770F8E3881844E0800420F9F76AF825
:109650002389184420813DE001210420F9F754F8C2
:109660008B4D6F88784387B204202781F9F75AF829
:109670003844208101210520F9F746F82D886843F8
:1096800085B26581E0E6824B0325B3F804909846E5
:1096900028460221F9F738F800FB09F0012187B2CA
:1096A0002846F9F731F8C5F106035B0838F813309E
:1096B00000FB037087B224F815702846F9F732F8DA
:1096C000384424F815000135072DE1D16C4BDA88B8
:1096D0006C4B1A806F4DDFF8E491AB6813F0200FEC
:1096E00033D00020F9F71EF8208080460120F9F7DA
:1096F00019F8694B644FDB79608033B3674B1B68A3
:109700001B7813F0020F664B23D0D9F800C0B3F9D1
:1097100000109CF90E209CF906C0B3F902304A43B0
:10972000CCF1000C03FB0CF3322192FBF1F26FF051
:10973000310C92B293FBFCFC9444E04493FBF1F1B6
:10974000A7F800800A4410447880D9F8001000235C
:1097500019E0D9F80010B3F902C091F90620B3F965
:1097600000300CFB02FC32229CFBF2FCE044A7F828
:10977000008091F90E104B4393FBF2F2E3E7E252C3
:109780000233102B0CD0E05E31F9232001EB83076C
:1097900090427F88F3DB3AB28242A8BF0246EEE7EE
:1097A0003E4B1B681B785B0704D436493478088825
:1097B00001231BE03B4B00241F780423043FFFB22E
:1097C0005FFA87F84FFA88F2D4420BD4364A03F195
:1097D0000109381932F813105FFA89F9C0B2F9F7A4
:1097E0002CFC4B460134042CECD1DEE7A34208D21A
:1097F00031F9132000B28242A8BF104680B2013373
:10980000F4E72A4B4FEA44081A68AB6803F4805522
:109810000395254D03F01009254BB5F90660254D3C
:109820001B782F68244D03F00403DBB2D5F800C089
:1098300002930023434563D0B2F802A004B254451A
:1098400005DD104CC0EB0A0A1D5B55441D53039DFA
:109850000C4C002D34D07D8931F903A0AE42CBBF32
:10986000BCF802509588B2F802B0BCF800B0AA4526
:1098700003DBDA45B4BF55465D46E55239E000BF2B
:1098800052020020662300208200002046020020B1
:10989000B0170020C01D00203002002088160020D4
:1098A00098030020B3090020DE0600207C1600206B
:1098B00096230020841600207816002074160020BD
:1098C00031F903A01588B2F802B0AA4503DBDA45E6
:1098D000B4BF55465D46E55204EB030ABC89A64277
:1098E00007DAB9F1000F01D1148800E09488AAF8D2
:1098F0000040029C14B9044C1C5BCC52023399E723
:1099000005B0BDE8F08F00BFA81900202DE9F04791
:10991000284C137CA46804F0400704F4005C032B7B
:1099200045D80C265E43244D741994F8088010EA3B
:10993000080F03F1010837D0735D4BB1012B07D03D
:10994000032B04D0042B14BF0423032300E00223C1
:109950001A4E1D0106EB050937B916F805A0AAF144
:10996000030ABAF1010F1FD9BCF1000F02D1755DD6
:10997000042D19D04D7B1DB199F80C60354213D0E0
:109980004E68D9F80450AE420ED38E68D9F808500C
:10999000AE4209D81370C2F808905460D16082F8C2
:1099A00010801046BDE8F0875FFA88F3B7E7002023
:1099B000BDE8F087C01D0020380000206C2F010892
:1099C000094B30B59D68094B05F480551868084B64
:1099D0001C6800230DB1828800E0A28805495A5214
:1099E0000233182BF6D130BDC01D002078160020A0
:1099F0007C160020A81900203F4A2DE9F84F9168F5
:109A000040F201130B4040F201118B4293460AD100
:109A10003A4B9A7C93F81390DA74B9EB020918BFA9
:109A20004FF0010901E04FF001094FF00008344BFD
:109A30005FFA88F41B78A3425CD9324B324E1B6824
:109A4000324F23B93B685B8926F814304FE03A68FF
:109A5000072C94BF12F804A0A24629485146984703
:109A6000DBF808300546DB0509D5B9F1000F06D053
:109A7000274B50461B6829461B68DB699847A5F2AF
:109A8000EE2240F2DC5392B29A4288BF3B68DBF888
:109A9000082088BF5D8942F2010313402BB31D4BA0
:109AA0001978164B01F0030202EB840293F874005C
:109AB00003EB420295821A4620B9032915D90121E8
:109AC00083F8741002EBC403D98A9D8A02EB440226
:109AD0000D44198B5B8B0D441D44ADB2A2F876503A
:109AE00004232DB295FBF3F5ADB226F8145008F11E
:109AF00001089CE7BDE8F88FC01D0020B4180020C5
:109B0000A70B0020B00B0020DE0600202C01002057
:109B100020020020FC10002013B50446006800F06D
:109B200007FB236801A81A8892B242F001021A804A
:109B3000637B8DF8043001238DF805308DF80630F5
:109B40008DF80730FCF776FD02B010BD024B0348DC
:109B50001968034AFEF7C6B9B4000020254501087C
:109B6000AC3E010810B50748FCF74EFF0024064B39
:109B70000648E218E15852680C34FEF7B3F9E42CB9
:109B8000F5D110BD4F450108EC2F010865450108CE
:109B90002DE9F041002407462546114B3946E65889
:109BA00004EB0308304606F029F958B10D48314658
:109BB000FEF798F940460021FEF716FC0A48FEF72A
:109BC00091F90135143440F664239C42E5D125B95E
:109BD0000648BDE8F041FCF717BFBDE8F08100BFC3
:109BE0005432010803460108974501086D450108F4
:109BF0002DE9F74F044606F0C5F8054620B10128C7
:109C000019D123782A2B16D15248FCF7FDFE0024E7
:109C1000514B5248E618E158FEF764F930462946A0
:109C2000FEF7E2FB4E48FCF7EFFE143440F66423E7
:109C30009C42EDD18AE020463D2106F096F80028AE
:109C40007FD0034613F8012C202A01D1013BF9E70C
:109C5000451C2846C4EB030A06F0E9F8834628466B
:109C6000F8F712FF0026054614237343DFF8E89047
:109C700053F8097003EB0908384606F083F80346E9
:109C80001A4620463946019306F084F8019B0028C5
:109C90004ED15FFA8AF29A424AD1D8F80C0003F00A
:109CA0008DF80146284603F08FFA00283ED0D8F8F8
:109CB000100003F083F80146284603F07BFA0028E1
:109CC00034D098F804309C064FF0140303FB06963A
:109CD000327958BF5D4610062946B36806D521483B
:109CE0004FF49A7490F8A00504FB003302F03F0291
:109CF000042A0BD004D8013A012A0CD819700AE0C2
:109D0000102A05D0202A05D0082A04D1198002E0A3
:109D1000196000E01D6039461348FEF7E3F830464D
:109D2000002103B0BDE8F04FFEF75EBB0F4803E033
:109D30000136852E98D10E4803B0BDE8F04FFCF7F0
:109D400063BE204603B0BDE8F04F21E703B0BDE895
:109D5000F08F00BF85450108543201080346010811
:109D600097450108C01D00209A450108A545010836
:109D70006D4501082DE9F04F624C23686249581C7B
:109D80000A78894602F0FF0C0AB10346F6E7277A03
:109D9000667AA57AE1682360E0461FFA88F213B27A
:109DA0001F2B00F39380594901EB8300C278807820
:109DB00031F82310C0F1FF0080B2002861D0C0F15B
:109DC000FF0050433C23B1FBF3FA0012BAF1050F38
:109DD0005AD8DFE80AF0030B1A283846161A4E4301
:109DE000C5B2B6FBF3F62E44F6B248E0B1FBF3F78A
:109DF00003FB1717BFB2C5B2C7F13C07101A4743A0
:109E0000B7FBF3F72F44164629E0B1FBF3F503FB4C
:109E10001515C7B2ADB2101A4543B5FBF3F53D4475
:109E2000EDB2164630E0B1FBF3F603FB1616B6B200
:109E3000C7B2C6F13C06101A4643B6FBF3F63E44E1
:109E40001546F6B220E0B1FBF3F703FB1717C6B2D5
:109E5000BFB2101A4743B7FBF3F737441546FFB2BA
:109E600012E0B1FBF3F503FB1515ADB2C6B2C5F1B7
:109E70003C05101A4543B5FBF3F53544EDB21746E2
:109E800002E01546164617464FEA072A4AEA064AEE
:109E90004AEA050A1723012199400CF1170211EA39
:109EA0000A0FC3EB02021A490CBF0920112092B21B
:109EB00013F1FF338854EED20CF1180C08F10108AD
:109EC0001FFA8CFC1FFA88F8124966E7012389F80B
:109ED0000030114BE28040F22A3227726672A5727E
:109EE000E160A4F804C05A600C4A002191841188F2
:109EF00089B241F0010111801A6842F001021A6032
:109F0000BDE8F08F441900208E2300205C0600205D
:109F1000E80B00204C1900206C00024000040040B7
:109F2000826A8169436B1144D960416A914203D9C5
:109F30008A1A5A60816204E001698A1A5A60002212
:109F40008262002280F844201A6842F001021A60FE
:109F50007047F8B501210446FEF752FC01283C4F3A
:109F600001D0002616E04FF6FE732382A68D002551
:109F7000B6B22046795DF9F721F8364B142202FB80
:109F80000030C36813B1007C314698470235082D74
:109F9000EFD1E6E7BD5D95B920460221FEF730FC22
:109FA000012850D14FF6FD73238229462046F9F748
:109FB00005F8284B142202FB0030A18E3EE0042D50
:109FC00012D120462946FEF71BFC01283BD14FF653
:109FD000FB73238229462046F8F7F0FF1D4B14221D
:109FE00002FB0030218F29E0082D12D1204629469E
:109FF000FEF706FC012826D14FF6F7732382294687
:10A000002046F8F7DBFF134B142202FB0030A18F30
:10A0100014E00C2D17D120461021FEF7F1FB01288A
:10A0200011D14FF6EF73238229462046F8F7C6FF79
:10A03000084B142202FB0030B4F84010836889B248
:10A040000BB1007C98470236082EA3D1F8BD00BFA3
:10A05000AC2F0108B80700202DE9F041067B04462B
:10A060000F460068314690461D46F8F7A7FF0F28B7
:10A0700008D8194B142202FB0030C0F80880C560D4
:10A0800006710774237B22680C2B1CD8DFE803F0D1
:10A09000071B1B1B0C1B1B1B111B1B1B1600938977
:10A0A0009BB243F002030DE093899BB243F004039B
:10A0B00008E093899BB243F0080303E093899BB2C5
:10A0C00043F01003938125B193899BB243F00103C0
:10A0D0009381BDE8F08100BFB8070020134B0268F0
:10A0E00010B51C68D1430C401C605C68214059606D
:10A0F00019680A431A6002689C68D1430C409C604E
:10A10000DC682140D9604179102906D19968114352
:10A110009960D9680A43DA6010BD01F1804303F504
:10A12000823319680A431A6010BD00BF0004014061
:10A13000254B10B55343254A254C12680139B2FB13
:10A14000F3F20388013AA04289B292B29BB212D0D4
:10A1500004F50064A0420ED0B0F1804F0BD0A4F5FE
:10A160009834A04207D004F58064A04203D004F5DF
:10A170008064A04202D123F070039BB2154CA04230
:10A1800006D004F58064A0421CBF23F440739BB248
:10A1900003800F4B8185984202850FD003F5006341
:10A1A00098420BD003F54063984207D003F58063D3
:10A1B000984203D003F58063984201D100230386BF
:10A1C0000123838210BD00BF40420F009C0000208D
:10A1D000002C014000100040284BF0B51D68002203
:10A1E0002748165C1418AB19597801F0040101F0E6
:10A1F000FF0371B10132102AF2D10020F0BD1BB172
:10A2000003EB83035B00DBB210F8012B303A1344FD
:10A21000DBB2221A022AF2DC002184420AD919B1E7
:10A2200001EB81014900C9B210F8012B303A114409
:10A23000C9B2F2E72E2E14D1601C00220424067845
:10A2400002EB8202AF197F7852007F0792B203D5EA
:10A25000303A3244013092B2013C14F0FF04EED1A6
:10A2600000E00022074806244143642000FB02125C
:10A270000548B2FBF4F200FB0320F0BDB80000205B
:10A280003B0F002040420F008096980030B500221E
:10A2900013460D495C5C9CB12E2C04D1013378B17E
:10A2A0001C1800250D550A246243C95CA1F1300435
:10A2B000092C9CBF303A52180E2B03D80133E8E723
:10A2C000104630BD002030BD3B0F00200EB40FB54E
:10A2D00005AB53F8042B0190064901A80393FDF741
:10A2E0003BFD019B00221A7004B05DF804EB03B043
:10A2F000704700BF6D2100082DE9F0438DB0054681
:10A3000005F040FDC0B2002858D104467F4B002123
:10A310001E68142207A805F0F4FCA500002303A979
:10A3200005A80393059377190B7183801A46DFF80C
:10A33000F8E1B7F802C03EF8138018EA0C0F0CD011
:10A340000EF10A0E0DF1300813F80EE002F1010CC7
:10A35000424402F824EC5FFA8CF20133052BE6D17B
:10A3600000231A46DFF8C4E1B7F802C013F80E80E4
:10A3700018EA0C0F0CD00EF1060E0DF1300813F890
:10A380000EE002F1010C424402F81CEC5FFA8CF280
:10A390000133062BE6D1735D8DE803001A0907A887
:10A3A0005B4903F00F03FFF791FF2146594807AAC5
:10A3B0000134FDF797FD202CA8D1A4E0284605F034
:10A3C00036FD1F28044600F3928028462021E4B27F
:10A3D00005F0CBFC1F2C01D94F4889E04B4B471CA3
:10A3E0001B68002103EB84042046042205F089FC4D
:10A3F00000254A4B07AE304600210A2215F803908B
:10A400005FFA85F805F07DFC0023FA5CF91832B19B
:10A410000A2B04D04A4502D0F2540133F5E74A45ED
:10A4200001F1010768D1B8F1020F0DD0B8F1030FA7
:10A430000CD0B8F1010F0BD0304605F0F8FC2378B2
:10A44000C0B243EA00100AE0002219E0002226E030
:10A45000304605F0ECFC237800F00F001843207024
:10A4600039E00133062B0AD02D4800F11D069E5D10
:10A470008E42F6D10344D97D63880B436380013259
:10A480000CA9D3B20B4413F8141C21B30023EBE73F
:10A49000412B1ED0542B08BF04230ED00132D3B25F
:10A4A0000DF13008434413F8143CA3B1492B01D1FA
:10A4B000002302E0572B08D10123194901EB430384
:10A4C000198963880B436380E8E7462BE0D10223B8
:10A4D000F3E70323F1E70135042D8AD10124F8F7CE
:10A4E00047FCF8F781FCF8F75BFC64B974E70D48AA
:10A4F0002021FDF7F7FC06E020460021042205F0AC
:10A5000000FC0024EBE70DB0BDE8F0835806002006
:10A51000C5450108D145010818430108CF2F01089E
:10A52000AC2F0108DD450108B42F0108C32F010835
:10A5300070B5064600240B4BE5182A7916420AD05E
:10A54000E1580948FDF7CEFC28460021FDF74CFFF5
:10A550000648FCF759FA143440F664239C42EAD1C9
:10A5600070BD00BF54320108FF450108974501083E
:10A5700060492DE9F04F604B0A68B3F90640B2F824
:10A58000583085B09C420FDBB4F5FA6F92F85660F4
:10A5900007DAE11A4E43A3F5FA6396FBF3F6643645
:10A5A00003E0C6F1640600E06426544B0020B3F8D3
:10A5B00018B193F9EC3015465B429BB20393014608
:10A5C0004D4B40F2E637C35E0293CBEB030303F23D
:10A5D000F31EBE4503D8002BB8BF5B4201E04FF429
:10A5E000FA730229DFF820C12ED092F8D47027B177
:10A5F000BB42CCBFC7EB030300236427DFF8049101
:10A6000093FBF7FE6FF0630A39F81E800AFB0E3ADF
:10A610000EF1010E39F91E900FFA88FECEEB090EED
:10A620000EFB0AFE9EFBF7FEC6442CF800E092F8F3
:10A6300054E003FB0EFE324B9EFBF3F33B449BB214
:10A64000734393FBF7F717E092F8D57027B1BB423D
:10A65000CCBFC7EB03030023DDF80CE003FB0EF7D0
:10A66000ACF8047092F85570002BB8BF5B427B4386
:10A67000234F93FBF7F76437531893F804C0DFF8C0
:10A680008CE007FB0CFC64239CFBF3FC01F80EC080
:10A6900095F80E800EF1030C07FB08F898FBF3F811
:10A6A00001F80C8095F818C00EF1060E07FB0CF7A8
:10A6B00097FBF3F301F80E30029BDFF84CE05B45AB
:10A6C00004DA3EF800305B422EF8003001310329F5
:10A6D00000F1020005F101057FF472AF074FB7F8F2
:10A6E0001A319C4214DBB4F5FA6FA8BF4FF4FA6438
:10A6F0000FE000BFDC030020DE060020C01D0020AC
:10A700000CFEFFFF5819002052020020661900209D
:10A710001C46E41A4FF47A725443C3F5FA63B4FB4F
:10A72000F3F36420A44C93FBF0F204EB42016FF0CE
:10A73000630606FB0233098B04EB4202B2F91A608E
:10A740000AB2B21A534393FBF0F09C4B01441A88AF
:10A750009B4D5606AEF806103ED59A4B1888238EB0
:10A76000C01A00B201F088FF91A3D3E9002301F0E1
:10A77000E9FF02F019FA064605F0F2FC8046304681
:10A7800005F062FD0646B5F9020002F017FB8146AE
:10A79000B5F9000002F012FB4146824602F062FB6E
:10A7A00031468346484602F05DFB0146584602F0BA
:10A7B0004FFA02F01DFD41462880484602F052FB48
:10A7C00031468046504602F04DFB0146404602F0BD
:10A7D00041FA02F00DFD6880BA6840F602031340AA
:10A7E000002B53D0784B06211D88636B1D4494F8D1
:10A7F000383065630133DBB2B3FBF1F084F83830F5
:10A8000001FB103313F0FF0F40D1900706D5FCF782
:10A8100005F8FBF7EDFF684B83F83900BB681905B5
:10A8200032D56A4BE16B5A7B694B33F8120008232F
:10A8300091FBF3F280B28A1A0244E26392FBF3F2D4
:10A8400092B240F6E4435A43624B40F6FF71B2FBCA
:10A85000F1F219684FF47A73C8888988121A5A433A
:10A8600092FBF1F255435C4995FBF3F30A60D4E99E
:10A870001001C01841EBE371C4E910010023574AED
:10A8800002F0FCFC564B186000236363554E4A4BA4
:10A89000327B94F8398002B1012283F84820BB68EA
:10A8A000514D13F4807F2CD0DFF850912878D9F8DF
:10A8B0000030C0F380001B685B68984760B10123DB
:10A8C00084F84930D9F800301B68DB68984718B124
:10A8D000394B022283F84920D9F800301B689B6865
:10A8E000984728B12B785A075CBF022384F8493077
:10A8F000D9F800301B689B69984710B1002384F891
:10A9000049303A4B1A6893060DD5737A13B9354B13
:10A910009B7A2BB1364B1B78980701D4012300E0BA
:10A92000002384F84A3094F84920234B022A02D1AC
:10A930004C204E211EE0012A06D153204D214C22ED
:10A940000B46FEF797F92CE093F84A20012A03D131
:10A95000532001464E2206E093F84820012A04D1F4
:10A960005320014602464D23EBE7B8F1000F04D017
:10A9700053204D210A464423E3E710490A88110673
:10A9800003D553204D210246DAE71A4A12781AB14C
:10A990003220FEF73DF904E0404683F84B80F7F79C
:10A9A00029FE2B785A072BD5134B08225A6180E0D9
:10A9B000399D52A246DF913F5819002046020020DF
:10A9C00052020020D4040020F004002028070020B8
:10A9D00038070020280F0020A8050020407E050031
:10A9E000AC05002030020020962300202C0200201D
:10A9F000720200208E040020000C0140A00B0020F9
:10AA000032781AB9994A43F001031370984A1368CF
:10AA100013F0020302D0974A1288A2B9964A12880C
:10AA200002B12BB9954B1B88003318BF012300E0FE
:10AA3000012343B1924BDA6882F00802DA602B7886
:10AA400023F001032B708F4B1B78180703D42B784E
:10AA500023F001032B70337D1BB12B7823F001030E
:10AA60002B702B78884A13F0010F05D00023E36484
:10AA7000834B082119610BE0E16C136841B98349EC
:10AA800003F5F42303F59073CB647D4B08215961E2
:10AA9000E36C12686BB1D21A002A0ADB784A03F51C
:10AAA000F423D16803F5907381F00801D160774AEF
:10AAB000D364774B1B780BB100F022FD754B1B78EC
:10AAC00013B1FCF743FE16E3DFF8F48198F84A303F
:10AAD000012B05D0704B08F14C089845F6D10AE3DC
:10AAE0006E4BD8F800206E49C3F800800A60994682
:10AAF0006B4E3068F7F79AFD0028EBD03068F7F717
:10AB000090FDD9F8003093F84820DAB9B0F124016B
:10AB10004A424A4183F84820002AE9D12B785B0752
:10AB2000E6D4232802D1FCF711FEE1E75D4B1B6858
:10AB30001B7D8342DCD15C4A5C4B1A605C4A5D4BF6
:10AB4000DA60D5E7012A04D14D2814BF0022022281
:10AB5000CEE2022A04D13C2814BF00220322C7E21D
:10AB6000032A0AD140284FF0000200F2C1821A7174
:10AB7000DA71587198710422BAE2042A06D19A79DE
:10AB800083F84900504098710522B1E2052AAFD1FF
:10AB900059791A799142997906D941409971511C94
:10ABA000197113441872A3E7814240F09E8293F812
:10ABB000490000F093FE002840F09282D9F800305E
:10ABC00093F84930C83B322B00F2B482DFE813F02F
:10ABD0007A002C02920033004D0102020A02780131
:10ABE000F701500235004800B101E901A801B202A5
:10ABF000B202B202B202B202B202B202B202B202B5
:10AC0000B202B202B202B202B202B202B202B202A4
:10AC1000B202B202B202B202B202B202B2028500C3
:10AC2000B202B202B202B202B202B202B202B20284
:10AC3000B202B20228020026E8E02B7803F00403F7
:10AC400003F0FF06002B40F04882FBF72BFE0228A2
:10AC500087F8A00540F2B981174B83F8A065B4E1ED
:10AC6000FBF72AFE154B188037E200BF9623002021
:10AC70002C02002084230020600400208C2300206C
:10AC8000000C01407202002080230020581900208F
:10AC90009005002090230020AC0900203C060020F5
:10ACA00040060020F8080020EFBEADDEF04F002087
:10ACB0000400FA0500ED00E0C01D00206E05002034
:10ACC000140900200026FBF7F7FDCA4B9853023603
:10ACD000102EF8D10122C84BC8E1C84ED6F800A00A
:10ACE000FBF7EAFDAAF85E003668FBF7E5FDA6F87B
:10ACF0005C00F2E1C14E33681B78022B69D100265B
:10AD0000DFF8F8A2DAF800B0FBF7CCFD06F1080294
:10AD10000BEB820B02F04EF8B94902F057F9CBF871
:10AD20000400DAF800B0FBF7BDFD06F10A020BEBF8
:10AD3000820B02F03FF8B34902F048F9CBF8080063
:10AD4000DAF800B0FBF7AEFD06F10E020BEB820B5A
:10AD500002F030F8AC4902F039F90136032ECBF895
:10AD60000400CDD1072E1BD1DFF890B2DBF8002014
:10AD70000092FBF797FD02F01DF8A14902F026F9B9
:10AD8000009ADBF800B09064FBF78CFD02F012F83B
:10AD90009B4902F01BF9CBF84C00FBF783FD14E054
:10ADA000DAF800B0FBF77EFD0BEB06031871DAF85A
:10ADB00000B0FBF777FD0BEB06039873DAF800B0F1
:10ADC000FBF770FD0BEB0603187601360A2EC9D18E
:10ADD00083E14FF0000AD6F800B0FBF763FD0BEB00
:10ADE0000A031871D6F800B0FBF75CFD0BEB0A0301
:10ADF0009873D6F800B0FBF755FD0BEB0A030AF188
:10AE0000010ABAF10A0F1876E5D166E17F4B1A788C
:10AE10009A4696420FD2794BD3F800A07C4B16F895
:10AE200003B0FBF749FD0BF12003C0F30B004AF818
:10AE300023000136EAE700269AF800309E4280F0AF
:10AE40004C81734BF25C6D4B01361B6803EB820B3C
:10AE5000DBF880300193FBF72FFD019BC0F30B0063
:10AE600043EA0043CBF88030E6E764490E68FBF71D
:10AE700019FD624A86F850001668FBF713FD5F4B18
:10AE800086F851001E68FBF70DFD5C4986F85400FA
:10AE90000E68FBF707FD594A86F855001668FBF760
:10AEA00001FD564B86F856001E68FBF7FBFC534924
:10AEB00086F852000E68FBF7F5FC86F853000CE1AB
:10AEC000FBF7FAFCFBF7F8FCA7F8D000FBF7F4FC63
:10AED000A7F8D200FBF7F0FC484AA7F8D4001668A0
:10AEE000FBF7EAFCA6F81E01FBF7E6FCFBF7EEFC1D
:10AEF000424B1E68FBF7E0FC00EB80004000A6F828
:10AF00005A00FBF7CFFC87F80401FBF7CBFC87F86E
:10AF10000601FBF7C7FC87F80501FBF7C3FCDCE083
:10AF20000026FBF7C9FC3B4B98530236102EF8D194
:10AF3000D3E00026DFF8C4A0DAF800200092FBF787
:10AF4000BBFC009A06F11B034FEAC30B5A449080E6
:10AF5000DAF800200092FBF7AFFC009A5A44D08048
:10AF6000FBF7AAFC072804D8DAF8002002EB0B0351
:10AF7000D872A0F57A739BB2B3F57A7F05D8DAF868
:10AF8000003003EBC603A3F8E000DAF800A0FBF7FB
:10AF900089FC0AEBC6030136082E83F8E200C9D10A
:10AFA0009BE00026154BD3F800A0FBF77BFC0AEBD7
:10AFB000C6030136082E83F8E300F3D18DE02B7829
:10AFC0005E0700F18A80FCF7C1FCFAF72EF9F9F769
:10AFD0009BFE82E02B7858077FD40F4B4FF4C8724A
:10AFE0001A807AE02B78590777D40C4B1A7842F004
:10AFF00004023BE0DE0600201C020020DC030020EF
:10B00000000020410000C84200007A4411090020DD
:10B01000FC080020A8190020600400207202002013
:10B020002B785A07D1D585E0FBF73CFC454B1A78C5
:10B0300010B142F0020201E022F002021A70FBF7A6
:10B0400031FC414B414E1870FBF740FC3060FBF780
:10B050003DFC7060FBF730FC3D4B1880FBF72CFC8F
:10B060003C4B18803C4B1A7842F002021A7034E0D4
:10B07000FBF718FC0090FBF729FC0190FBF726FC7E
:10B080008246FBF723FC0646FBF716FCFBF714FC95
:10B09000FBF708FC9DE80C0082B93049A3660B88D9
:10B0A000C4F86CA023F010030B80264B1A7842F0F2
:10B0B00001021A708EB12A4B1E600EE0102A0CD1CC
:10B0C0002367C4F874A00EB1254B1E6025480223E7
:10B0D000011D84F87830FCF7EDFD0020FBF72EFC15
:10B0E000D9F800309879FBF7FAFBD9F80030002244
:10B0F00083F84820FCE41C4A13689B0614D51B4BBC
:10B10000E26F1B689A1A002A0EDB0F4A1278042A93
:10B110000AD9174A03F5123303F5F873D367154BB1
:10B12000DA6882F01002DA60134B9B683BB1134877
:10B13000984704E001200021FBF7E2FBD0E705B0CF
:10B14000BDE8F08F72020020E8050020B005002065
:10B150001A060020160600209D230020460200202B
:10B1600048020020C81900202C0200208023002063
:10B1700058190020000C0140E0030020A205002027
:10B180002DE9F0418CB01E469DF848308846012BD1
:10B19000174608D19C4B984240F02D81042203F5BC
:10B1A00048431A615CE0994B984255D19848994BB5
:10B1B00087600360984BB507436103F58073836133
:10B1C0004FF48073C3600361904B036503F1040384
:10B1D0008364C36403F5484303F154030363A3F199
:10B1E0001403D3F8D42F436342F48042C3F8D42F1E
:10B1F000D3F8D02F42F00102C3F8D02F4FF0020352
:10B200008DF803304FF40073ADF800304FF01803A1
:10B210008DF8023003D581486946F7F727FF4FF4D0
:10B220008063ADF80030F4074FF048038DF802302A
:10B2300003D57A486946F7F719FF0E238DF80430D5
:10B2400001A801238DF805308DF806308DF8073000
:10B250006F4CFBF7EFF94EE06B4B984240F0CF801C
:10B260006F486C4B876003608023C3604023036199
:10B270006C4B436180338361634B036504338364A8
:10B28000C36403F5E53303F5FE73DA69B00742F4EE
:10B290000032DA615A6942F001025A614FF002034A
:10B2A0008DF803304FF00403ADF800304FF0180371
:10B2B0008DF8023003D559486946F7F7D7FE0823C1
:10B2C000ADF80030F1074FF048038DF8023003D598
:10B2D00052486946F7F7CAFE26238DF80430022249
:10B2E000012301A88DF805308DF806208DF8073070
:10B2F000FBF7A0F94A4C0025012384F8443025626D
:10B30000E561A5626562C4F82C806671A760A571CD
:10B310002046FDF70FFAE36CF20701934FF48053D8
:10B320000A934FF0800302950395049505950795C0
:10B33000089509950B95069324D5206BD0B1E36849
:10B3400004932023099363690293FBF7FCF801A996
:10B35000206BFBF7DAF8236B1A6842F001021A60DF
:10B36000226D918A89B241F0400191825B689BB263
:10B37000236407E0236D4FF6DF721A80DA6842F02B
:10B380002002DA60A36C002501934FF480530A93E6
:10B3900080230693B30702950395049505950795B9
:10B3A000089509950B951ED5606BB8B12369049378
:10B3B00010230393FBF7C7F8606B01A9FBF7A5F80F
:10B3C000636B1A6842F002021A605D605D60236D73
:10B3D0009A8A92B242F080029A8204E0236DDA687F
:10B3E00042F08002DA60236D20469A8992B242F4DC
:10B3F00000529A8104E0054B98423FF4D7AE0020FA
:10B400000CB0BDE8F08100BF0044004000380140AE
:10B41000641D0020D42F0108D81900200008014025
:10B42000101D0020D81B00202DE9F04F87B0984652
:10B4300082460F4616469DF84040FDF7D9FE0DF1B5
:10B44000080E0546034600F1100C1868596872464C
:10B4500003C2083363459646F7D12B7B0BB903969D
:10B460000496504602A9F9F700FC054640B143682E
:10B47000586830B1504602A92A46FEF747FAF4E769
:10B4800034E0AB6895F800B093F80090B9F1040F80
:10B490002CD8DFE809F003062B0F110000941548A3
:10B4A00001E015480094394632464346FFF768FEEE
:10B4B00004460BE0002000E00120394623463246D6
:10B4C000F9F710FE41460446F7F79CF86CB10B4BB8
:10B4D00084F8049003EB8B03C3F8C0426B682046EA
:10B4E0005C60FBF7C9FA80F809A0204607B0BDE808
:10B4F000F08F00BF0038014000440040D819002000
:10B500002DE9F743F7F708FC814E0546337883426F
:10B5100000F0FB807F4C23681B78002800F0A78098
:10B520006BBB0420FBF77EFA7B4F01463860DFF8E7
:10B53000F48198B143794FF4165188F8D03283687A
:10B54000C8F8D432F7F768F838680221F7F75AF8E4
:10B550003868FBF791FA0423437210E06F4B042024
:10B560001B684FF416529B7800930223FFF75CFF91
:10B570004379386088F8D0328368C8F8D4322368B9
:10B5800093F80090B9F1010F2AD10420FBF74AFA91
:10B59000634F01463860DFF88C8198B143794FF4EE
:10B5A000964188F8D8328368C8F8DC32F7F734F867
:10B5B00038684946F7F726F83868FBF75DFA042340
:10B5C00043720DE000904B4604204FF49642FFF783
:10B5D0002BFF4379386088F8D8328368C8F8DC32AA
:10B5E00023681F78022F40F081800420FBF71AFAAD
:10B5F0004C4C0146C4F8E002A8B143794FF496419F
:10B6000084F8E4328368C4F8E832F7F705F8D4F830
:10B61000E0023946F6F7F6FFD4F8E002FBF72CFA21
:10B62000042343720EE000903B4604204FF4964200
:10B63000FFF7FAFE4379C4F8E00284F8E432836845
:10B64000C4F8E832D4F8E072374C94F84A20022A61
:10B650004ED1364B1C60002C48D0204600214C2295
:10B6600004F04FFB0223276084F84A303EE083B9A0
:10B67000294FDFF8B080386898F8D012F6F7C2FF8B
:10B680003868D8F8D412F6F7C7FF3868FBF7F4F932
:10B69000457223681B78012B11D1214FDFF884807C
:10B6A000386898F8D812F6F7ADFF3868D8F8DC1289
:10B6B000F6F7B2FF3868FBF7DFF90023437223681F
:10B6C0001B78022B12D1174CD4F8E00294F8E41244
:10B6D000F6F798FFD4F8E002D4F8E812F6F79CFFEA
:10B6E000D4F8E002FBF7C8F90023437235700CE090
:10B6F00094F89630022B01D14C34AAE7002AA8D046
:10B700004C34002B18BF0024A3E703B0BDE8F0833E
:10B710009105002094050020980500201C0F0020B2
:10B7200024060020D8190020140900203806002023
:10B73000F7B5284B1B78042B45D12020FBF772F975
:10B74000044670B12046F6F762FF18B90A20FBF7ED
:10B75000ACFAF7E7204B20461B681969F6F75CFF47
:10B760000AE01D4B21461B6800901A692020032324
:10B77000FFF75AFE044630B3184B08221A61102214
:10B780001A61174D2868F6F751FF50B1134E08277C
:10B7900077612868F6F745FF01462046F6F758FF1F
:10B7A00037612046F6F742FF0028EAD00B4E1027FB
:10B7B000776120462D68F6F734FF01462846F6F7F4
:10B7C00047FF3761DDE7074803B0BDE8F040FBF70E
:10B7D0001BB900BFC40B0020C00B0020000C0140AF
:10B7E000E40B0020094601082DE9F047054604F066
:10B7F000C9FA2E4B0446D3F808809A4690B92C48D3
:10B80000FBF702F92B4B53F8241049B10123A34055
:10B8100013EA080F02D02848FCF764FB0134F1E773
:10B82000264821E028462649224604F0B3FA58B9B2
:10B830002448FBF7E9F8244C54F8041F0029EFD002
:10B840001D48FCF74FFBF7E72B7800262D2B03BF95
:10B85000013504F1FF344FF001094FF00009154B99
:10B8600053F8267027B91948BDE8F047FBF7CCB864
:10B8700028463946224604F08DFAA8B90120B04086
:10B88000B9F1000F03D0F7F71DFA114804E040EAC0
:10B890000800CAF808000F48FBF7B6F839460E480A
:10B8A000BDE8F047FCF71EBB0136D8E7C01D0020FD
:10B8B00001480108D0300108D0410108974501082E
:10B8C0008247010814480108CC30010829480108C2
:10B8D000404801084A4801086845010870282DE9D8
:10B8E000F84300F0898200F2D380692800F01582C5
:10B8F00000F2A480662800F0658100F2948064283C
:10B9000000F03581652840F03B840B20FBF716F8EA
:10B91000CF4BB3F90000FBF714F8CE4B188800B2F8
:10B92000FBF70FF8CC4B1B68C3F3C000C3F38002D6
:10B93000800040EA4200C3F340021043C3F34012C8
:10B9400040EAC20003F010031843FAF7FAFFC34BB2
:10B950001A88C34B02F0080493F8069093F8078006
:10B9600093F808C044EA891444EAC81444EA0C2451
:10B9700093F80CC012F0010F44EA0C3493F80DC098
:10B980000CBF4FF0000E4FF0020E44EA4C3493F817
:10B990000FC012F0020F44EACC3493F810C00CBF71
:10B9A0000027042744EA0C4493F811C012F0040F56
:10B9B00044EA4C4493F812C00CBF0026102644EA17
:10B9C0008C4493F813C01B7D44EACC4444EA0354EE
:10B9D000A44B12F0400F1B780CBF00252025C3F3A9
:10B9E00080031C4344EA0E043C4312F0100F44EA67
:10B9F00006040CBF00204FF400702C4312F0200FFF
:10BA00000CBF00214FF480610443974B12F4807FF8
:10BA100044EA01040CBF00224FF4006200201978B0
:10BA200014430346B9E0672800F00581682840F018
:10BA3000A7831020FAF782FF002466E16C2800F04B
:10BA40007F8117D86A2800F02E836B2840F09883F6
:10BA50000520FAF773FF854BB3F90000FAF771FF81
:10BA6000834BB3F90000FAF76CFF824B187800F0B3
:10BA700001000AE36E2800F0718100F29781062030
:10BA8000FAF75CFF7C4B1868FAF780FF7B4B29E3E1
:10BA9000772800F0C08245D8732800F0F98239D8A1
:10BAA000712800F03B82722840F06A83744C1620A3
:10BAB000FAF744FF0020FAF744FFB4F9D000FAF790
:10BAC00040FF704DB4F9D200FAF73BFFB4F9D4004F
:10BAD000FAF737FF2B68B3F91E01FAF732FF00209F
:10BAE000FAF72FFF0020FAF751FF2B68B3F95A003D
:10BAF0000A2390FBF3F0FAF724FF94F80401FAF715
:10BB0000EEFE94F80601FAF7EAFE94F80501FAF75A
:10BB1000E6FEB9E2752800F0F58100F29782002771
:10BB2000012450E2A02800F019830AD8782800F0F8
:10BB3000BD807B2840F024830820FAF7FFFE002414
:10BB4000D7E0F02800F0FB82FE2800F0EC82A42869
:10BB500040F016834C4D0024A8782E46800001301A
:10BB6000C0B2FAF7EBFEA878FAF7B9FEC4E20720F4
:10BB7000434CFAF7E3FEE620FAF7B1FE6079FAF7F4
:10BB8000AEFE0020FAF7ABFE94F824013F4B404A8A
:10BB900000280CBF10461846EDE28B420CD23D4AFD
:10BBA0009D5C012202FA05F5254218BF9A4003F177
:10BBB000010318BF1043F0E7FAF7E8FE304B93F8A3
:10BBC000A00562E21220FAF7B9FE334B334C1B8812
:10BBD000B3F5806F22D90025605F082390FBF3F056
:10BBE0000235FAF7AEFE062DF6D12D4CB4F9000061
:10BBF000FAF7A7FEB4F90200FAF7A3FEB4F90400BD
:10BC0000284CFAF79EFEB4F90000FAF79AFEB4F950
:10BC10000200FAF796FEB4F904009CE2B4F90000C1
:10BC2000FAF78FFEB4F90200FAF78BFEB4F90400BC
:10BC3000FAF787FED9E71020FAF780FE00241A4BA6
:10BC4000185D0134FAF74BFE102CF8D195E200BFD5
:10BC5000F0040020A21600202C0200204602002042
:10BC60003002002096230020110900201806002031
:10BC70001C0600209D2300204C020020B803002059
:10BC8000C01D0020DC030020C41C00203C000080FC
:10BC900034000080FC08002000000020A8040020E0
:10BCA000E80400206C020020820000203820FAF70F
:10BCB00045FE0025AF4E05F11B043368E400234424
:10BCC000B3F90400FAF73DFE336801352344B3F9B4
:10BCD0000600FAF736FE33682344B3F90800FAF792
:10BCE00030FE33681C44A07AFAF7F9FD082DE1D143
:10BCF00043E2A04B1B6803EBC40393F8E300013459
:10BD0000FAF7EDFD082CF4D137E29B4B185D0134B6
:10BD1000FAF7E5FD102CF8D12FE2984D0024287891
:10BD2000400000F0FE00FAF709FE2B789C4280F0FC
:10BD30002482934B33F91400FAF703FE0134F4E73D
:10BD4000904C0620FAF7FAFDB4F90000FAF7F9FD75
:10BD5000B4F90200FAF7F5FD8B4BC3E10720FAF7BF
:10BD6000EDFD8A4B4FF6FF741878FAF7B8FD884B53
:10BD70001868A042A8BF204620EAE07000B2FAF797
:10BD8000E0FD844BB3F90000FAF7DBFD824B93F83A
:10BD90000C21824B18680028B8BF40420AB10A2320
:10BDA0005843A042A8BF204600B2D4E1714C0720FE
:10BDB000FAF7C4FD236893F85000FAF790FD236862
:10BDC00093F85100FAF78BFD236893F85400FAF7C3
:10BDD00086FD236893F85500FAF781FD236893F8F0
:10BDE0005600FAF77CFD236893F85200FAF777FDC6
:10BDF000236893F8530048E15E4D1E20FAF79EFD3C
:10BE00002B6800241B78022B69D12B68644903EB53
:10BE10008403586A01F026F804F0D8F9FA28A8BF7C
:10BE2000FA2020EAE070C0B2FAF759FD2B685D49AC
:10BE300003EB8403186B01F015F804F0C7F9FA2836
:10BE4000A8BFFA2020EAE070C0B2FAF748FD2B68DC
:10BE5000554903EB8403D86B01F004F804F0B6F9FC
:10BE60006428A8BF642020EAE070C0B20134FAF769
:10BE700036FD032CC9D1072C2B681ED1986C48497C
:10BE800000F0F0FF04F0A2F9FA28A8BFFA2020EA97
:10BE9000E070C0B2FAF723FD2B684149D86C00F07E
:10BEA000E1FF04F093F9FA28A8BFFA2020EAE07035
:10BEB000C0B2FAF714FD00200BE023441879FAF71A
:10BEC0000EFD2B682344987BFAF709FD2B68234469
:10BED000187E0134FAF703FD0A2CCCD14DE12B6812
:10BEE00023441879FAF7FBFC2B682344987BFAF774
:10BEF000F6FC2B682344187E0134FAF7F0FC0A2C78
:10BF0000EDD13AE12F20FAF719FD284C14F8010F72
:10BF1000002800F03281FAF7E2FCF7E7244D002414
:10BF20002878800000F0FC00FAF708FD2B789C428E
:10BF30000CD2204A0F4BA25C1B68203253F822001F
:10BF40000134C0F30B00FAF7FCFCEFE700242B7878
:10BF50009C4280F01281074B164A1B68A25C013498
:10BF600003EB8203B3F88200C0F30B00FAF7E9FC9D
:10BF7000EDE700BFDC03002066230020A70B0020B4
:10BF8000DE06002098030020D4040020A405002031
:10BF9000AC050020FE100020C01D0020A8050020D8
:10BFA000000020410000C84200007A441B31010813
:10BFB00011090020FC080020002C00F0DE80F8B2FF
:10BFC000FAF7BCFC002400256F4B1B789D42F3DA86
:10BFD0006E4BE95C00236E4A03EB02089A5C8A42CE
:10BFE00004D00C33B3F5847FF5D112E0D8F8040007
:10BFF00003F0C8FE81460CB9264601E0074408E07C
:10C000004E4506DAD8F80430985DFAF768FC013638
:10C01000F6E70135D8E75C4D00242878FAF78EFC66
:10C020002B789C4280F0A980584BE05C0023584A52
:10C0300099189A5C824204D00C33B3F5847FF6D110
:10C0400002E0087AFAF74BFC0134E9E7FAF72AFC38
:10C0500006461220FAF772FC002E46D14D4B1D68A1
:10C060005C683046FAF73BFC2846FAF78FFC20461E
:10C07000FAF78CFC484B1868FAF788FC0020FAF7AE
:10C0800060FC0020FAF75DFC0020FAF728FC74E061
:10C090000820FAF753FC0124E0B20134FAF71FFC40
:10C0A000092CF9D169E01020FAF748FC3B4B3C4CD5
:10C0B000187800F00200FAF712FC3A4B1878FAF7F9
:10C0C0000EFC2068FAF762FC6068FAF75FFC364BFA
:10C0D000B3F90000FAF735FC344BB3F90000FAF776
:10C0E00030FC334BB3F9000035E0102E01D1314B59
:10C0F000B5E700242546B4E7B3789C423DD22E4DE7
:10C10000285DFAF7ECFB05F11003185DFAF7E7FB81
:10C1100005F12003185D3035FAF7E1FB285DFAF7E9
:10C12000DEFB0134E8E70820FAF708FC0024234B83
:10C13000185F0234FAF705FC082CF8D11DE0204CFA
:10C140000420FAF7FBFB2368B3F95E00FAF7F9FB6A
:10C150002368B3F95C00FAF7F4FB0EE00C20FAF761
:10C16000EDFB184B1868FAF711FC174B1868FAF733
:10C170000DFC164B1868FAF709FC0120BDE8F8839E
:10C180000020BDE8F88300BF11090020FC08002052
:10C190004C310108C0190020480200207202002022
:10C1A000B0050020E80500201A0600201606002031
:10C1B000C41C0020C8190020C71C0020081D002036
:10C1C000DC030020E8F7FF1FECF7FF1FF0F7FF1F6D
:10C1D0000148FDF7BEBE00BF000800400148FDF762
:10C1E000B8BE00BF000400404FF08040FDF7B1BE74
:10C1F0000148FDF7AEBE00BF002C014038B5194C18
:10C20000236D1D88ADB2AA0612D5E26A1AB19888CC
:10C2100080B290470CE09B88E2696169DBB28B5485
:10C22000E269E3680132B2FBF3F103FB1123E3613E
:10C230002B0616D5A26A616A0A4B8A420CD098690D
:10C24000196D805C0132C0B288801969B2FBF1F0CF
:10C2500001FB10229A6238BD1B6DDA6822F0800261
:10C26000DA6038BD101D00200D4BD3F8A4201188D2
:10C27000090613D5D96F986F81420BD0D86E405CF8
:10C280000131C0B290805A6EB1FBF2F002FB101186
:10C29000D9677047D36823F08003D360704700BF2D
:10C2A000101D00200B480C4B4FF400525A60D0F880
:10C2B00088204FF6FE7311680B401360826FC36FC6
:10C2C0009A4202D05430FDF72BBE012380F89830FB
:10C2D000704700BF101D002000000240FAF7F4BBB9
:10C2E000FAF7F2BB084A13689B020BD5074B0021F3
:10C2F000197007494FF6FE73086803400B604FF44E
:10C3000000135360704700BF000002408E230020DE
:10C310006C000240F9F764BEF9F762BEFCF700BD9D
:10C32000FCF7FEBC074B1A685969490408D552044A
:10C3300006D54FF480425A61034B012283F8A820AE
:10C34000704700BF00040140101D00200F4B1A6809
:10C3500042F001021A6059680D4A0A405A601A6890
:10C3600022F0847222F480321A601A6822F4802249
:10C370001A605A6822F4FE025A604FF41F029A6053
:10C38000044B4FF000629A60704700BF00100240FB
:10C390000000FFF800ED00E0024B1A6801321A605D
:10C3A000704700BFBC1D002008B5084BB3F8D8008B
:10C3B00093F8A8250023D9B2914204D2044921F868
:10C3C00013000133F7E7F6F784F9FEE7BC1D002000
:10C3D0006623002081F0004102E000BF83F00043AB
:10C3E00030B54FEA41044FEA430594EA050F08BF10
:10C3F00090EA020F1FBF54EA000C55EA020C7FEAD4
:10C40000645C7FEA655C00F0E2804FEA5454D4EB50
:10C410005555B8BF6D420CDD2C4480EA020281EA1A
:10C42000030382EA000083EA010180EA020281EA52
:10C430000303362D88BF30BD11F0004F4FEA0131A4
:10C440004FF4801C4CEA113102D0404261EB4101B3
:10C4500013F0004F4FEA03334CEA133302D0524239
:10C4600063EB430394EA050F00F0A780A4F10104F5
:10C47000D5F1200E0DDB02FA0EFC22FA05F280182F
:10C4800041F1000103FA0EF2801843FA05F3594115
:10C490000EE0A5F120050EF1200E012A03FA0EFC94
:10C4A00028BF4CF0020C43FA05F3C01851EBE371BE
:10C4B00001F0004507D54FF0000EDCF1000C7EEBDB
:10C4C00000006EEB0101B1F5801F1BD3B1F5001F19
:10C4D0000CD349085FEA30004FEA3C0C04F1010438
:10C4E0004FEA445212F5800F80F09A80BCF1004F61
:10C4F00008BF5FEA500C50F1000041EB045141EAE3
:10C50000050130BD5FEA4C0C404141EB010111F4E3
:10C51000801FA4F10104E9D191F0000F04BF01468E
:10C520000020B1FA81F308BF2033A3F10B03B3F16C
:10C5300020020CDA0C3208DD02F1140CC2F10C02FC
:10C5400001FA0CF021FA02F10CE002F11402D8BF5A
:10C55000C2F1200C01FA02F120FA0CFCDCBF41EA26
:10C560000C019040E41AA2BF01EB0451294330BDF5
:10C570006FEA04041F3C1CDA0C340EDC04F11404D2
:10C58000C4F1200220FA04F001FA02F340EA0300A9
:10C5900021FA04F345EA030130BDC4F10C04C4F1EF
:10C5A000200220FA02F001FA04F340EA03002946CF
:10C5B00030BD21FA04F0294630BD94F0000F83F419
:10C5C000801306BF81F480110134013D4EE77FEAFC
:10C5D000645C18BF7FEA655C29D094EA050F08BF48
:10C5E00090EA020F05D054EA000C04BF1946104629
:10C5F00030BD91EA030F1EBF0021002030BD5FEA6D
:10C60000545C05D14000494128BF41F0004130BD94
:10C6100014F580043CBF01F5801130BD01F00045E8
:10C6200045F0FE4141F470014FF0000030BD7FEA5B
:10C63000645C1ABF194610467FEA655C1CBF0B4656
:10C64000024650EA013406BF52EA033591EA030F6D
:10C6500041F4002130BD00BF90F0000F04BF002165
:10C66000704730B54FF4806404F132044FF0000598
:10C670004FF0000150E700BF90F0000F04BF002111
:10C68000704730B54FF4806404F1320410F0004577
:10C6900048BF40424FF000013EE700BF42004FEA72
:10C6A000E2014FEA31014FEA02701FBF12F07F43EF
:10C6B00093F07F4F81F06051704792F0000F14BFEC
:10C6C00093F07F4F704730B54FF4607401F0004530
:10C6D00021F0004120E700BF50EA010208BF704787
:10C6E00030B54FF000050AE050EA010208BF70477C
:10C6F00030B511F0004502D5404261EB41014FF4E5
:10C70000806404F132045FEA915C3FF4DCAE4FF0E8
:10C7100003025FEADC0C18BF03325FEADC0C18BFCF
:10C72000033202EBDC02C2F1200300FA03FC20FA20
:10C7300002F001FA03FE40EA0E0021FA02F114446D
:10C74000C1E600BF70B54FF0FF0C4CF4E06C1CEA82
:10C7500011541DBF1CEA135594EA0C0F95EA0C0FF7
:10C7600000F0DEF82C4481EA030621EA4C5123EA6A
:10C770004C5350EA013518BF52EA033541F4801199
:10C7800043F4801338D0A0FB02CE4FF00005E1FB4C
:10C7900002E506F00042E0FB03E54FF00006E1FB96
:10C7A00003569CF0000F18BF4EF0010EA4F1FF04D9
:10C7B000B6F5007F64F5407404D25FEA4E0E6D4119
:10C7C00046EB060642EAC62141EA55514FEAC5202A
:10C7D00040EA5E504FEACE2EB4F1FD0C88BFBCF5A6
:10C7E000E06F1ED8BEF1004F08BF5FEA500E50F157
:10C7F000000041EB045170BD06F0004646EA01011D
:10C8000040EA020081EA0301B4EB5C04C2BFD4EB4E
:10C810000C0541EA045170BD41F480114FF0000E47
:10C82000013C00F3AB8014F1360FDEBF002001F0B5
:10C83000004170BDC4F10004203C35DA0C341BDC2F
:10C8400004F11404C4F1200500FA05F320FA04F001
:10C8500001FA05F240EA020001F0004221F0004135
:10C8600010EBD37021FA04F642EB06015EEA430EA8
:10C8700008BF20EAD37070BDC4F10C04C4F12005D8
:10C8800000FA04F320FA05F001FA04F240EA02008B
:10C8900001F0004110EBD37041F100015EEA430E5C
:10C8A00008BF20EAD37070BDC4F1200500FA05F27C
:10C8B0004EEA020E20FA04F301FA05F243EA0203FB
:10C8C00021FA04F001F0004121FA04F220EA02000A
:10C8D00000EBD3705EEA430E08BF20EAD37070BD50
:10C8E00094F0000F0FD101F00046400041EB010130
:10C8F00011F4801F08BF013CF7D041EA060195F012
:10C90000000F18BF704703F00046520043EB0303CB
:10C9100013F4801F08BF013DF7D043EA06037047B8
:10C9200094EA0C0F0CEA135518BF95EA0C0F0CD0C3
:10C9300050EA410618BF52EA4306D1D181EA030109
:10C9400001F000414FF0000070BD50EA410606BF03
:10C950001046194652EA430619D094EA0C0F02D148
:10C9600050EA013613D195EA0C0F05D152EA03368D
:10C970001CBF104619460AD181EA030101F00041AB
:10C9800041F0FE4141F470014FF0000070BD41F0F4
:10C99000FE4141F4780170BD70B54FF0FF0C4CF4CE
:10C9A000E06C1CEA11541DBF1CEA135594EA0C0FED
:10C9B00095EA0C0F00F0A7F8A4EB050481EA030E3A
:10C9C00052EA03354FEA013100F088804FEA033321
:10C9D0004FF0805545EA131343EA12634FEA0222EF
:10C9E00045EA111545EA10654FEA00260EF00041B0
:10C9F0009D4208BF964244F1FD0404F5407402D202
:10CA00005B084FEA3202B61A65EB03055B084FEA92
:10CA100032024FF480104FF4002CB6EB020E75EB8F
:10CA2000030E22BFB61A754640EA0C005B084FEAB7
:10CA30003202B6EB020E75EB030E22BFB61A754634
:10CA400040EA5C005B084FEA3202B6EB020E75EB7F
:10CA5000030E22BFB61A754640EA9C005B084FEAF7
:10CA60003202B6EB020E75EB030E22BFB61A754604
:10CA700040EADC0055EA060E18D04FEA051545EAF3
:10CA800016754FEA06164FEAC30343EA52734FEA9C
:10CA9000C2025FEA1C1CC0D111F4801F0BD141EA15
:10CAA00000014FF000004FF0004CB6E711F4801F7A
:10CAB00004BF01430020B4F1FD0C88BFBCF5E06F5A
:10CAC0003FF6AFAEB5EB030C04BFB6EB020C5FEA6A
:10CAD000500C50F1000041EB045170BD0EF0004EBF
:10CAE0004EEA113114EB5C04C2BFD4EB0C0541EAF1
:10CAF000045170BD41F480114FF0000E013C90E6EE
:10CB000045EA060E8DE60CEA135594EA0C0F08BFB1
:10CB100095EA0C0F3FF43BAF94EA0C0F0AD150EAB0
:10CB200001347FF434AF95EA0C0F7FF425AF104643
:10CB300019462CE795EA0C0F06D152EA03353FF46B
:10CB4000FDAE1046194622E750EA410618BF52EAE8
:10CB500043067FF4C5AE50EA41047FF40DAF52EABC
:10CB600043057FF4EBAE12E74A0011D212F5001232
:10CB700011D20DD56FF47873B3EB62520ED44FEA35
:10CB8000C12343F0004343EA505323FA02F07047B5
:10CB90004FF00000704750EA013002D14FF0FF30F3
:10CBA00070474FF0000070474FEA4102B2F1E04396
:10CBB00024BFB3F5001CDCF1FE5C0DD901F0004C84
:10CBC0004FEAC0024CEA5070B2F1004F40EB8300D4
:10CBD00008BF20F00100704711F0804F21D113F100
:10CBE0003872BCBF01F00040704741F480114FEA39
:10CBF0005252C2F11802C2F1200C10FA0CF320FAC2
:10CC000002F018BF40F001004FEAC1234FEAD323DE
:10CC100003FA0CFC40EA0C0023FA02F34FEA430348
:10CC2000CCE77FEA625307D150EA01331EBF4FF0D1
:10CC3000FE4040F44000704701F0004040F0FE40EC
:10CC400040F40000704700BF80F0004002E000BFE9
:10CC500081F0004142001FBF5FEA410392EA030FE7
:10CC60007FEA226C7FEA236C6AD04FEA1262D2EB31
:10CC70001363C1BFD218414048404140B8BF5B4236
:10CC8000192B88BF704710F0004F40F4000020F0CF
:10CC90007F4018BF404211F0004F41F4000121F0E5
:10CCA0007F4118BF494292EA030F3FD0A2F101022F
:10CCB00041FA03FC10EB0C00C3F1200301FA03F16D
:10CCC00000F0004302D5494260EB4000B0F5000F90
:10CCD00013D3B0F1807F06D340084FEA310102F14F
:10CCE0000102FE2A51D2B1F1004F40EBC25008BF01
:10CCF00020F0010040EA03007047490040EB0000CB
:10CD000010F4000FA2F10102EDD1B0FA80FCACF1F9
:10CD1000080CB2EB0C0200FA0CF0AABF00EBC250F8
:10CD200052421843BCBFD0401843704792F0000FE6
:10CD300081F4000106BF80F400000132013BB5E739
:10CD40004FEA41037FEA226C18BF7FEA236C21D0AF
:10CD500092EA030F04D092F0000F08BF0846704714
:10CD600090EA010F1CBF0020704712F07F4F04D1E2
:10CD7000400028BF40F00040704712F100723CBFF5
:10CD800000F50000704700F0004343F0FE4040F41F
:10CD9000000070477FEA226216BF08467FEA2363DD
:10CDA0000146420206BF5FEA412390EA010F40F4C8
:10CDB000800070474FF0000304E000BF10F0004314
:10CDC00048BF40425FEA000C08BF704743F09643FB
:10CDD00001464FF000001CE050EA010208BF704716
:10CDE0004FF000030AE000BF50EA010208BF70479D
:10CDF00011F0004302D5404261EB41015FEA010CB2
:10CE000002BF84460146002043F0B64308BFA3F1A9
:10CE10008053A3F50003BCFA8CF2083AA3EBC2538B
:10CE200010DB01FA02FC634400FA02FCC2F12002AA
:10CE3000BCF1004F20FA02F243EB020008BF20F0E1
:10CE40000100704702F1200201FA02FCC2F1200247
:10CE500050EA4C0021FA02F243EB020008BF20EA3C
:10CE6000DC7070474FF0FF0C1CEAD0521EBF1CEA6A
:10CE7000D15392EA0C0F93EA0C0F6FD01A4480EA58
:10CE8000010C400218BF5FEA41211ED04FF0006341
:10CE900043EA501043EA5111A0FB01310CF000406D
:10CEA000B1F5000F3EBF490041EAD3715B0040EA93
:10CEB000010062F17F02FD2A1DD8B3F1004F40EB63
:10CEC000C25008BF20F00100704790F0000F0CF036
:10CED000004C08BF49024CEA502040EA51207F3AFA
:10CEE000C2BFD2F1FF0340EAC250704740F40000D5
:10CEF0004FF00003013A5DDC12F1190FDCBF00F0C6
:10CF000000407047C2F10002410021FA02F1C2F173
:10CF1000200200FA02FC5FEA310040F1000053EA0F
:10CF20004C0308BF20EADC70704792F0000F00F05D
:10CF3000004C02BF400010F4000F013AF9D040EA63
:10CF40000C0093F0000F01F0004C02BF490011F4F7
:10CF5000000F013BF9D041EA0C018FE70CEAD153F5
:10CF600092EA0C0F18BF93EA0C0F0AD030F0004C75
:10CF700018BF31F0004CD8D180EA010000F0004029
:10CF8000704790F0000F17BF90F0004F084691F0E7
:10CF9000000F91F0004F14D092EA0C0F01D1420221
:10CFA0000FD193EA0C0F03D14B0218BF084608D1EA
:10CFB00080EA010000F0004040F0FE4040F4000034
:10CFC000704740F0FE4040F4400070474FF0FF0CC7
:10CFD0001CEAD0521EBF1CEAD15392EA0C0F93EA0E
:10CFE0000C0F69D0A2EB030280EA010C49024FEA60
:10CFF000402037D04FF0805343EA111143EA101319
:10D000000CF000408B4238BF5B0042F17D024FF4D0
:10D01000000C8B4224BF5B1A40EA0C00B3EB510FAB
:10D0200024BFA3EB510340EA5C00B3EB910F24BF94
:10D03000A3EB910340EA9C00B3EBD10F24BFA3EB19
:10D04000D10340EADC001B0118BF5FEA1C1CE0D1E1
:10D05000FD2A3FF650AF8B4240EBC25008BF20F094
:10D06000010070470CF0004C4CEA50207F32C2BFE8
:10D07000D2F1FF0340EAC250704740F400004FF085
:10D080000003013A37E792F0000F00F0004C02BFB6
:10D09000400010F4000F013AF9D040EA0C0093F080
:10D0A000000F01F0004C02BF490011F4000F013BDA
:10D0B000F9D041EA0C0195E70CEAD15392EA0C0F42
:10D0C00008D142027FF47DAF93EA0C0F7FF470AF7A
:10D0D000084676E793EA0C0F04D14B023FF44CAFBD
:10D0E00008466EE730F0004C18BF31F0004CCAD152
:10D0F00030F000427FF45CAF31F000437FF43CAF8E
:10D100005FE700BF4FF0FF3C06E000BF4FF0010CAF
:10D1100002E000BF4FF0010C4DF804CD4FEA400291
:10D120004FEA41037FEA226C18BF7FEA236C11D0DB
:10D1300001B052EA530C18BF90EA010F58BFB2EB8E
:10D14000030088BFC81738BF6FEAE17018BF40F00E
:10D15000010070477FEA226C02D15FEA402C05D1C2
:10D160007FEA236CE4D15FEA412CE1D05DF8040B47
:10D17000704700BF844608466146FFE70FB5FFF7DA
:10D18000C9FF002848BF10F1000F0FBD4DF808ED92
:10D19000FFF7F4FF0CBF012000205DF808FB00BF83
:10D1A0004DF808EDFFF7EAFF34BF012000205DF8DD
:10D1B00008FB00BF4DF808EDFFF7E0FF94BF01202A
:10D1C00000205DF808FB00BF4DF808EDFFF7D2FF27
:10D1D00094BF012000205DF808FB00BF4DF808ED6A
:10D1E000FFF7C8FF34BF012000205DF808FB00BF37
:10D1F0004FEA4002B2F1FE4F0FD34FF09E03B3EB64
:10D2000012620DD94FEA002343F0004310F0004FA3
:10D2100023FA02F018BF404270474FF000007047F9
:10D2200012F1610F01D1420205D110F0004008BF98
:10D230006FF0004070474FF00000704742000ED280
:10D24000B2F1FE4F0BD34FF09E03B3EB126209D441
:10D250004FEA002343F0004323FA02F070474FF0F7
:10D260000000704712F1610F01D1420202D14FF06C
:10D27000FF3070474FF00000704700BF73B96AB9C4
:10D28000002908BF0028BCBF00204FF00041C4BFE8
:10D290006FF000414FF0FF3000F03CB882B0EC4638
:10D2A0002DE9005000F006F8DDF804E002B00CBCF7
:10D2B000704700BF2DE9704F089E14461D468046FA
:10D2C000894600F029F804FB01F3A4FB00AB00FB46
:10D2D00005329344B8EB0A0869EB0B09C6E90089EB
:10D2E000BDE8708F2DE9704F089E14461D4680469C
:10D2F000894600F061F900FB05F5A0FB04AB04FBD7
:10D300000154A344B8EB0A0869EB0B09C6E900898C
:10D31000BDE8708F704700BF00292DE9F00FC0F203
:10D32000A1800024002BC0F29880154606460F46C7
:10D33000002B3FD18A4258D9B2FA82F34BB1C3F1E4
:10D34000200201FA03F720FA02F29D4000FA03F6E8
:10D350001743290CB7FBF1F201FB1277A8B200FBCF
:10D3600002F34FEA164C4CEA0747BB4209D97F1932
:10D3700002F1FF3C80F00581BB4240F20281023A9B
:10D380002F44FF1AB7FBF1F301FB137100FB03F00D
:10D39000B6B246EA0141884208D9491903F1FF377C
:10D3A00080F0F180884240F2EE80023B43EA024284
:10D3B000002303E08B420AD900231A46104619467F
:10D3C00014B1404261EB4101BDE8F00F7047B3FA80
:10D3D00083F8B8F1000F40F088808B4202D382427C
:10D3E00000F2E28000230122E8E712B90123B3FB37
:10D3F000F2F5B5FA85F2002A3AD17F1B280C1FFA04
:10D4000085FC0123B7FBF0F100FB11770CFB01F267
:10D410004FEA164848EA0747BA4207D97F1901F18F
:10D42000FF3802D2BA4200F2C4804146BF1AB7FBAD
:10D43000F0F200FB12700CFB02FCB6B246EA0040B0
:10D44000844507D9401902F1FF3702D2844500F222
:10D45000AE803A4642EA0142B0E7E443524263EB0F
:10D46000430362E7404261EB41014FF0FF3459E76B
:10D470009540C2F1200927FA09F126FA09F99740E7
:10D48000280CB1FBF0F800FB18111FFA85FC0CFB0F
:10D4900008F349EA07094FEA194747EA01418B4275
:10D4A00006FA02F608D9491908F1FF327AD28B42FE
:10D4B00078D9A8F102082944C91AB1FBF0F300FB9E
:10D4C00013170CFB03F21FFA89F949EA0747BA421E
:10D4D00007D97F1903F1FF3160D2BA425ED9023B0E
:10D4E0002F44BF1A43EA08438CE7C8F1200225FA0B
:10D4F00002F103FA08FC27FA02F320FA02F207FA13
:10D5000008F741EA0C0C4FEA1C49B3FBF9F109FB9F
:10D5100011331FFA8CFA0AFB01FB17433A0C42EA5B
:10D5200003439B4505FA08F008D913EB0C0301F1FE
:10D53000FF3235D29B4533D902396344CBEB030329
:10D54000B3FBF9F209FB12330AFB02FABFB247EA56
:10D550000347BA4508D917EB0C0702F1FF331BD27A
:10D56000BA4519D9023A674442EA0145A5FB0001D0
:10D57000CAEB07078F424FF000030AD305D02A46B3
:10D580001CE76246FDE63B4610E706FA08F68642CF
:10D59000F5D26A1E002311E71A46E5E70B46A0E71D
:10D5A0001146CBE7904687E74346424606E7023AF4
:10D5B00050E702392F4439E72DE9F00F14460546AC
:10D5C0000E46002B43D18A4253D9B2FA82F757B1A3
:10D5D000C7F1200620FA06F601FA07F302FA07F46B
:10D5E00000FA07F51E43210CB6FBF1F201FB1266AF
:10D5F000A0B200FB02F32F0C47EA0646B34209D95A
:10D60000361902F1FF3780F0FD80B34240F2FA8014
:10D61000023A2644F61AB6FBF1F301FB136100FB54
:10D6200003F0ADB245EA0141884208D9091903F176
:10D63000FF3680F0E980884240F2E680023B43EA10
:10D640000242002310461946BDE8F00F70478B4296
:10D650004CD8B3FA83F6002E4FD18B4202D38242CC
:10D6600000F2DD80BDE8F00F0023012210461946CC
:10D67000704712B90124B4FBF2F4B4FA84F2002A20
:10D6800040F08280091B260CA7B20123B1FBF6F003
:10D6900006FB101107FB00F24FEA154C4CEA014162
:10D6A0008A4207D9091900F1FF3C02D28A4200F2EE
:10D6B000C8806046891AB1FBF6F206FB121107FB1F
:10D6C00002F7ADB245EA0145AF4208D92C1902F183
:10D6D000FF3180F09B80A74240F29880023A42EAF4
:10D6E000004210461946BDE8F00F704700231A4665
:10D6F00010461946BDE8F00F7047C6F1200522FA22
:10D7000005F703FA06F421FA05F301FA06FB20FAFD
:10D7100005F53C434FEA1448B3FBF8FC08FB1C3307
:10D720001FFA84F909FB0CFA45EA0B0B4FEA1B457B
:10D7300045EA03439A4502FA06F204D91B190CF193
:10D74000FF356FD3AC46CAEB0303B3FBF8F508FB18
:10D75000153309FB05F91FFA8BFB4BEA0347B94563
:10D7600004D93F1905F1FF3362D31D4645EA0C4C3D
:10D77000ACFB0223C9EB07079F424FF000054AD3D9
:10D7800046D062462B465DE79440C2F1200921FA5B
:10D7900009FC914020FA09F9260CBCFBF6F806FBBF
:10D7A00018CCA7B207FB08F349EA01094FEA19416F
:10D7B00041EA0C4C634500FA02F509D91CEB040C54
:10D7C00008F1FF323BD2634539D9A8F10208A444DD
:10D7D000C3EB0C0CBCFBF6F306FB13C107FB03F217
:10D7E0001FFA89F949EA01418A4207D9091903F167
:10D7F000FF3022D28A4220D9023B2144891A43EACF
:10D80000084343E73A4605E7334618E70A4666E722
:10D81000B0409042B5D20CF1FF32002312E73346FC
:10D8200032460FE79A458DD9ACF1020C23448AE7C2
:10D83000B9459AD9023D274498E70346DEE790466A
:10D84000C6E70238214435E74FF0FF3C06E000BF51
:10D850004FF0010C02E000BF4FF0010C4DF804CD79
:10D860004FEA410C7FEA6C5C4FEA430C18BF7FEA39
:10D870006C5C1BD001B050EA410C0CBF52EA430C67
:10D8800091EA030F02BF90EA020F0020704710F1E7
:10D89000000F91EA030F58BF994208BF90422CBF76
:10D8A000D8176FEAE37040F0010070474FEA410C6F
:10D8B0007FEA6C5C02D150EA013C07D14FEA430C8D
:10D8C0007FEA6C5CD6D152EA033CD3D05DF8040BFE
:10D8D000704700BF8446104662468C461946634630
:10D8E00000E000BF01B5FFF7B7FF002848BF10F107
:10D8F000000F01BD4DF808EDFFF7F4FF0CBF01204C
:10D9000000205DF808FB00BF4DF808EDFFF7EAFFC7
:10D9100034BF012000205DF808FB00BF4DF808ED82
:10D92000FFF7E0FF94BF012000205DF808FB00BF77
:10D930004DF808EDFFF7CEFF94BF012000205DF801
:10D9400008FB00BF4DF808EDFFF7C4FF34BF01200E
:10D9500000205DF808FB00BF1C481D4902680060FC
:10D960008A4200F01D80002100F004B8194B5B587A
:10D97000435004311848194B42189A42FFF4F6AF4D
:10D98000174A00F003B8002342F8043B154B9A42B3
:10D99000FFF4F9AFFEF7DAFC00F036F8FFF7FEBF50
:10D9A000114E124830601248016821F07061016028
:10D9B000410201600F4C182020600F490F48086099
:10D9C0000F48D0F800D0406800470000F04F00201A
:10D9D000EFBEADDED055010800000020240100207C
:10D9E00028010020B0230020181002400900000088
:10D9F00004000140140C0140000C01404434434435
:10DA000000F0FF1FFFF7FEBF2DE9804893B0F2F74B
:10DA10007FFBA14EA14CD6F80880002318F0080F18
:10DA20002370374600F0CA8063681B7A042B00F22B
:10DA3000C380DFE803F00303056D9400237ABCE0A4
:10DA4000627A964B002A00F0B78000225A7293F84F
:10DA50002020150700F1B080D97A9A7A01F00700EA
:10DA600042EA00225A621A7B02F03F00400140EA7B
:10DA7000D1019962597B890041EA92119A7B02F0A7
:10DA8000010041EA8021D962D97B01F00F00C00179
:10DA900040EA52021A631A7C02F07F00000140EA59
:10DAA00011115963597C490041EAD212997C01F065
:10DAB000030042EA40229A63DA7C02F01F008001F0
:10DAC00040EA9101D963197DC90041EA5212997D5A
:10DAD0001A645A7D01F0070042EA00225A64DA7D96
:10DAE00002F03F00400140EAD1019964197E8900AB
:10DAF00041EA92115A7E02F0010041EA8021D96484
:10DB0000997E01F00F01C90141EA52021A6551E004
:10DB100094F85420614B002A4ED0002283F8542000
:10DB200093F85620012A47D193F87A20102A84BF0F
:10DB3000102283F87A2094F87A10594A0023D8B238
:10DB4000884202F1020235D212F8010C12F8025C8E
:10DB500040EA0525534840F823500133EFE794F895
:10DB6000BC204E4B42B3002283F8BC2093F8BD206A
:10DB7000A82A21D193F8D050F5B9484901EB4503C3
:10DB800093F8C00093F8C13003EB0020FEF764FD6A
:10DB90003DA3D3E90023FEF7FFFE3DA3D3E9002315
:10DBA000FEF71CFCFEF7E0FF3F4B43F82500013574
:10DBB000082DE2D1012300E00023237018F4804FE8
:10DBC00008D094F8F43023B1344B002283F8F420C9
:10DBD00001232370237843B118F4807F05D02F4BA5
:10DBE000D3F8F8301B681B689847304B22781B68C5
:10DBF00032B92A4AD2F8FC209A1AD243D20F00E056
:10DC000001227AB3F6F7CCF994F80021234B002ACD
:10DC100000F0CB83D3F80421500740F1C68393F87A
:10DC20000B21C2B1B3F81E1101F0080292B2002A12
:10DC300040F0BB8341F00801A3F81E11D3F8241172
:10DC4000C3F83421C3F82011B3F83011C3F83821D8
:10DC5000A3F82811A9E3B3F81E2122F00802A3F8C3
:10DC60001E21A2E3D4F83C21511CC4F83C11052A22
:10DC700000F29383DFE812F01C00AE001C01700379
:10DC80006A038C03AFF300809A9999999999194086
:10DC90000000000000707740C01D00202801002017
:10DCA00080010020A4010020FC010020802300202E
:10DCB000D4F80421784D110740F16F83D5F8402145
:10DCC0009A1A002AC0F2698303F5C33805F5A270D9
:10DCD00008F1A008C5F84081F7F784FF6F4B05F500
:10DCE000A27001461A78F8F7CBFC95F84A1105F5B1
:10DCF000A27011F0040F17D0C5F84C810022BB1898
:10DD00000025A3F8FE50644B855A03F5A87E22F83F
:10DD10000E5003F5AB7E22F80E500232062AEED1E9
:10DD200021F0040183F84A1194F85C315A4AA3B1F6
:10DD3000B2F84411B6F8FE30CB1AA2F84431B2F86A
:10DD40004611B6F80031CB1AA2F84631B2F84811A4
:10DD5000B6F80231CB1AA2F84831D4F84C314E4A09
:10DD6000002B00F01A834E49C3EB08038B4202F5E7
:10DD7000A87502F5AB7119D84A4BDA6882F008022F
:10DD8000DA600023C25A35F903E017B2BE45C4BFBA
:10DD9000DFF818E123F80E2031F903E0BE45BCBFDF
:10DDA000414FDA530233062BECD1F6E20023C2F8DE
:10DDB0004C3135F903E0C85EFA1870444FF0020E9A
:10DDC000734490FBFEF0062BA2F8FE00F1D1F9F7A8
:10DDD000B7FFE2E2D4F804212F4D520740F1DD8273
:10DDE000D5F860219A1A002AC0F2D782C5F86031AE
:10DDF00095F86431012B14D002D3022B29D0CCE248
:10DE0000D5F870319847D5F874319847012385F8D3
:10DE10006431B5F86A21D5F860311344C5F8603132
:10DE2000BBE2D5F878319847D5F86C319847D5F8EA
:10DE30006031B5F8682105F5C0701344C5F860314C
:10DE400005F5C271D5F87C319847022385F8643115
:10DE5000A3E2D5F89001D5F88C1100784B1C00276F
:10DE6000834285F86471D5F888E1D5F8802103D123
:10DE7000012385F894313B460748C4F88C3100EB08
:10DE80008101C1F8982100EB8301D1F89811724407
:10DE9000521AC4F8882180E2280100208F23002034
:10DEA0007FC3C901000C01407E02002078020020DF
:10DEB000D4F80421B14D570740F16F8295F89421B1
:10DEC000002A00F06A82D5F85822C2EB030B46F212
:10DED000A712934540F26182A94FC5F85832B7F8AE
:10DEE0000080B8F1000F2FD0D5F89031D5F85C2222
:10DEF0001878D5F888310138B3FBF0F0082392FB8D
:10DF0000F3F1521A1044C5F85C0290FBF3F0FEF7EF
:10DF100055FF9C49FFF75AF89B4902F025FA014644
:10DF20004FF07E50FEF794FE9849FEF79BFFFFF7F7
:10DF30005FF908F1FF380023C5F86002A7F80080F8
:10DF4000C5F86432C5F86832D4F89051D4F88831F5
:10DF500028780138B3FBF0F0FEF72CFF8949FFF772
:10DF600035F8894902F000FA01464FF07E50FEF77D
:10DF70006FFE8649FEF776FF02F028F96F6881464A
:10DF8000D4F86C02FEF71AFF3946FEF76BFF8046A5
:10DF9000D4F86002C0EB0900FEF710FF3946814655
:10DFA0004FF07E50FEF754FE01464846FEF75AFFFA
:10DFB00001464046FEF74EFE02F008F9B4F97072D1
:10DFC000B4F97232002FB8BF7F42002BB8BF5B425A
:10DFD0009F42B8BF1F46DFF8C8813FB2FA2F824682
:10DFE000D8F8000014DCFEF7E9FE81463846FEF75B
:10DFF000E5FE01466648FEF72BFE01464846FEF761
:10E0000031FF6349FEF7E2FFFFF7F2F8074601E050
:10E010004FF0FF377B1EC62BC8F8007006D8C7EB41
:10E020000A03C4F87432C4F86C722EE0D4F8743267
:10E03000002FDFF84891C3EB0A0A02DCC9F86CA292
:10E0400023E0C7F59670FEF7B9FE5249FEF7BEFF12
:10E0500080463846FEF7B2FE4146FEF703FF07460C
:10E060005046FEF7ABFE414682464FF07E50FEF72B
:10E07000EFFD01465046FEF7F5FE01463846FEF735
:10E08000E9FDFFF7B5F8C9F86C02434B1868019336
:10E09000FEF790FE41490746FEF7E4FE8246D4F8BB
:10E0A0008002FEF78BFE8046D4F88402FEF786FEDF
:10E0B00001464046FEF78AFFD4F888120490FEF726
:10E0C000D1FE3946FEF7CEFE4FF07C51D4F8648283
:10E0D000D5F80C90D4F86C720290FEF7C3FE51464E
:10E0E000FEF7C0FE5146024640460392FEF7BAFED6
:10E0F000039A01461046FEF7ADFDD4F86812FEF70C
:10E10000A9FD4946FEF7AEFE82463846FEF756FEAA
:10E11000494602464FF07E500392FEF799FD039A5E
:10E1200001461046FEF79EFE01465046FEF792FD60
:10E13000DDF808C0C4F86802814661464046FEF733
:10E1400089FD0022C4F86402C4F87822C4F87C2255
:10E15000C4F88022C4F88422019B80461A60084BD0
:10E160001B88002B40F019810D4B1B68013BC62B0F
:10E1700018D80249C1F824711AE000BF2801002014
:10E180008423002080E6C547B1DC423ED048874A60
:10E19000000061440000C84288230020BD37863556
:10E1A000980000204846FFF723F8A64AC2F8240149
:10E1B000D4F88C02381AFEF701FEA349FEF752FE8E
:10E1C00081465846FEF7F6FD01464846FEF7FEFE3C
:10E1D000FFF70EF840F2DC539C4A9842A8BF18465D
:10E1E0009042B8BF10460A21C4F88C72F4F7E8FBDD
:10E1F000AD68814629464046FEF734FE074648464C
:10E20000FEF7DCFD294680464FF07E50FEF720FDEC
:10E2100001464046FEF726FE01463846FEF71AFD47
:10E22000C4F8640201F0D2FF05218146F4F7C8FB6F
:10E23000B4F8702240F23E6302F21F3292B29A4268
:10E24000C4F89002D4F894820AD87E4AB2F87202D6
:10E2500000F21F3080B298428CBF0020012000E005
:10E26000002000286CD094F89832764F13BBD7F872
:10E270002021D7F824317648D31AB3F5FA7FA8BF06
:10E280004FF4FA738342A8BF18460A21F4F798FBAB
:10E29000D7F89C32DD788023684390FBF3F5B5F521
:10E2A000967FA8BF4FF49675A3F5D6739D42B8BF6D
:10E2B0001D4601E0D7F8A052D4F89C32C9EB0509FD
:10E2C0005F7A202209FB07F797FBF2F7B7F5967FF5
:10E2D000A8BF4FF49677A2F5A672DD7C9742B8BF2F
:10E2E0001746D4F83421587F09FB0525594AB5F55E
:10E2F000C81FA8BF4FF4C8159542B8BF1546C4F84B
:10E300003451FEF75BFD414681460498FEF7A2FCBE
:10E3100001464846FEF7A6FD4FF06C51FEF7A2FD00
:10E32000FEF766FF6FF095039628A8BF96209842E7
:10E33000B8BF1846381A4FF4005795FBF7F5284434
:10E34000049BC4F83801C4F8943226E0B3681D0673
:10E3500023D5F4F7C5FE20E0D4F80421394BD006CC
:10E360001BD53D4AD3F8A41212683C318A4214D31B
:10E37000C3F8A422D3F8AC72384A394DC3F8A822A6
:10E380003B880B202B61F8F785FC3B886B6104E030
:10E39000B368990301D5F6F7E7F9D4F83C31052BBA
:10E3A00003DD284B0022C3F83C21F8F773FB2D4B0B
:10E3B0001860B3892BB1D4F8B022821A002AC0F2B7
:10E3C0005E8718441F4DC4F8B0027079D4F8BC328F
:10E3D000059005F53270D4F8B472984705F532709F
:10E3E000014694F8CE22F8F74BF91F4B1B88002BFF
:10E3F00000F0B580D5F8D0324FF000091B7805F554
:10E4000035750493C846184BB3F800A0174BBAF5FE
:10E410007A7F03D1002243F809202A61144A32F995
:10E42000080053F80920024443F80920FEF7C6FC0F
:10E430002A690132012A2A611CD100236860286000
:10E44000AB6042E0280100200024744924FAFFFF59
:10E450000CFEFFFF0000E7FFBC1D0020980000201D
:10E46000000C0140802300208C2300203804002071
:10E47000F0030020D5F800C003926146CDF808C033
:10E480000190FEF7E5FB039A83461046FEF796FCE3
:10E4900001465846FEF79AFDDDF808C00146604681
:10E4A000FEF7D8FB019B02461146686018460392AE
:10E4B000FEF7CEFB01465846FEF7D4FCA968FEF7EE
:10E4C000C9FB039AE8602A60A860694A002302F148
:10E4D000540BBAF1010F28F8023028F80B30DFF89E
:10E4E000A0A12DD12869012807DD0138FEF766FCBF
:10E4F0000146E868FEF76AFD00E0002002F0BCF883
:10E500000499034661B108460193FEF757FC019B4D
:10E5100001461846FEF762FE10B14FF47A731CE014
:10E52000544B4FF47A7259F803300A2003F5FA730A
:10E5300093FBF2F32BF808300F210122F8F7BFFB11
:10E5400008F10208B8F1060F09F1040905F11405F4
:10E550007FF459AFBAF80030013BAAF8003000232D
:10E56000454D05F5327205F54771985A595A411AC9
:10E5700099520233062BF3D1D5F8043113F002037C
:10E5800000F01883D5F8283305F54C70984705F549
:10E590004C70014695F83623F8F772F8B5F8383321
:10E5A00005F54C78002B45D00022D5F83C031346E6
:10E5B000314D38F902C0B5F8381305F5507EB1F584
:10E5C000C87F04BF00214EF803105EF803102A4DE7
:10E5D00061444EF80310043300210C2B28F802107C
:10E5E000815202F10202E3D1B5F83833012B1CD17C
:10E5F000D5F840334FF4C872C83393FBF2F303806D
:10E60000D5F84433C83393FBF2F34380D5F848334D
:10E61000C83393FBF2F2194B1B88D21A8280A7F8F9
:10E620005C10A7F85E10F9F78BFBB4F83833013BA8
:10E63000A4F83833B3685A0740F18580B4F84C2306
:10E640000D4B322A1ED1D3F83C231188A3F84E1368
:10E6500051889288A3F85013A3F85223B7F85C208E
:10E66000A3F85423B7F85E20A3F856230CE000BFAC
:10E67000F0030020380400202801002000000020C2
:10E680008C230020002A3CD00021D4F83C530A46B9
:10E69000914838F901E0B0F84C3300F55676322B4A
:10E6A00004BF0023B350B0588B4B7044B0500432B9
:10E6B00000200C2A28F80100685201F10201E7D17C
:10E6C000B3F84C23012A17D183F86523022283F87B
:10E6D0006623B3F84E2383F864032A80B3F85023EB
:10E6E0006A80B3F85223AA80B3F85423B3F85633A0
:10E6F000A7F85C20A7F85E30B4F84C33013BA4F8CF
:10E700004C3394F86723744BEAB1D3F85853D3F8D9
:10E710003C133220002295FBF0F583F867230D802F
:10E72000D3F85C5395FBF0F54D80D3F8603393FB41
:10E73000F0F06A4B1B88C01A8880A7F85C20A7F805
:10E740005E20F9F7FDFAD4F83C33B4F830131A8898
:10E7500000268A1AA4F83023B4F832135A88B14636
:10E760008A1AA4F832239B88B4F83423D31AA4F865
:10E770003433F8F78FF9D4F868330546C31A1846CE
:10E780000493FEF717FBD4F86C130690FEF76AFBB0
:10E79000D4F87083C4F8685398F800A00790354601
:10E7A0004F4F785FFEF70AFB0799FEF75BFB09A95D
:10E7B0008851BAF1000F2DD05046FEF7FFFA0146FE
:10E7C0004FF07E50FEF702FC0246114607F1AC0BFB
:10E7D0004FF07E500392FEF73BFA56F80B10FEF70F
:10E7E00041FB07F168018446485FCDF808C0FEF799
:10E7F000E5FA039AB8371146FEF734FBDDF808C096
:10E8000001466046FEF726FA4BF80600FEF7F0FCDC
:10E81000785304E007F1B8026837E95BA952314F39
:10E820000436EA5F0235062D02FB0299B8D12B4D62
:10E830004FF0640A2A880AFB09F3524393FBF2FA69
:10E84000AAF1490A07F1080009A91FFA8AFAF3F7A1
:10E8500085FFBAF13B0FD8F8046011D9B4F99403DD
:10E86000FEF7ACFAD4F8906301463046FEF7B6FCEA
:10E87000194F94F84A31002838D043F0080337E0A4
:10E880004FF07E513046FEF7E5F901464FF07E50DD
:10E89000FEF79CFB4FF0000B8246134B304653F8BB
:10E8A0001B100193FEF7DEFA024637F90B000392C4
:10E8B000FEF784FA039A01461046FEF7CBF951465B
:10E8C000FEF7D0FA019B43F81B000BF1020BBBF1E2
:10E8D000060FE2D1C2E700BF28010020000000209F
:10E8E000F0030020A8040020B004002023F0080357
:10E8F0003146D4F88C0387F84A3101F033FD0746DE
:10E90000C4F89803D4F88803D4F890B300F1004613
:10E91000D4F88C030146FEF7A5FA594682465846BC
:10E92000FEF7A0FA01465046FEF794F901F0A4FE66
:10E930000146304601F016FD0646C4F89C033846F1
:10E94000FDF7ACFEACA3D3E90023FDF7FBFEFEF719
:10E950002BF901F03BFCA4F870023046FDF79EFE57
:10E96000A5A3D3E90023FDF7EDFEFEF71DF901F0A5
:10E970002DFCD4F80431A4F872021B0739D5A24843
:10E9800009A9F3F7EBFED8F808904FF07E514846FE
:10E99000FEF760F901464FF07E50FEF717FB4FF08F
:10E9A000000B8246994D484605F5687353F81B10D5
:10E9B0000193FEF757FA05F5A271024631F90B00F3
:10E9C0000392FEF7FBF9039A01461046FEF742F95F
:10E9D0005146FEF747FA019B43F81B000BF1020B6F
:10E9E000BBF1060FDED11846F3F770FFA5F8AC03B4
:10E9F00041E0DFF828A209A90AF10400F3F7AEFE0E
:10EA00006868D5F808B00146FEF72CFAD5F80C90E6
:10EA1000594605465846FEF725FA01462846FEF7B0
:10EA200019F9494605464846FEF71CFA01462846AC
:10EA3000FEF710F901F020FE00210546FEF7A6FBC7
:10EA4000A0B9DAF804002946FEF7C0FA2946CAF848
:10EA50000400DAF80800FEF7B9FA2946CAF80800F7
:10EA6000DAF80C00FEF7B2FACAF80C006848F3F7BF
:10EA70002DFFA4F8AC0367490698FEF7F3F907F1F8
:10EA80000047814606F10046B4F9AC030C970D9699
:10EA9000FEF794F900F10040FDF700FE58A3D3E91A
:10EAA0000023FDF74FFEFEF77FF80E90B4F98003C8
:10EAB000FEF784F90F90B4F98203FEF77FF9109006
:10EAC000B4F98403FEF77AF90CA911900FA8F3F7B3
:10EAD00045FE98F801304D4D012B19D14E4B1B7856
:10EAE0005E070ED4D5F8B033402093FBF0F0181A2F
:10EAF000FEF764F91199FEF7ADF8FEF779FBC5F85A
:10EB0000B003424BD3F8B003402390FBF3F001E095
:10EB1000424B1888FEF752F901461198FEF798F813
:10EB2000D4F8B81311904846FEF794F801464846C9
:10EB3000FEF74CFAD4F8B453064629461198FEF76E
:10EB400087F801463046FEF78DF901462846FEF764
:10EB500081F80646C4F8B4030F98D4F8787201F02F
:10EB600035FBD4F8BC532978F3F72AFF3844C4F8AE
:10EB700078021098D4F87C7201F028FB2978F3F71A
:10EB80001FFF3844C4F87C023046D4F8807201F08C
:10EB90001DFB6978F3F714FF214B049D1A68384474
:10EBA0002A441A60D4F88432C4F880020133C4F8CD
:10EBB000843205E0A5F83033A5F83233A5F83433B4
:10EBC000DFF84890059DB9F8C832012DA9F8C03387
:10EBD000B9F8CA32A9F8C23324D1B9F9C623B9F9B0
:10EBE000CC3203EB4203032293FBF2F39BB2A9F86E
:10EBF000C433A9F8C63319E03B597E90A9E7814098
:10EC0000399D52A246DF913FC80400202801002010
:10EC100004000020BD378635962300200000002028
:10EC200088230020B9F8CC32A9F8C433F7F732FFB3
:10EC3000C74B01261860D9F8CC33C9F8CC03C31AE6
:10EC4000A9F8C833FBF794FC99F81C31C14D89F839
:10EC50000061002B00F08B80B5F81E31180600F122
:10EC6000CE80BD4B1B7859076FD595F8D023BB4B91
:10EC700012B195F8D1233AB10022C9F8D423012268
:10EC80001A74002289F8D1231B7CD9F8B452032BC3
:10EC900095F80080AF4E05F1040789F8D03306D10E
:10ECA000384606F576714C2201F022F843E0012B3C
:10ECB00007D106F5767039464C2201F019F8002389
:10ECC00002E0022B02D1012386F82434012384F8C8
:10ECD000253484F826340023C4F82834C4F82C34AE
:10ECE0009F4A94F82434C4F83074D35C9D4A1D4480
:10ECF00084F83534C4F8D423287984F83484FEF7B2
:10ED00005DF89949FEF762F9C4F83804A87BFEF76C
:10ED100055F89649FEF75AF9C4F83C04287EFEF7E8
:10ED20004DF89349FEF79EF8C4F84004FEF786FAC2
:10ED300000232876AB73B9F81E3143F08003A9F89D
:10ED40001E31012389F8443459E00027D5F8D40353
:10ED50003946FEF71BFA8046002850D1F8F7F0FF3D
:10ED60007E4BC5F8D47385F8D0831E7447E0B5F8A0
:10ED70001EA11AF0800F37D095F8D023774F511E7F
:10ED8000012924D87949D5F83C04FEF76BF8FEF741
:10ED900055FAD5F8306495F835847649B04488F84A
:10EDA0000A00D5F84004FEF75DF8FEF747FA88F848
:10EDB00014003078FEF702F80146FDF74BFFFEF72E
:10EDC0003DFAB37AB0703373337DB37505E0032A2F
:10EDD00003D185F8D0333E7402E03B7C01333B74B1
:10EDE0002AF08003A9F81E315B4B1B785A0706D422
:10EDF00099F844341BB1574B012283F8D123D9F839
:10EE00000481544A18F0080F5B4D38D0B2F82E1127
:10EE100001F145039BB28A2B2DD8B2F81E315B0756
:10EE200029D5B2F8AC03B2F8463499F84A61C21A4F
:10EE300092B293B218B2B330BCBF02F5B4739BB2B6
:10EE40001AB2B32AC4BFA3F5B4739BB2370795F8BF
:10EE5000EC00404A13D540B240424343D2F8B402DA
:10EE60001BB2007B43436FF01D0093FBF0F319448A
:10EE7000A2F82E1103E0B9F8AC33A9F8463418F023
:10EE8000040F00F09580B9F81E21324B160740F1AF
:10EE90008F8093F84A2102F0100202F0FF0052B175
:10EEA000B3F82C1195F92501D3F8382100FB021293
:10EEB000A3F82C217CE0D3F8B42292F8D71092F872
:10EEC000D62071B3B3F83071B3F928113EB2C1EB5B
:10EED000060EBEF1000FB8BFCEF1000E96450EDD56
:10EEE0008E42C8BF5242BFB2C8BF92B2C3F834010B
:10EEF0003A44012083F84804A9F8302158E093F8F7
:10EF000048242AB1D3F8242183F84804C3F82021E7
:10EF1000D9F83831B5F8D2201944B5F8D030994233
:10EF20003FE0B3F92801B3F93061361A86EAE67793
:10EF3000A7EBE677974221DD022296FBF2F601224B
:10EF4000C3F8A06283F8982283F8482421E000BF28
:10EF500080230020280100209623002000000020AC
:10EF6000702301080000A0410000204100007A4405
:10EF70005555553F9A99993FC01D002093F8482454
:10EF80003AB1D3F8242183F89812C3F8202183F8EA
:10EF90004814D9F83821B5F8D0300244B5F8D21069
:10EFA0009A4203DB8A42B4BF13460B46A9F83031BC
:10EFB000D9F8B462A64F96F8DAA0BAF1000F5CD087
:10EFC000B7F81E31980758D0B7F83001D7F88C231E
:10EFD0000490D7F88803D7F890B301460392FDF761
:10EFE00041FF039A0346114610460193FDF73AFF8D
:10EFF000019B01461846FDF72DFE5946034658462B
:10F000000193FDF72FFF019B01461846FDF722FEF5
:10F0100001F032FB01465846FDF7D8FF8D49834683
:10F02000FEF7C8F818BB584601F04CF9D7F84C1455
:10F03000FDF718FF01F0CAF8B0F5617FA8BF4FF4E3
:10F040006170FDF719FB80A3D3E90023FDF7A4FC51
:10F05000FDF7AAFD01F0F8F807465046FDF7AEFEB1
:10F060003946FDF7FFFE01F0B1F880B200E0002064
:10F07000DDF810A08244A9F830A118F0200F00F0AC
:10F080008B80B9F81E31DFF8C8A103F03003002BE4
:10F0900000F082809AF84A31D9077DD5BAF9AC03DD
:10F0A000FDF78CFE6C49FDF7DDFE074601F0CCF85C
:10F0B0000490384601F054F8DAF85034804693F85A
:10F0C00003B0BAF95A04654FBBF1000F34D0BAF857
:10F0D0005624CBF1000A93B212B2801A0193F3F7CF
:10F0E0005BFF5045019B03DB5845A8BF584600E035
:10F0F0005046B9F854140344B9F958048AB209B215
:10F100009BB2401AA9F8563403920193F3F744FFD7
:10F110005045039A019B03DB5845B4BF8246DA464B
:10F1200092441FFA8AFAA4F854A418B2FDF746FED6
:10F1300083460FFA8AF004E0FDF740FE8346BAF9F1
:10F140005804FDF73BFE414682465846FDF78AFECD
:10F150000499034650460193FDF784FE019B014646
:10F160001846FDF775FD3E49FDF730FFFEF740F804
:10F17000049938805846FDF775FE4146834650464F
:10F18000FDF770FE01465846FDF764FD3449FDF772
:10F190001DFFFEF72DF87880324B301D1F6806F1F9
:10F1A000500106F15C03B5F8F620B847FAF78CF881
:10F1B000D9F85C34002B60D0254B93F86034013BC8
:10F1C000142B55D8DFE803F00B5454275754541F21
:10F1D00054545454542F5454545454272F00D9F891
:10F1E00064345B782BB1204B00205989F3F725FF5D
:10F1F00043E01E4B1B7803F0040303F0FF00002BD9
:10F20000F1D10146F2E7184D0020E988F3F715FF28
:10F2100001202989EAE7144D00202989F3F70DFF21
:10F2200001206989E2E7104D0020E988F3F705FF26
:10F2300001202989F3F701FF02206989F3F7FDFE18
:10F240000320A989D2E700BFA2EB0FE5DD169640A7
:10F25000280100208FC2753C35FA8E3C9223002095
:10F26000000020419400002082000020962300200E
:10F27000AB689A0601D5F3F7EBFEF3F72AFAD14B08
:10F280001B78002B40F0B082DFF84C93D9F808309F
:10F290005B0540F1A982CC4E96F86834002B00F053
:10F2A000A382F3F739FD002800F09E8296F86934B6
:10F2B000002B00F09982D6F86C341B78002B40F0BC
:10F2C0005481D6F87004F3F7B1F9002840F04D816D
:10F2D000DFF80883D6F87424D8F800309A1A7C2A0C
:10F2E00040F24381C6F8743496F878340746013307
:10F2F00086F8783407F12400B34DC0B2F3F7B2F9C1
:10F3000005F5607333F91700FDF758FDAF4B8246E2
:10F310001888FDF753FD01465046FDF757FEAC49EE
:10F32000FDF7A0FDFDF764FF013700B2F3F7C6F962
:10F33000032FDFD13020F3F795F9B5F99002F3F7F9
:10F34000BDF9F3F79DF995F8780410F0030A29D177
:10F350001020F3F787F9D5F86C32642793FBF7F0A8
:10F3600000B2F3F7ABF92120F3F77CF9D5F86C3252
:10F3700093FBF7F007FB103787EAE770A0EBE77025
:10F3800000B2F3F79BF91420F3F76CF9B5F9AC036D
:10F39000F3F794F91C20F3F765F95046F3F78EF96B
:10F3A000F3F76EF996F87834874D5F0740F0B78031
:10F3B0000220F3F757F9B5F97A040A2790FBF7F022
:10F3C000F3F77CF9D9F80830980765D5DFF8109283
:10F3D00095F87C2499F8003040F63401B2FBF3F242
:10F3E0004A432A21B2FBF1F2B5F87E14062091FBC4
:10F3F000F3FA03FB1A1A4FEA0A1A1FFA8AFA4AEAC0
:10F40000022A1FFA8AFAC2F303224AEA020AF3F72F
:10F4100029F90FFA8AF0F3F751F9B5F87E2499F833
:10F420000030013292B292FBF3F103FB1123A5F8F5
:10F430007E3495F87C344FF06E0909FB03F91523EF
:10F4400099FBF3F93A204FF0640BF3F70BF9B9FB92
:10F45000FBFA5046F3F732F93B20F3F703F90BFBC5
:10F460001A9080B2053090FBF7F000B2F3F726F95E
:10F470002820F3F7F7F8D5F8800490FBF7F000B2F6
:10F48000F3F71CF90420F3F7EDF8D5F8840480F3C2
:10F49000100000B2F3F712F9D6F804314A4D99067C
:10F4A0003BD50FA9D5F88804F3F714FC1320F3F724
:10F4B000D9F8BDF93C00F3F701F91B20F3F7D2F8B6
:10F4C000BDF93E00F3F7FAF82320F3F7CBF8D5F8AF
:10F4D0008834002BACBF4E205320F3F7EFF80FA970
:10F4E000D4F88C04F3F7F6FB1220F3F7BBF8BDF960
:10F4F0003C00F3F7E3F81A20F3F7B4F8BDF93E0047
:10F50000F3F7DCF82220F3F7ADF8D4F88C34002BB5
:10F51000ACBF45205720F3F7D1F8F3F7B1F896F8D0
:10F520007834282B21D1284B0022D8F8005083F8BA
:10F5300078244FF47A73B5FBF3F817203C25F3F7E2
:10F5400091F8B8FBF5F7B7FBF5F005FB107000027A
:10F5500000B2F3F7B3F81820F3F784F805FB17802F
:10F5600000B2F3F7ABF8F3F78BF8D6F86C34164D1E
:10F570001B78012B40F01681F7F78CFAD5F8903400
:10F58000144AC31A9342064640F2A98095F87C2497
:10F59000002385F8B22485F8A82495F84A2185F837
:10F5A000963485F8983485F8B33485F8A93495F8FD
:10F5B000C034920785F8DB3414D42D2385F8DC346D
:10F5C0008AE000BF902300202801002000000020D6
:10F5D00000007A443F0D0300C01D0020BC1D002028
:10F5E00092000020042B8CBF3323322385F8DC34B7
:10F5F000C048D4F88854DFF83CC395FBF0F70CFB07
:10F6000007584FF0060E0EFB08F8BB4B07EB8707B9
:10F6100098FBF3F903FB198807EB87074FFA89F981
:10F62000D4F88C1409EB8707BFB291FBF0F084F893
:10F63000CB743F0A84F8CC740CFB00170EFB07F761
:10F64000ED0F84F8CA5497FBF3F503FB157364229E
:10F6500093FBF2F384F8D2341B1284F8D334B4F859
:10F66000EE3498FBF2F8B3FBF2F202EBC202920026
:10F6700092B2B4F8F03484F8C824120A84F8C92489
:10F6800084F8D434B4F8F2241B0A84F8D5340A235D
:10F69000B2FBF3F300EB800003F5FA739BB26DB29B
:10F6A00000EB800005EB800084F8D6341B0A80B2A2
:10F6B00084F8D734B4F8F43484F8CD84C90F4FEA11
:10F6C000282884F8D004000A84F8CE8484F8CF1463
:10F6D00084F8D10484F8DD34884BC3F89064874DF6
:10F6E00095F8F6842F46B8F1000F0DD1D5F8FC043B
:10F6F000F2F79CFF012807D90228814C00F0BD8257
:10F70000F2F799FF01236374D5F800257B4C002A9A
:10F7100048D094F8F6743FB1D4F8083540F6B731C4
:10F72000F31A8B420BD83DE00123D4F8FC040221EC
:10F7300084F8F634F2F766FF84F80C7530E094F83C
:10F7400004355BB9D4F8FC040121C4F8003584F811
:10F75000F634F2F757FFF2F76EFF21E0013BDBB220
:10F7600084F8043594F80C1594F80D0543B901306C
:10F770004B1C84F80D0584F80C35D4F8FC040DE01E
:10F78000134613F8012B0130114484F80D05D4F809
:10F79000FC0484F80C15C4F800351146F2F758FF44
:10F7A000C5F80865554CD4F86C341B78022B1BD176
:10F7B000D4F81035C3B1C4F814351B68514AC4F8E5
:10F7C0001835D4F81C3513449878FCF787F8D4F82A
:10F7D00014359879F7F783F8D4F81C350133092BE1
:10F7E00088BF0023C4F81C35DFF84CA1DAF80830D4
:10F7F000DC037EF50EA9414C94F820352546002BFC
:10F800003EF407A9404B1B78002B7EF402A9F7F7C2
:10F8100041F9D4F824350746C31ADB43DB0F0493C0
:10F82000D4F82835C31A6FEA0309D4F82C354FEA07
:10F83000D979C31A6FEA030B4FEADB7BBBF1000FE8
:10F8400006D1B9F1000F03D1049B002B3EF4E1A8CF
:10F850004FF0000895F8B4355FFA88F69E42DFF85D
:10F860009CC06BD22949DCF83035B20009681344DA
:10F870006244C2F834155988C8050BD48B0536D5B7
:10F88000234B1B785E0754BF224B234B1B68C2F8E7
:10F8900034352CE01946214A30460193CDF808C092
:10F8A000F9F7ACFBDDF808C0019BBCF81E2112F093
:10F8B000400F03D030461946194A16E0500703D5C9
:10F8C00030461946174A10E0110703D5304619464D
:10F8D000154A0AE0900703D530461946134A04E05A
:10F8E000D10704D5124A30461946F9F787FB08F1CB
:10F8F0000108AFE78096980040420F0028010020E1
:10F9000000000020702301088E230020B83C01086D
:10F91000962300207C23010880230108842301080A
:10F920008A23010890230108962301089C230108DB
:10F93000A2230108806967FFC01D00209E000023EC
:10F94000B3421FD0D5F83025B3491A445288520526
:10F9500016D501F23452D0580890B1F9BC0578217F
:10F96000A0F57A7048434FF47A7190FBF1F000F201
:10F970002B1040F2671190FBF1FE01FB1E01995222
:10F980000433DDE7BBF1000F28D007F5C333A03304
:10F99000C4F82C3594F8DA359F4EE3B986F8DB3598
:10F9A000DAF808304FF00108980786F8DA8504D5B0
:10F9B000F6F71EFF08B186F8DB85D4F8DC35964EE5
:10F9C0001B689B68984748B196F8DB3543F0020303
:10F9D00086F8DB3502E0002386F8DA3594F8DB257B
:10F9E0008D4B1AB9B9F1000F3DD160E093F8DAE51B
:10F9F000BEF1000F06D093F8E015013101F00301CC
:10FA000083F8E015002695F8B415F0B28142824BD8
:10FA1000E8D9D3F83015800001444988090620D57B
:10FA200093F8E015BEF1000F0CD121B9D10718D51C
:10FA300003447A4912E0012913D9910711D50344EF
:10FA400077490BE021B9D1070BD50344754905E08F
:10FA5000012906D9910704D5734903440968C3F8FD
:10FA600034150136CFE7B4F92C31B4F92A2132210B
:10FA7000002AB8BF5242002BB8BF5B4293FBF1F3A0
:10FA800092FBF1F1DBB2C9B28B4238BF0B46674A39
:10FA90000BB192FBF3F23A44C4F8282594F8E1251F
:10FAA0005D4B0AB9012200E0002283F8E12594F8B9
:10FAB000E125594B22B95E4AC3F8E425002009E04C
:10FAC000584AF9E7D3F8301594000E19768876066F
:10FAD00007D4013095F8B415C2B291424E4BF1D81B
:10FAE000A8E0B3F92A61322E21DD11F822E093F863
:10FAF000E8C50EF00F08E045D3F8E46508DC93F89C
:10FB0000E9C5BCEB1E1F03DC23443468C3F834454D
:10FB100011F8224095F8EAE504F00F0CF4453E4B4D
:10FB20002DDB93F8E9E5BEEB141F28DC22E032362A
:10FB300025DA11F822E093F8E8C50EF00F08E04549
:10FB4000D3F8E46508DC93F8EBC5BCEB1E1F03DBC0
:10FB500023443468C3F8344511F8224095F8EAE5A7
:10FB600004F00F0CF4452C4B09DB93F8EBE5BEEBEE
:10FB7000141F04DB346803EB8203C3F83445B5F982
:10FB80002C41254B322C1BDD11F822E093F8E8655F
:10FB90000EF00F0CB445D3F8E4450ADC93F8E9C540
:10FBA000BCEB1E1F05DCD4F800E003EB8203C3F8B6
:10FBB00034E511F8223003F00F01B1421EDD88E771
:10FBC000323486DA11F822E093F8EA650EF00F0C71
:10FBD000B445D3F8E4450ADB93F8E9C5BCEB1E1F36
:10FBE00005DCD4F800E003EB8203C3F834E511F838
:10FBF000223003F00F01B142FFF66BAF95F8EB1521
:10FC0000B1EB131FFFF665AF034B03EB82022368D2
:10FC1000C2F834355DE700BF28010020A8230108A1
:10FC2000AC230108B83C0108B0230108400D0300D3
:10FC3000B4230108049DE5B193F8ED2593F8EC1584
:10FC400007F543478818013890FBF2F402FB1400D3
:10FC500083F8EF15013183F8EE0591FBF2F002FB1A
:10FC600010125037D2B2C3F8247583F8F02583F808
:10FC7000EC25FAF77FF8FDF7CCBE637C23B1C5F81D
:10FC8000F86484F811803FE5D5F8F834F31AB3F539
:10FC90007A6FFFF439AD0123D5F8FC046374F2F7F1
:10FCA000C0FC0446D5F8FC04F2F7BBFC802C7FF4C2
:10FCB0002BAD8A2802D08E280DD025E5D5F8043149
:10FCC0009B067FF521AD95F8F634002B7FF41CAD33
:10FCD00007F2C14706E095F8F634002B7FF414AD27
:10FCE00007F294472D23C5F8007585F804350BE518
:10FCF00010B50023934203D0CC5CC4540133F9E720
:10FD000010BD02440346934202D003F8011BFAE7F8
:10FD1000704700000D4B70B51D680022845C2B19E4
:10FD20005B7803F00303012B8B5C08BF2034EE18D3
:10FD3000767806F00306012E08BF2033E41A02D1BC
:10FD40000132002BEAD1204670BD00BFB800002070
:10FD500010B50446224613780134002BFAD1CC5C4E
:10FD6000D4540133002CFAD110BDC9B2024610F8A8
:10FD7000013B1BB18B42F9D1104670470029FBD0E3
:10FD800018467047034613F8012B002AFBD1181AB6
:10FD9000013870470F4BF0B51E680023934215D011
:10FDA000C55C7419647804F00304012CCC5C08BFB2
:10FDB000203537197F7807F00307012F08BF20345B
:10FDC0002D1B04D10133002CE8D100E0002528468A
:10FDD000F0BD00BFB800002010B5034632B111F8E5
:10FDE000014B013A03F8014B002CF7D11A4493421E
:10FDF00003D0002103F8011BF9E710BD30B50378EB
:10FE00000BB1044604E00B78002B18BF002030BD76
:10FE100022461078013438B10023C85C28B1D55C83
:10FE20008542F5D10133F8E730BD104630BD0021E1
:10FE30000A2200F001B92DE9F04E82468B461F469A
:10FE4000144612B90020BDE8F08E002BFAD000262F
:10FE5000A642F7D2A5196D0807FB05B950464946D9
:10FE6000089B9847002802DB03D06E1C25462C46D1
:10FE7000EEE74846BDE8F08E174B2DE9F0411D68CE
:10FE80000646AC6D0F46FCB9502000F0E3F8A865BB
:10FE90008460AB6D046044601C61DC60AB6D9C6190
:10FEA0005C61AB6DDC629C62AB6D5C631C63AB6DD3
:10FEB000DC639C63AB6D5C641C64AB6DDC649C6454
:10FEC000AB6D1C77AB6D5C6230463946AA6D012381
:10FED000BDE8F04100F002B81C010020F0B508B9FF
:10FEE000106828B3044614F8015B0F4617F8016B3D
:10FEF0003EB1B542FAD10BB12046F3E7146003706E
:10FF0000F0BD4DB915602846F0BD17F8016BAE4243
:10FF100007D0002EF9D11C46234613F8015B0F468B
:10FF2000F3E715B10021217000E02B461360F0BD0E
:10FF3000F0BD000084463F482DE9F04FD0F8008026
:10FF40000E46344614F8015B08EB0500407800F0DB
:10FF5000080000F0FF0708B12646F2E72D2D03D177
:10FF6000B41C7578012703E02B2D04BF7578B41CF1
:10FF700033F010000DD1302D08D1207800F0DF00D3
:10FF8000582851D165781023023402E0002B08BFB5
:10FF90000A23002F0CBF6FF0004A4FF0004ABAFB53
:10FFA000F3F903FB19AA0026304608EB050B9BF872
:10FFB00001B01BF0040F01D0303D0BE01BF0030B30
:10FFC0001BD0BBF1010F14BF4FF0570B4FF0370B95
:10FFD000CBEB05059D4210DAB6F1FF3F0AD048454C
:10FFE00006D801D1554503DC03FB0050012601E092
:10FFF0004FF0FF3614F8015BD7E7731C0CD1002FCC
:020000040801F1
:100000004FF022030CBF6FF000404FF00040CCF8DF
:1000100000302AB9BDE8F08F07B1404242B106B1C5
:10002000611E1160BDE8F08F002B08BF0823B0E708
:10003000BDE8F08FB800002030B51346044A0546ED
:100040000C46106829462246BDE83040FFF772BFD3
:100050001C010020024B0146186800F003B800BFE5
:100060001C01002070B5CD1C25F0030508350C2DB2
:1000700038BF0C25002D06463FDB8D423DD3214B7A
:100080001C6818462146A1B10B685B1B0ED40B2BD4
:1000900003D90B60CC18CD501FE08C4202D16268AE
:1000A00002601AE04B6863600C4616E00C46496833
:1000B000E9E7154C23681BB9304600F027F82060AB
:1000C0002946304600F022F8431C014615D0C41CD6
:1000D00024F0030484420AD1256004F10B00231D9F
:1000E00020F00700C31A0BD05A42E25070BD3046D0
:1000F000611A00F00BF80130EED10C2333600020C0
:1001000070BD00BFA4230020A023002038B5064CFA
:10011000002305460846236000F008F8431C02D17E
:10012000236803B12B6038BDAC230020094A136853
:1001300063B118446946884202D810601846704777
:10014000054B0C221A604FF0FF307047034B1360D1
:10015000EFE700BFA8230020AC230020B02300203D
:1001600000B5194A20F00043934283B0014617DDE1
:10017000B3F1FF4F04DBFCF76BFD03B05DF804FB4C
:10018000694601F03BF800F00302012A009801994A
:1001900011D0022A0AD09AB1012201F0F3FDECE756
:1001A000002101F0F3F903B05DF804FB01F0EEF972
:1001B00000F10040E1E701F0E5FD00F10040DCE77F
:1001C00001F0E4F9D9E700BFD80F493F30B5C0F3DB
:1001D000C754A4F17F031E2B83B0014620DC581CBA
:1001E0001BDB162B4FEAD17509DDC1F3160040F475
:1001F0000000963CA04005B1404203B030BD114B19
:1002000053F825402046FCF725FD01900198214632
:10021000FCF71EFD20F0004333B9002003B030BDD1
:10022000FCF7E6FF03B030BDC0F31604C0F3C750BF
:1002300044F40004C0F1960024FA00F0002DDCD054
:10024000DAE700BF8C51010800B51D4A20F00043D9
:10025000934283B0014618DDB3F1FF4F04DBFCF796
:10026000F7FC03B05DF804FB694600F0C7FF00F03F
:100270000300012818D002280ED0D0B100980199AF
:1002800001F084F900F10040EBE70021002201F0C9
:1002900079FD03B05DF804FB00980199012201F09B
:1002A00071FD00F10040DCE70098019901F06EF962
:1002B000D7E700980199012201F064FDD1E700BF62
:1002C000D80F493F70B58AB0054600F023FA224C9A
:1002D000064694F90030013303D0284601F0C4FFEC
:1002E00010B930460AB070BD284601F06BFF4FF0E0
:1002F0007E51FCF773FF0028F3D018490122002338
:100300002846009208930191FCF7C8F902460B4673
:100310001348CDE90423CDE9022301F0ABFD94F9A4
:100320000030CDE90601022B0BD0684601F0A0FD9C
:1003300038B1089B53B9DDE90601FCF735FC0AB07A
:1003400070BD02F00FF821230360F2E702F00AF813
:10035000089B0360EFE700BF2001002094510108D3
:10036000A051010800F03EBB2DE9F0418AB00746DC
:100370000C4600F0C7FB9B4E054696F90030013352
:1003800003D0204601F070FF18B928460AB0BDE836
:10039000F081384601F068FF8046002832D12046BF
:1003A0000021FCF7F3FE0028EFD08F4A01233846E6
:1003B00001920093CDF82080FCF770F9CDE902019D
:1003C0002046FCF76BF9894B96F900400022CDE9F5
:1003D0000623631CCDE904010DD0022C0BD0684626
:1003E00001F046FD002800F09A80089B1BB101F047
:1003F000B9FF089B0360DDE90601FCF7D5FB0AB0F5
:10040000BDE8F08138460021FCF7C0FE18B3204655
:100410000021FCF7BBFE8046002855D0724901221E
:1004200000233846009208930191FCF737F9CDE993
:1004300002012046FCF732F996F900400022002321
:10044000CDE90401CDE90623002CC8D0674B00227A
:10045000CDE90623CFE7284601F0B8FE8046002804
:1004600062D028460021FCF791FE00288DD0384646
:1004700001F0ACFE002888D0204601F0A7FE00283D
:1004800083D05949042200233846009208930191F1
:10049000FCF704F9CDE902012046FCF7FFF896F9D4
:1004A000004000220023022CCDE90401CDE90623FF
:1004B00000F08880684601F0DBFC002800F08280B4
:1004C000089B002B97D092E7204601F07FFE002882
:1004D0003FF45BAF20460021FCF762FE00283FF4AA
:1004E00054AF414A0123384601920093CDF8208051
:1004F000FCF7D4F8CDE902012046FCF7CFF83478B8
:10050000CDE904010022002C30D0394B022CCDE97A
:1005100006232ED101F026FF21230360D0E701F04E
:1005200021FF2123036060E7384601F04FFE0028D9
:1005300097D0204601F04AFE002892D0284601F0CC
:1005400093FE0346D8B92849012238460893009201
:100550000191FCF7A3F8CDE902012046FCF79EF8D3
:100560003478CDE90401002C31D100220023CDE9FB
:100570000623684601F07CFC0028A1D1CAE71A4A8C
:100580000323384600930192CDF82080FCF786F8CB
:10059000CDE902012046FCF781F896F90030CDE95B
:1005A0000401384643BB134B4FF060420021CDE9B4
:1005B0000623FCF7F5FD00283FD196F90030022B09
:1005C0007FF478AF01F0CEFE2223036078E70020AD
:1005D000002102460B46FCF7DFF9022CCDE90601AB
:1005E00098D0C6E7200100209C5101080000F03F90
:1005F0000000F0FFFFFFEF471C4B00220021CDE978
:100600000623FCF7CDFD0028D7D020464FF07C51C3
:10061000FCF728FCFCF742F804460D4601F030FCDC
:1006200002460B4620462946FDF764F90028C4D14E
:100630000F4B0022CDE90623BFE720464FF07C5147
:10064000FCF710FCFCF72AF804460D4601F018FCF4
:1006500002460B4620462946FDF74CF90028ACD14E
:10066000044B4FF06042CDE90623A6E70000F07F7F
:100670000000F0FFFFFFEFC770B58AB0054600F03D
:1006800031FF224C064694F90030013308D0284649
:1006900001F0EAFD20B128460021FCF781FD10B9E8
:1006A00030460AB070BD1A49012200232846019144
:1006B00000920893FBF7F2FF2478CDE90401CDE91D
:1006C00002017CB900220023CDE90623684601F02F
:1006D000CFFB88B1089BA3B9DDE90601FCF764FAFA
:1006E0000AB070BD0020002102460B46FCF754F909
:1006F000022CCDE90601E9D101F034FE212303608B
:10070000E8E701F02FFE089B0360E5E720010020E9
:10071000A4510108F8B520F00043B3F17E5F044610
:1007200010D008DCB3F17C5F11DAB3F10C5F00F399
:1007300084809D48F8BD0146FCF78AFA0146FCF723
:1007400045FCF8BD002840F3CD800020F8BD00280E
:10075000C0F2CA8001464FF07E50FCF779FA4FF0A4
:100760007C51FCF77FFB044600F0BCFE8F49064637
:100770002046FCF777FB8E49FCF76CFA2146FCF724
:1007800071FB8C49FCF764FA2146FCF76BFB8A4944
:10079000FCF760FA2146FCF765FB8849FCF758FA3C
:1007A0002146FCF75FFB8649FCF754FA2146FCF72B
:1007B00059FB844905462046FCF754FB8249FCF767
:1007C00047FA2146FCF74EFB8049FCF743FA2146E5
:1007D000FCF748FB7E49FCF73BFA2146FCF742FB5D
:1007E0004FF07E51FCF736FA01462846FCF7EEFB47
:1007F0003146FCF737FB26F47F6525F00F050746E9
:1008000029462846FCF72EFB01462046FCF720FA35
:10081000294604463046FCF71DFA01462046FCF7FF
:10082000D5FB01463846FCF715FA01462846FCF789
:1008300011FA0146FCF70EFAF8BD0146FCF712FB6F
:100840005A490546FCF70EFB5949FCF703FA2946BD
:10085000FCF708FB5749FCF7FBF92946FCF702FBBC
:100860005549FCF7F7F92946FCF7FCFA5349FCF720
:10087000EFF92946FCF7F6FA5149FCF7EBF929465E
:10088000FCF7F0FA4F4906462846FCF7EBFA4E49CA
:10089000FCF7DEF92946FCF7E5FA4C49FCF7DAF9F2
:1008A0002946FCF7DFFA4A49FCF7D2F92946FCF75A
:1008B000D9FA4FF07E51FCF7CDF901463046FCF7EE
:1008C00085FB01462046FCF7CDFA01464148FCF77E
:1008D000BFF901462046FCF7BBF901463E48FCF74C
:1008E000B7F9F8BD3D48F8BD4FF07E51FCF7B2F9BD
:1008F0004FF07C51FCF7B6FA2C490446FCF7B2FAEB
:100900002B49FCF7A7F92146FCF7ACFA2949FCF77B
:100910009FF92146FCF7A6FA2749FCF79BF92146E7
:10092000FCF7A0FA2549FCF793F92146FCF79AFA5F
:100930002349FCF78FF92146FCF794FA0646204636
:1009400000F0D0FD1F4905462046FCF78BFA1E49F2
:10095000FCF77EF92146FCF785FA1C49FCF77AF989
:100960002146FCF77FFA1A49FCF772F92146FCF799
:1009700079FA4FF07E51FCF76DF901463046FCF7ED
:1009800025FB2946FCF76EFA1249FCF761F901468E
:100990002846FCF75FF90146FCF75CF90146104870
:1009A000FCF756F9F8BD00BFDB0FC93F08EF11385F
:1009B000047F4F3A4611243DA80A4E3E90B0A63E11
:1009C000ABAA2A3E2EC69D3D6133303F2D570140D4
:1009D00039D119406821A233DA0FC93FDB0F4940F2
:1009E000DA0F494021F00042B2F1FF4FF8B504465A
:1009F00014DC20F00045B5F1FF4F06460EDCB1F1E6
:100A00007E5F3AD08F1707F0020747EAD07755B9D3
:100A1000022F2FD0032F2FD13148F8BD0846214691
:100A2000FCF718F9F8BDFAB1B2F1FF4F29D0B5F1D2
:100A3000FF4F19D0AA1AD2153C2A19DC002938DB3D
:100A40002046FCF7C3FA01F0BDFB01F0A5FA012F27
:100A50002CD0022F22D0002F2FD02249FCF7FAF8F9
:100A60002149FCF7F5F8F8BD002E15DB1F48F8BD4D
:100A70001E48ECE71C48F8BDF8BDBDE8F84001F0A1
:100A80008BBAB5F1FF4F19D0022FF3D0032FC3D08B
:100A9000012F1BD00020F8BD1548F8BD1149FCF707
:100AA000D9F801461048FCF7D3F8F8BD00F1004032
:100AB000F8BD3C32C4DA0020C9E7F8BD022F0CD0E3
:100AC000032F08D0012F04D00A48F8BD4FF0004092
:100AD000F8BD0948F8BD0948F8BD0948F8BD00BF90
:100AE000DB0F49C02EBDBB33DB0F4940DB0FC93FD5
:100AF000DB0FC9BFDB0F493FDB0F49BFE4CB16C09B
:100B0000E4CB16402DE9F04F31F0004987B00D4697
:100B10000C46074611D020F0004ABAF1FF4F80463C
:100B200005DD514807B0BDE8F04F01F0B7BBB9F1A2
:100B3000FF4F07DDBAF17E5FF3D14FF07E5007B073
:100B4000BDE8F08F002840DB0026B9F1FF4F34D01C
:100B5000B9F17E5F4CD0B4F1804F384655D0B4F136
:100B60007C5F1BD001F02EFB0146BAF1000F1DD0B7
:100B700028F04043B3F17E5F18D04FEAD87808F1EF
:100B8000FF3856EA080166D0B9F19A4F74DD374B49
:100B90009A4533DC002C37DB0020D0E7B8F1000F9A
:100BA000E0DB07B0BDE8F04F00F09CBC002C41DB5F
:100BB000B8F1000F32DB0846C1E7BAF17E5FBCD066
:100BC00027DD002CE8DB2846B9E7B9F1974F13DAA7
:100BD000B9F17E5F0ADB4FEAE953C3F1960349FAA4
:100BE00003F202FA03F34B4500F044820026AFE71C
:100BF000002C25DB3846A2E70226A6E71C4B9A45C7
:100C000040F39D82002CC7DD1A480146FCF72AF903
:100C100095E7002CC0DA05F1004090E7AAF17E5A72
:100C200056EA0A0A12D10846FCF712F80146FCF708
:100C3000CDF984E74FF07E50FCF7C8F90146B7E7DD
:100C400039464FF07E50FCF7C1F978E7012EB2D15A
:100C500001F1004073E739463846FBF7F9FF0146DA
:100C6000FCF7B4F96BE700BFA0510108F7FF7F3F25
:100C70000700803FCAF24971BAF5000F80F2028284
:100C80004FF09741FCF7EEF86FF017028246B34B36
:100C90004FEAEA51CAF3160A7F399A4501EB020C72
:100CA0004AF07E5740F3EB81AD4B9A4540F34282C8
:100CB00000220CF1010CA7F5000705920599A94B3C
:100CC000384653F82130CDF804C0194603920493F6
:100CD000FBF7BEFF049981463846FBF7BBFF014690
:100CE0004FF07E50FCF772F90346194648460293CE
:100CF000FCF7B8F87910039A41F00051BB4601F5B2
:100D0000802120F47F6727F00F070A4482461146AE
:100D100038460392FCF7A6F801464846FBF798FFD1
:100D2000039A814604991046FBF792FF0146584604
:100D3000FBF78EFF01463846FCF794F8014648461B
:100D4000FBF786FF029B1946FCF78CF85146834659
:100D50005046FCF787F801468146FCF783F8824944
:100D6000034648460293FCF77DF88049FBF772FF83
:100D70004946FCF777F87E49FBF76CFF4946FCF7DC
:100D800071F87C49FBF766FF4946FCF76BF87A4936
:100D9000FBF760FF4946FCF765F87849FBF75AFF17
:100DA000029B01461846FCF75DF8394681465046DD
:100DB000FBF750FF5946FCF755F84946FBF74AFF49
:100DC000394604903846FCF74DF86D490390FBF71F
:100DD00041FF0499FBF73EFF20F47F6929F00F09DA
:100DE00049463846FCF73EF8494607465846FCF760
:100DF00039F8634983464846FBF72AFF039A1146B0
:100E0000FBF726FF01460498FBF722FF5146FCF74B
:100E100029F801465846FBF71DFF834659463846D8
:100E2000FBF718FF20F47F6A2AF00F0A5046554955
:100E3000FCF718F8544981465046FCF713F8394638
:100E4000034650460293FBF703FF01465846FBF763
:100E5000FFFE4E49FCF706F8029B01461846FBF7D9
:100E6000F9FE4B4B059A53F82210FBF7F3FEDDF821
:100E700004C007466046FBF7A1FF464B059A049065
:100E800053F822B039464846FBF7E4FE5946FBF7D3
:100E9000E1FE0499FBF7DEFE20F47F6A2AF00F0AD8
:100EA00004995046FBF7D4FE5946FBF7D1FE49465C
:100EB000FBF7CEFE01463846FBF7CAFE24F47F64FA
:100EC00024F00F04013E56EA0806814621462846D2
:100ED0000CBF314F4FF07E57FBF7BAFE5146FBF780
:100EE000C1FF494606462846FBF7BCFF014630468F
:100EF000FBF7B0FE214606465046FBF7B3FF05461A
:100F000001463046FBF7A6FE00288146044620F045
:100F10000048AA4640F3F880B8F1864F00F3C2803B
:100F200000F0B280B8F17C5F00F3C4804FF000099C
:100F3000C84624F47F6424F00F0420461749FBF7C9
:100F400091FF514605462046FBF782FE014630469A
:100F5000FBF77EFE1249FBF785FF23E071C41C00FE
:100F6000D6B35D00BC51010842F1533E55326C3E90
:100F700005A38B3EABAAAA3EB76DDB3E9A99193FFB
:100F8000000040400038763FA0C39D364F38763F82
:100F9000B4510108AC510108000080BF0072313F1C
:100FA0001872313F864906462046FBF75BFF014633
:100FB0003046FBF74FFE064631462846FBF74AFE11
:100FC00029460446FBF744FE01463046FBF740FE47
:100FD000214606462046FBF745FF7A490546FBF7C2
:100FE00041FF7949FBF734FE2946FBF73BFF774980
:100FF000FBF730FE2946FBF735FF7549FBF728FE66
:101000002946FBF72FFF7349FBF724FE2946FBF720
:1010100029FF01462046FBF71BFE054629462046D0
:10102000FBF720FF4FF0804182462846FBF710FE79
:1010300001465046FBF7CAFF314605462046FBF7FE
:1010400011FF3146FBF706FE01462846FBF700FE7E
:101050002146FBF7FDFD01464FF07E50FBF7F8FD02
:101060008144B9F5000FC0F2A58049463846FBF728
:10107000F9FE64E502F00102C2F1020668E5002211
:1010800005921BE6002202E653493046FBF7E2FDDB
:10109000294682464846FBF7DBFD01465046FCF7F1
:1010A0009DF838B138464D49FBF7DCFE4B49FBF75C
:1010B000D9FE44E54FEAE858A8F17E084FF4000352
:1010C00043FA08F32344C3F3C7524548C3F3160851
:1010D000A2F17F0140FA01F1C2F1960248F4000842
:1010E00048FA02F8002C23EA01012846B8BFC8F1EB
:1010F0000008FBF7ADFD824651463046FBF7AAFDDE
:101100004FEAC859044614E7364B98450ADC7FF489
:1011100009AF2946FBF79CFD01463046FCF74AF82B
:101120000028C7D038463049FBF79CFE2E49FBF714
:1011300099FE04E501234FF400120593BEE54FF03C
:101140007E51FBF785FD29490746FBF78BFE2849B1
:1011500081463846FBF786FE394682463846FBF71D
:1011600081FE4FF07A5183463846FBF77BFE0146FD
:101170002048FBF76DFD3946FBF774FE01464FF042
:101180007C50FBF765FD01465846FBF76BFE1A499C
:10119000FBF768FE01465046FBF75AFD0746394605
:1011A0004846FBF757FD20F47F6A2AF00F0A4946AC
:1011B00050467DE6414601F075F8014656E700BF0E
:1011C0008CBEBF354CBB31330EEADD3555B38A38A2
:1011D000610B363BABAA2A3E3CAA3833CAF24971AE
:1011E000FFFF7F00000016436042A20D00AAB83F37
:1011F00070A5EC36ABAAAA3E3BAAB83F2DE9F04F4A
:10120000AB4A20F00044944289B006460D4664DDA6
:10121000A84A94421CDC0028A74940F3EC80FBF765
:1012200017FDA64B24F00F049C42064664D0A44947
:10123000FBF70EFD014628603046FBF709FDA0498B
:10124000FBF706FD01236860184609B0BDE8F08F82
:101250009C4A944262DDB4F1FF4F46DAE715863FBF
:10126000A4EBC7542046FBF7C3FFFBF7A7FD0346DB
:10127000014620460593FBF7EBFC4FF08741FBF757
:10128000F1FD8046FBF7B4FFFBF798FD01460446ED
:1012900040460694FBF7DCFC4FF08741FBF7E2FD8C
:1012A00000210790FBF772FF002800F0C580204660
:1012B0000021FBF76BFF002814BF012302238248A3
:1012C0000221019000913A4605A8294600F022FA31
:1012D000002EC0F2A780034603E00022286000230E
:1012E0004A60184609B0BDE8F08F0146FBF7B0FC34
:1012F000002368602860F4E77449FBF7A9FC74498F
:101300000446FBF7A5FC014628602046FBF7A0FC3D
:101310006F49FBF79DFC01236860E2E700F052FF94
:101320006C490746FBF79EFD4FF07C51FBF792FCA2
:10133000FBF75EFF8246FBF741FD5F498346FBF703
:1013400091FD01463846FBF783FC5D4980465846CF
:10135000FBF788FDBAF11F0F81464946404618DC6D
:101360005D4B0AF1FF3253F8223024F0FF029A421B
:101370000FD0FBF76DFC07462F6039464046FBF760
:1013800067FC4946FBF764FC002E686056DB534659
:10139000A7E7FBF75DFCE315C0F3C7529A1A082ACA
:1013A0000746E9DD494958460393FBF75BFD0746CD
:1013B00039464046FBF74CFC044621464046FBF7C5
:1013C00047FC3946FBF744FC414907465846FBF7C2
:1013D00049FD3946FBF73CFC814649462046FBF770
:1013E00037FC039BC0F3C7529B1A192B074641DCFD
:1013F0002860A046C1E7FBF72DFC304B24F00F041A
:101400009C42064623D02E49FBF724FC0146286067
:101410003046FBF71DFC2A49FBF71CFC4FF0FF335D
:1014200068605EE795E80C0003F1004102F10042BC
:1014300043422A60696054E7032340E707F100470D
:1014400000F100402F606860CAF1000349E71F49BE
:10145000FBF700FC1E490446FBF7FCFB0146286035
:101460002046FBF7F5FB1A49FBF7F4FB4FF0FF337F
:10147000686036E719495846FBF7F4FC07463946D9
:101480002046FBF7E5FB804641462046FBF7E0FBA4
:101490003946FBF7DDFB124904465846FBF7E2FCF0
:1014A0002146FBF7D5FB81464946404661E700BF30
:1014B000D80F493FE3CB1640800FC93FD00FC93F3B
:1014C00043443537800F49434452010800443537BF
:1014D00008A3852E84F9223FC451010800A3852E5C
:1014E00032318D2420F00042B2F1FF4FF8B50446AE
:1014F00003462DD25AB300283DDBB2F5000F4FEA68
:10150000E0502CD37F38C3F31603C20743F4000323
:1015100048BF5B00002740105B003E4619244FF097
:101520008072B5189D4202DC5B1BAE181744013C6B
:101530004FEA43034FEA5202F3D113B107F001031C
:101540001F447F1007F17C5707EBC050F8BDF8BD72
:101550000146FBF787FC2146FBF77CFBF8BD14F442
:1015600000020FD15B00190202F10102FAD5C2F1AB
:1015700001021044C6E70146FBF76AFB0146FBF790
:1015800025FDF8BD01221044BCE700BF2DE9F8435A
:1015900020F00046B6F1485F05460F4649DAFBF7F2
:1015A00027FE002800F09D8029462846FBF75AFCBC
:1015B0004E490446FBF756FC4D49FBF74BFB2146D1
:1015C000FBF750FC4B49FBF743FB2146FBF74AFC7A
:1015D0004949FBF73FFB2146FBF744FC4749FBF732
:1015E00037FB2146FBF73EFC4549FBF733FB214621
:1015F000FBF738FC804620464FF07C51FBF732FC6D
:10160000414606462046FBF72DFC3946044628464F
:10161000FBF728FC01462046FBF71AFB0146304643
:10162000FBF716FB01464FF07E50FBF711FBBDE8C0
:10163000F8830146FBF716FC2C490446FBF712FC25
:101640002B49FBF707FB2146FBF70CFC2949FBF76D
:10165000FFFA2146FBF706FC2749FBF7FBFA214678
:10166000FBF700FC2549FBF7F3FA2146FBF7FAFBF1
:101670002349FBF7EFFA2146FBF7F4FB214B8046A9
:101680009E42B8DD204B9E4227DC06F17F46314664
:101690004FF07E50FBF7DCFA814620464FF07C513C
:1016A000FBF7E0FB3146FBF7D3FA414606462046FE
:1016B000FBF7D8FB394604462846FBF7D3FB014627
:1016C0002046FBF7C5FA01463046FBF7C1FA014652
:1016D0004846FBF7BDFABDE8F883DFF834900B4EBF
:1016E000DBE74FF07E50BDE8F88300BF4ED747AD33
:1016F000F6740F317CF29334010DD037610BB63A9A
:10170000ABAA2A3D9999993E0000483F0000903EBF
:101710000000383F2DE9F04FDFB00B93013B0293FF
:10172000D31E48BF131DB84C06466898DB1054F80A
:10173000204023EAE3730C93DB4302EBC3030894DA
:101740000693089C029B0C9A1D190991C3EB020792
:101750001DD4699C3D4404EB870901354FF0000816
:1017600022AC0AE059F80800FBF728FB0137AF422A
:1017700044F8080008F1040809D0002FF2DA013714
:101780000020AF4244F8080008F10408F5D1089A97
:10179000002AC0F2DF82089A0B9B02F101089C002C
:1017A00022AF4FEA880827440025029A002AC0F297
:1017B000F28105EB070B4FF000094FF0000A56F8D5
:1017C00009005BF8041DFBF74DFB01465046FBF793
:1017D00041FA09F10409A1458246F0D14AA840F82E
:1017E00005A004354545E0D1089A0EAB03EB820312
:1017F0000D9391464FEA89030793079A5EAB134412
:10180000B9F1000F53F850AC23DD0DF134084AAFA5
:10181000174490440DAD4FF06E515046FBF722FB3C
:10182000FBF7E6FCFBF7CAFA4FF087418346FBF76C
:1018300019FB01465046FBF70BFAFBF7D9FC59465A
:1018400045F8040F57F8040DFBF704FA45458246A6
:10185000E1D15046069900F025FD4FF0785105463C
:10186000FBF700FB00F0BAFC4FF08241FBF7FAFAFD
:1018700001462846FBF7ECF90546FBF7B9FC824622
:10188000FBF79CFA01462846FBF7E2F9069A8046E8
:10189000002A40F3678109F1FF310EA850F821308A
:1018A000C2F1080043FA00F202FA00F01B1A06988F
:1018B0009244C0F1070743FA07F70EA840F8213019
:1018C000002F32DDB9F1000F0AF1010A40F37581F2
:1018D0000EAB079A19461144002507E0C2F5807047
:1018E00012B143F8040C01258B420BD053F8042BA2
:1018F000002DF3D0C2F1FF028B4243F8042C4FF0CD
:101900000105F3D1069B002B0DDD012B00F0328188
:10191000022B08D109F1FF330EA951F8232002F060
:101920003F0241F82320022F70D040460021FBF7F0
:101930002DFC002800F08380089A09F1FF35AA42A7
:101940000DDC079A0EAB0D981344002253F8041DCA
:10195000834242EA0102F9D1002A40F0E481089B67
:101960000EA85A1E50F82230002B40F0F18100EBF7
:101970008202012352F8041D01330029FAD04B449E
:1019800099450A933DDADDF82CA022AACA44DDF875
:10199000308002EB8A02C844C9EB0309131D03928D
:1019A0000593699A079B4FEA89094AAF02EB8808B9
:1019B000CDF810901F44002558F8040FFBF7FEF9EE
:1019C000029B039A002B50514FF0000B13DBDDF804
:1019D00014A04FF00009AA4456F809005AF8041D53
:1019E000FBF740FA01465846FBF734F909F10409C0
:1019F000A1458346F0D1049A0435954247F804BFC7
:101A0000DAD1DDF82890F5E65C55010841464FF043
:101A10007E50FBF71DF98046002D86D006994FF0C9
:101A20007E5000F03FFC01464046FBF711F980462E
:101A300040460021FBF7AAFB00287FF47DAF069B00
:101A400040465942CDF808A000F02CFC4FF08741E9
:101A50000446FBF7B9FB002800F07F814FF06E5180
:101A60002046FBF7FFF9FBF7C3FBFBF7A7F94FF0A5
:101A700087410546FBF7F6F901462046FBF7E8F8F3
:101A8000FBF7B6FB0EAB43F829002846FBF7B0FB8B
:101A9000069C09F1010508340EA9069441F82500B9
:101AA00006994FF07E5000F0FDFB002D04464FDB01
:101AB0006E1C4FEA8508C6EB867A0DF138094AABF1
:101AC000C1444FEA8A0A98444FF0000B59F80B00C2
:101AD000FBF774F92146FBF7C5F94FF06E5148F852
:101AE0000B002046FBF7BEF9ABF1040BD3450446CF
:101AF000ECD1DFF88C92DDF820A00024B3460395EA
:101B00000497BAF1000FB8BF002515DB0026374651
:101B1000002501E0A7420FDC58F8061059F806002E
:101B2000FBF7A0F901462846FBF794F80137BA45C0
:101B3000054606F10406EDDA5EA800EB84030134E5
:101B4000A345A8F1040843F8A05CDAD1039D049FE3
:101B5000689C032C00F29880DFE814F0CB009C0016
:101B60009C00310010D109F1FF330EA951F8237008
:101B70003F12A5E609F1FF330EA850F8232002F02A
:101B80007F0240F82320CEE64FF07C51FBF71CFB90
:101B900058B90746C9E64FF0000A4AA840F805A020
:101BA000043545457FF401AE1EE6B9F1000F4FF054
:101BB00002070AF1010A3FF78BAE0025A2E6002DCD
:101BC00040F3DC804FEA850B5EAB36AE05F1FF3AA1
:101BD0005B4406EB8A0A53F8A08C54465B4635AA50
:101BE000BB462F4600E0C84654F8045941462846F3
:101BF00001920093FBF72EF8814649462846FBF7F1
